:0200000480007A
:10000000970500009385856B130540006B10B500C4
:10001000EF00806A130510006B0005001385E18F67
:1000200017160D00130646F53306A640930500008B
:10003000EF00585B17E507001305451EEFD0C77AA0
:10004000EFF0174F130540006B000500EF10002084
:040050006FD0D71185
:10005400130101FF1305400023261100EF6005265C
:10006400B7270B809387C7F337660580B7250B80C6
:100074002320F500130606D5938585F2EFA0C30C63
:10008400130101FF1305400023261100EF6005232F
:10009400B7270B80938787F737660580B7250B80D2
:1000A4002320F500130686D9938545F6EFA0C309EE
:1000B400130101FE2326A10013058000232C8100D7
:1000C400232E1100232A9100EF60451F8325C100D0
:1000D40013040500EFF0051037A60580B7250B8043
:1000E400130606539385857113050400EFA0C30519
:1000F4009304050013050400EF60C5211385040073
:10010400EFB09767130101FE2326A10013058000B9
:10011400232C8100232E1100232A9100EF60051A5D
:100124008325C10013040500EFF0451037A60580B0
:10013400B7250B8013068656938585731305040033
:10014400EFA083009304050013050400EF60851CF1
:1001540013850400EFB05762130101FE2326A100AA
:1001640013058000232C8100232E1100232A9100E3
:10017400EF60C5148325C10013040500EFF00511D9
:1001840037A60580B7250B80130686589385857797
:1001940013050400EF90537B93040500130504003A
:1001A400EF60451713850400EFB0175D130101FFDD
:1001B4001305400023261100EF604510B7270B807C
:1001C400938787F737660580B7250B802320F500D2
:1001D400130686D9938545F6EF901377130101FF33
:1001E4001305400023261100EF60450DB7570B801F
:1001F4009387872137260780B7550B802320F50086
:10020400130686F593854520EF901374130101FDC1
:100214002326A10013058001232611022324810231
:1002240023229102EF60850913040500EF10560D97
:100234008325C10093071000232EA100130681011A
:1002440013050400232CF100EF105656B7470B801A
:10025400938787AF130504002320F400EFA0852CB7
:100264009305050013050401EF7097086F00000261
:100274009304050013050400EF10961213050400FF
:10028400EF60450913850400EFB0174F3726068049
:10029400B7450B80130646C7938505AA13050400CA
:1002A400EF90936A930405006FF05FFD130101FE64
:1002B400232821011309050013058001232C810043
:1002C400232A9100232E110093840500EF50157FFB
:1002D4001304050063820402EF1097462326A1004D
:1002E40013068100930509001305040023249100DB
:1002F400EF10D64B6F000001EF109600930410002E
:100304006FF0DFFDB7470B80938787AF13050400B9
:100314002320F400EFA00521930505001305040133
:10032400EF70077D6F0000029304050013050400BD
:10033400EF10160713050400EF50D57D1385040054
:10034400EFB0974337260680B7450B80130646C7A0
:10035400938505AA13050400EF90135F9304050029
:100364006FF05FFD03C701966316070013071000C3
:100374002380E19603C781956316070013071000D5
:10038400238CE19403C7019563160700130710003B
:100394002388E19403C781946316070013071000B0
:1003A4002384E19403C70194631607001307100024
:1003B4002380E19403C78193631607001307100099
:1003C400238CE19203C701936316070013071000FF
:1003D4002388E19203C78192631607001307100074
:1003E4002384E19203C701926316070013071000E8
:1003F4002380E19203C7819163160700130710005D
:10040400238CE19003C701916316070013071000C2
:100414002388E19003C78190631607001307100037
:100424002384E1906780000003C7019F63160700DF
:10043400130710002388E19E03C7819E63160700FB
:10044400130710002384E19E03C7019E631607006F
:10045400130710002380E19E03C7819D63160700E4
:1004640013071000238CE19C03C7019D631607004A
:10047400130710002388E19C03C7819C63160700BF
:10048400130710002384E19C03C7019C6316070033
:10049400130710002380E19C03C7819B63160700A8
:1004A40013071000238CE19A03C7019B631607000E
:1004B400130710002388E19A03C7819A6316070083
:1004C400130710002384E19A03C7019A63160700F7
:1004D400130710002380E19A03C78199631607006C
:1004E40013071000238CE19867800000130101FFBB
:1004F40023229100B71400002324810093840494E0
:1005040037040D801304C40213850400232611004C
:1005140023269400EFF0973F2324A40063100502E0
:1005240023260400232204008320C1000324810025
:100534008324410013010101678000002322A400E9
:1005440023209500232205006FF01FFE03C701B787
:1005540063160700130710002388E1B603C781B6AA
:1005640063160700130710002384E1B603C701B61E
:1005740063160700130710002380E1B603C781B593
:100584006316070013071000238CE1B403C701B5F9
:1005940063160700130710002388E1B403C781B46E
:1005A40063160700130710002384E1B403C701B4E2
:1005B40063160700130710002380E1B403C781B357
:1005C4006316070013071000238CE1B26780000054
:1005D40003C701BD63160700130710002388E1BC9D
:1005E40003C781BC63160700130710002384E1BC12
:1005F40003C701BC63160700130710002380E1BC86
:1006040003C781BB6316070013071000238CE1BAEC
:1006140003C701BB63160700130710002388E1BA60
:1006240003C781BA63160700130710002384E1BAD5
:1006340003C701BA63160700130710002380E1BA49
:1006440003C781B96316070013071000238CE1B8B0
:1006540067800000130101FF2324810037E40C802C
:1006640037250780130684BF9385018E1305C5E3E0
:1006740023261100EFD0872D130684BF03248100A5
:100684008320C100372507809385C18D130585E339
:10069400130101016FD0872BB70700009387070070
:1006A4006388070037E50780130585216FD087131A
:1006B40067800000130540006B00050097F10C00F3
:1006C40093818181F32610029396A601732600027A
:1006D4009315A6001316260037F1FF6F3301B140BE
:1006E4003301D1403301C100F326100263860600B2
:1006F400130500006B00050067800000130101FE74
:10070400232E8100130401022326A4FE9307000074
:10071400138507000324C10113010102678000004F
:10072400130101FE232E1100232C81001304010266
:100734002326A4FE2324B4FE2322C4FE2320D4FEB5
:1007440083A7418E03A7C7000326C4FEB7670A80A8
:100754009385073C13050700EFD0D75B1300000017
:100764008320C10103248101130101026780000079
:10077400130101DF23261120232481202322912029
:100784001304012137C3FFFF33016100B7C7FFFF23
:10079400130704FFB307F70023A6A7E0B7C7FFFFBB
:1007A400130704FFB307F70023A4B7E0B7C7FFFF9D
:1007B400130704FFB307F70023A2C7E0B7C7FFFF7F
:1007C400130704FFB307F700130744EE1306800072
:1007D40083A547E013050700EFB04344930744EEB5
:1007E40013850700EFA043679307050093C717001D
:1007F40093F7F70F63880704B7670A809385473E2A
:10080400B7070D80138547C4EF70542813070500FC
:10081400B7C7FFFF930604FFB387F60083A547E03D
:1008240013050700EF70942613070500B7870480AB
:10083400938507D813050700EF70C40E93040000D6
:100844006F0040199307C4E113850700EF80C45576
:10085400930744EE13850700EFA0835F1307050099
:100864009307C4E19305070013850700EF70C431B3
:10087400930744E01307C4E19305070013850700B9
:10088400EF808479930744E013850700EF901458B0
:10089400930705002320F4E0130604E0B7C7FFFF25
:1008A400130704FFB307F7001307000093060000C3
:1008B4009305100003A5C7E0EF509040930705008F
:1008C4002326F4FE8327C4FE639A0702B7670A80CF
:1008D40093858740B7070D80138547C4EF70141BB9
:1008E40013070500B7870480938507D8130507000D
:1008F400EF704403930400006F00400C9307000062
:10090400130700009306000013060000930500007F
:100914000325C4FEEF70905D930705002324F4FEC5
:10092400832784FE638A0708B7C7FFFF938707E11D
:10093400130704FF3307F700B7C7FFFF930604FF4D
:10094400B385F60093070000B74600003716000091
:100954001306361883A585E00325C4FEEF900160D5
:10096400B7670A8093854743B7070D80138547C44B
:10097400EF70D41113070500B7870480938507D857
:1009840013050700EF60147AB7C7FFFF938707E1E9
:10099400130704FFB307F70093850700B7070D801B
:1009A400138547C4EF70940E0325C4FEEF70C0573F
:1009B400930400006F0080008324C4FE930744E086
:1009C40013850700EF90441A9307C4E113850700C9
:1009D400EF804455930744EE13850700EFB0C30935
:1009E400938704006F00800493040500930744E098
:1009F40013850700EF9044176F00800093040500EF
:100A04009307C4E113850700EF80C4516F00800091
:100A140093040500930744EE13850700EFB0C30564
:100A24009387040013850700EFB00755138507006B
:100A340037430000330161008320C1200324812057
:100A4400832441201301012167800000130101FB6D
:100A54002326110423248104232291041304010571
:100A6400232EA4FA232CB4FA232AC4FAB7670A80E3
:100A740013858744EF00C84F13054000EF90437A75
:100A840093070500232CF4FC13070000832684FD40
:100A940013064000B7170000938537160325C4FBDF
:100AA400EFB0D10E93070500232AF4FCB7670A8040
:100AB40013854746EF00C84B832744FD6382070430
:100AC400B7670A809385C747B7070D80138547C466
:100AD400EF70C47B13070500B7870480938507D89C
:100AE40013050700EF601464832784FD6386070001
:100AF400032584FDEF801337930700006F00003B4C
:100B040013054000EF90C371930705002328F4FCFC
:100B140013070000832604FD13064000B7170000E6
:100B2400938557160325C4FBEFB0510693070500C0
:100B3400232AF4FCB7670A8013858749EF004843EA
:100B4400832744FD638A0704B7670A809385474B6C
:100B5400B7070D80138547C4EF704473130705006E
:100B6400B7870480938507D813050700EF60945B6B
:100B7400832784FD63860700032584FDEF80932E7D
:100B8400832704FD63860700032504FDEF80932D6E
:100B9400930700006F00803113054000EF90436815
:100BA400930705002326F4FC232604FE8327C4FEB2
:100BB400639407048327C4FE93972700032704FD47
:100BC400B307F70083A607008327C4FE9397270083
:100BD4000327C4FCB304F70013850600EF904364B5
:100BE4009307050023A0F4008327C4FE938717000E
:100BF4002326F4FE6FF09FFB130700008326C4FC3A
:100C040013064000B7170000938567160325C4FB3D
:100C1400EFB0C17793070500232AF4FCB7670A8075
:100C24001385074EEF00C834832744FD638A070AFF
:100C3400B7670A809385874FB7070D80138547C42C
:100C4400EF70C46413070500B7870480938507D841
:100C540013050700EF60144D832784FD63860700A6
:100C6400032584FDEF801320832704FD638607009A
:100C7400032504FDEF80131F232404FE832784FE31
:100C840063940704832784FE939727000327C4FCF7
:100C9400B307F70083A7070063800702832784FE56
:100CA400939727000327C4FCB307F70083A7070023
:100CB40013850700EF80131B832784FE9387170097
:100CC4002324F4FE6FF09FFB8327C4FC6386070094
:100CD4000325C4FCEF801319930700006F00001D67
:100CE400232204FE832744FE63900714832744FED3
:100CF40093972700032784FDB307F70083A7070012
:100D0400032784FB631AF710B7670A809385C751DA
:100D1400032544FBEFD0477B930705002324F4FC11
:100D2400832784FC63960708832784FD6386070072
:100D3400032584FDEF801313832704FD63860700D6
:100D4400032504FDEF801312232004FE832704FEF1
:100D540063940704832704FE939727000327C4FCA6
:100D6400B307F70083A7070063800702832704FE05
:100D7400939727000327C4FCB307F70083A7070052
:100D840013850700EF80130E832704FE9387170053
:100D94002320F4FE6FF09FFB8327C4FC63860700C7
:100DA4000325C4FCEF80130C930700006F000010B0
:100DB400B7670A8013850752EF00881B832744FE18
:100DC400939727000327C4FCB307F70003A5070084
:100DD400832744FE93972700032704FDB307F700F6
:100DE40083A70700832684FC13860700930510005D
:100DF400EFE0D74BB7670A8013850753EF00481716
:100E0400032584FCEFC0574AB7670A801385C7538C
:100E1400EF0008166F004001832744FE93871700F4
:100E24002322F4FE6FF01FEC832784FD6386070002
:100E3400032584FDEF801303832704FD63860700E5
:100E4400032504FDEF801302232E04FC8327C4FD35
:100E5400639407048327C4FD939727000327C4FCE6
:100E6400B307F70083A70700638007028327C4FD45
:100E7400939727000327C4FCB307F70083A7070051
:100E840013850700EF80037E8327C4FD9387170033
:100E9400232EF4FC6FF09FFB8327C4FC63860700BA
:100EA4000325C4FCEF80037C93071000138507001F
:100EB4008320C10403248104832441041301010514
:100EC40067800000130101FC232E1102232C8102F0
:100ED4001304010437C3FFFF33016100B7C7FFFFE9
:100EE400130704FFB307F70023AEA7FCB7C7FFFF40
:100EF400130704FFB307F70023ACB7FCB7C7FFFF22
:100F0400130704FFB307F70023AAC7FCB7C7FFFF03
:100F1400130704FFB307F70037670A809305875464
:100F240003A547FDEFD0475A930705002326F4FE97
:100F34008327C4FE63960700930700006F004022D6
:100F440013062000930500000325C4FEEFD0D765E7
:100F54000325C4FEEFE08735930705002322F4FE42
:100F64000325C4FEEF10483C832744FE1385070085
:100F7400EF90032B930705002320F4FE832704FE40
:100F8400032744FE8326C4FE1306070093051000BE
:100F940013850700EFD0D71A0325C4FEEFC0D7305E
:100FA400232E04FC1308C4FD930584FD130704FEDB
:100FB400930644FEB7C7FFFF938787FD130604FF1C
:100FC4003306F600B7C7FFFF130504FF3305F5002A
:100FD40093870500930510000325C5FDEF60506E4F
:100FE400930705002324F4FE832704FE6388070087
:100FF400832704FE13850700EF80C3668327C4FD9F
:10100400638A0702B7670A809385C754B7070D80C0
:10101400138547C4EF70842713070500B78704803E
:10102400938507D813050700EF60D40F93070000DA
:101034006F000013832784FD638A0702B7670A8061
:101044009385C756B7070D80138547C4EF700424F2
:1010540013070500B7870480938507D81305070095
:10106400EF60540C930700006F00800FB7C7FFFFB9
:10107400938787FD130704FF3306F70093070000E7
:10108400130700009306000093051000032584FE57
:10109400EF70C06593070500232EF4FC8327C4FD7D
:1010A400638E070A8327C4FD93850700B7670A8008
:1010B40013858758EFF0D76BB7C7FFFF130704FFFB
:1010C400B307F70083A587FDB7C7FFFF938787FEA4
:1010D400130704FF3307F70093070000B746000027
:1010E4003716000013063618032584FEEF801167B7
:1010F400B7670A809385C759B7070D80138547C41E
:10110400EF70C41813070500B7870480938507D8C8
:1011140013050700EF601401B7C7FFFF938787FE2D
:10112400130704FFB307F70093850700B7070D8083
:10113400138547C4EF70841513070500B78704802F
:10114400938507D813050700EF60C47D032584FE4B
:10115400EF60905D930700006F008000832784FE9A
:101164001385070037430000330161008320C10366
:10117400032481031301010467800000130101FCAF
:10118400232E1102232C810213040104232EA4FC18
:10119400232CB4FC232AC4FC2328D4FC2326E4FCFB
:1011A400232604FE0327C4FE9307200063C4E70438
:1011B4008327C4FE939727000327C4FCB307F700D3
:1011C40083A70700638007028327C4FE9397270041
:1011D4000327C4FCB307F70083A7070013850700A0
:1011E400EF4010258327C4FE938717002326F4FEBF
:1011F4006FF05FFB832784FD63860700032584FD6E
:10120400EF20D00D832704FD63860700032504FD2A
:10121400EFB0401C832744FD63860700032544FD8B
:10122400EF6090508327C4FD638607000325C4FD47
:10123400EF10904B130000008320C10303248103AB
:101244001301010467800000130101812326117E2C
:101254002324817E1304017F37E3FFFF130303B6C6
:1012640033016100B7D7FFFF130704FFB307F7008B
:1012740023AEA738B7D7FFFF130704FFB307F70060
:1012840023ACB738B7670A801385075BEFF0574E76
:1012940083A7418E83A7870013850700EFC0973982
:1012A400B7670A801385475CEFF0D766B7670A8093
:1012B4001385475DEFF01766B7670A801385875E6D
:1012C400EFF05765B7670A8013850760EFF09764FE
:1012D400B7670A8013858762EFF0D763B7670A8020
:1012E4001385C763EFF01763B7670A801385076533
:1012F400EFF05762B7D7FFFF130704FFB307F700F8
:1013040003A7C7399307100063DAE70AB7D7FFFFCB
:10131400130704FFB307F70083A7873993874700B0
:1013240083A7070093850700B7670A801385C766FC
:10133400EFF01744B7D7FFFF130704FFB307F70015
:1013440083A787399387470003A70700B7670A80F5
:101354009385C76713050700EF20C80893070500A6
:1013640093B7170093F7F70F63880700B7670A80EE
:1013740013850765EFF0175AB7D7FFFF130704FF6C
:10138400B307F70083A787399387470003A70700AC
:10139400B7670A809385076813050700EF20880460
:1013A4009307050093B7170093F7F70F63880700B7
:1013B400B7670A8013854768EFF0D755B7D7FFFFA3
:1013C400130704FFB307F70003A7C73993072000E7
:1013D40063DAE70AB7D7FFFF130704FFB307F70081
:1013E40083A787399387870083A70700938507001E
:1013F400B7670A801385C769EFF09737B7D7FFFF40
:10140400130704FFB307F70083A78739938787007F
:1014140003A70700B7670A809385C767130507000A
:10142400EF10587C9307050093B7170093F7F70F55
:1014340063880700B7670A8013850765EFF0974D47
:10144400B7D7FFFF130704FFB307F70083A7873954
:101454009387870003A70700B7670A809385076807
:1014640013050700EF1018789307050093B71700CA
:1014740093F7F70F63880700B7670A8013854768F7
:10148400EFF05749232E04D81307C4D9930704DA7D
:10149400130607009385070013054006EFE0D022EA
:1014A40093070500232CF4FC832784FD638607023D
:1014B40083A7418E03A7C700832684FDB7670A80EC
:1014C4001386C76AB7670A809385C76D130507003B
:1014D400EFD04704EFC00729130000008327C4D9C5
:1014E40093850700B7670A8013850770EFF05728C4
:1014F400232604FE0327C4FE8327C4D96378F73266
:101504008325C4FEB7670A8013858772EFF05726D8
:101514008327C4FE93972700130704FFB307F7003C
:1015240003A507DBB7D7FFFF9387073A130704FF29
:10153400B307F7001307000093860700B7370000CE
:1015440013860780B717000093850790EFE0D04A11
:1015540093070500232AF4FC832744FD63860702CE
:1015640083A7418E03A7C700832644FDB7670A807B
:1015740013864773B7670A809385C76D1305070001
:10158400EFC05779EFC0071E13000000B7D7FFFF65
:101594009387073A130704FFB307F70093850700FF
:1015A400B7670A8013850778EFF0971C8327C4FE7A
:1015B40093972700130704FFB307F70003A507DB7E
:1015C400B7D7FFFF9387073A130704FFB307F70062
:1015D4001307000093860700B737000013860780BF
:1015E400B717000093851790EFE0104193070500AB
:1015F4002328F4FC832704FD6386070283A7418E16
:1016040003A7C700832604FDB7670A8013860779FA
:10161400B7670A809385C76D13050700EFC0976FFE
:10162400EFC0471413000000B7D7FFFF9387073AB2
:10163400130704FFB307F70093850700B7670A8011
:101644001385C77DEFF0D7128327C4FE9397270035
:10165400130704FFB307F70003A507DBB7D7FFFFA2
:101664009387073A130704FFB307F7001307000033
:1016740093860700B737000013860780B71700006A
:1016840093852790EFE05037930705002326F4FC59
:101694008327C4FC6386070283A7418E03A7C70080
:1016A4008326C4FCB7670A801386C77EB7670A809F
:1016B4009385C76D13050700EFC0D765EFC0870A90
:1016C40013000000B7D7FFFF9387073A130704FFFF
:1016D400B307F70093850700B7770A80138547831C
:1016E400EFF017098327C4FE93972700130704FF1D
:1016F400B307F70003A507DBB7D7FFFF9387073AC4
:10170400130704FFB307F7001307000093860700CD
:10171400B737000013860780B7170000938537900A
:10172400EFE0902D930705002324F4FC832784FC29
:101734006386070283A7418E03A7C700832684FC20
:10174400B7770A8013864784B7670A809385C76D85
:1017540013050700EFC0175CEFC0C70013000000BB
:10176400B7D7FFFF9387073A130704FFB307F700C0
:1017740093850700B7770A8013850789EFF0477FC1
:101784008327C4FE93972700130704FFB307F700CA
:1017940003A507DBB7D7FFFF9387073A130704FFB7
:1017A400B307F7001307000093860700B73700005C
:1017B40013860780B717000093854790EFE0D02386
:1017C400930705002322F4FC832744FC6386070265
:1017D40083A7418E03A7C700832644FCB7770A80FA
:1017E4001386078AB7670A809385C76D13050700B8
:1017F400EFC05752EFB0177713000000B7D7FFFFC1
:101804009387073A130704FFB307F700938507008C
:10181400B7770A801385078FEFF087758327C4FE97
:10182400938717002326F4FE6FF0DFCC8327C4D9F7
:1018340063960700930710006F10800D232404C0E3
:10184400032504DA930784C01307C4C09306400633
:101854009305400013060000EFF08037930705005E
:101864002320F4FC832704FC6386070283A7418EAC
:1018740003A7C700832604FCB7770A801386479022
:10188400B7670A809385C76D13050700EFC09748B3
:10189400EFB0576D130000008327C4D99385070068
:1018A400B7770A8013850795EFF0876C232404FE2D
:1018B400032784FE832784C0637EF740832584FE48
:1018C400B7670A8013858772EFF0876A832784FEDF
:1018D40093972700130704FFB307F70003A5C7C1B5
:1018E400B7D7FFFF9387073A130704FFB307F7003F
:1018F4001307000093860700B7370000138607809C
:10190400B71700009385B702EFF0407793070500FF
:10191400232EF4FA8327C4FB6386070283A7418E30
:1019240003A7C7008326C4FBB7770A801386C7972B
:10193400B7670A809385C76D13050700EFC0973D0D
:10194400EFB0576213000000B7D7FFFF9387073A41
:10195400130704FFB307F70093850700B7770A80DE
:101964001385879CEFF0C760832784FE9397270035
:10197400130704FFB307F70003A5C7C1B7D7FFFFD9
:101984009387073A130704FFB307F7001307000010
:1019940093860700B737000013860780B717000047
:1019A4009385C702EFF0806D93070500232CF4FAAA
:1019B400832784FB6386070283A7418E03A7C7009E
:1019C400832684FBB7770A801386C79DB7670A808E
:1019D4009385C76D13050700EFC0D733EFB0975851
:1019E40013000000B7D7FFFF9387073A130704FFDC
:1019F400B307F70093850700B7770A80138587A29A
:101A0400EFF00757832784FE93972700130704FFFB
:101A1400B307F70003A5C7C1B7D7FFFF9387073AFA
:101A2400130704FFB307F7001307000093860700AA
:101A3400B737000013860780B71700009385F702B5
:101A4400EFF0C06393070500232AF4FA832744FBCD
:101A54006386070283A7418E03A7C700832644FB3E
:101A6400B7770A80138607A4B7670A809385C76D82
:101A740013050700EFC0172AEFB0D74E130000007C
:101A8400B7D7FFFF9387073A130704FFB307F7009D
:101A940093850700B7770A80138507A9EFF0474DB0
:101AA400832784FE93972700130704FFB307F700E7
:101AB40003A5C7C1B7D7FFFF9387073A130704FFEE
:101AC400B307F7001307000093860700B737000039
:101AD40013860780B71700009385D702EFF0005AEA
:101AE400930705002328F4FA832704FB638607027F
:101AF40083A7418E03A7C700832604FBB7770A8018
:101B0400138687AAB7670A809385C76D13050700F4
:101B1400EFC05720EFB0174513000000B7D7FFFF01
:101B24009387073A130704FFB307F7009385070069
:101B3400B7770A80138587AFEFF08743832784FE46
:101B440093972700130704FFB307F70003A5C7C142
:101B54009307C4BB130700009386070013064000D5
:101B6400B717000093852700EFF040519307050055
:101B74002326F4FA8327C4FA6386070283A7418ED7
:101B840003A7C7008326C4FAB7770A80138607B170
:101B9400B7670A809385C76D13050700EFC09717D1
:101BA400EFB0573C130000008327C4BB93850700A4
:101BB400B7770A801385C7B6EFF0873B832784FE87
:101BC40093972700130704FFB307F70003A5C7C1C2
:101BD4009307C4BB13070000938607001306400055
:101BE400B71700009385C700EFF04049930705003D
:101BF4002324F4FA832784FA6386070283A7418E99
:101C040003A7C700832684FAB7770A80138607B927
:101C1400B7670A809385C76D13050700EFC0970F58
:101C2400EFB05734130000008327C4BB938507002B
:101C3400B7770A80138507BFEFF08733832784FEC5
:101C440093972700130704FFB307F70003A5C7C141
:101C5400930704BB13070000938607001306800054
:101C6400B71700009385F701EFF040419307050093
:101C74002322F4FA832744FA6386070283A7418E5A
:101C840003A7C700832644FAB7770A80138647C19F
:101C9400B7670A809385C76D13050700EFC09707E0
:101CA400EFB0572C13000000032704BB832744BB69
:101CB4001306070093860700B7770A80138507C7C2
:101CC400EFF0072B832784FE938717002324F4FE69
:101CD4006FF01FBE832784C063960700930710002C
:101CE4006F001043930720FE2326F4BA1306C4C0E2
:101CF400130646009307C4BA13070000B706008012
:101D0400938646729305100013050000EF7051107E
:101D1400930705002320F4FA8327C4BA63880702D3
:101D240083A7418E03A7C7008327C4BA93860700FD
:101D3400B7770A80138647C9B7670A809385C76D4A
:101D440013050700EFC0077DEFB0D721832704FAFE
:101D5400232EF4F8930720FE2324F4BA832704C126
:101D6400130784BA13062000930600009385070026
:101D74000325C4F9EF10806E93070500232CF4F8B3
:101D8400832784BA6388070283A7418E03A7C70009
:101D9400832784BA93860700B7770A80138647CDD2
:101DA400B7670A809385C76D13050700EFC0877670
:101DB400EFB0571B832784F9232AF4F8232804F867
:101DC400232E04BE232004C0232204C0B7770A8034
:101DD400938507D2B7070D801385C7D5EF60044BF1
:101DE40013070500B7870480938507D813050700F8
:101DF400EF505433032704C1B7770A801386C7D43E
:101E0400930507000325C4F9EFF0CF8B9307050072
:101E14002322F4FE832744FE639A0710B7770A80CF
:101E24009385C7D5B7070D801385C7D5EF600446E2
:101E340013070500B7870480938507D813050700A7
:101E4400EF50542E032704C1B7770A80138687D82E
:101E5400930507000325C4F9EFE09F91930705005C
:101E64002322F4FE832744FE639407029307C4BF2E
:101E740013870700832604F9032644FE832544F9C7
:101E84000325C4F9EFF08FAF930710006F005028BB
:101E9400B7770A80938547D9B7070D801385C7D5CF
:101EA400EF60C43E13070500B7870480938507D805
:101EB40013050700EF501427032704C1B7770A80DE
:101EC4001386C7D493050700032544FEEFE01FB82B
:101ED4009307050093B7170093F7F70F638C070672
:101EE400B7770A809385C7DBB7070D80138547C48E
:101EF400EF60C43913070500B7870480938507D8BA
:101F040013050700EF5014229307C4BF138707007B
:101F1400832604F9032644FE832544F90325C4F9E2
:101F2400EFF0CFA5930710006F00901EB7770A80DB
:101F34009385C7DDB7070D801385C7D5EF600435DA
:101F440013070500B7870480938507D81305070096
:101F5400EF50541DB7770A80138587DFEFF04701F0
:101F640083A7418E83A7870013850700EFB0976C82
:101F7400930720FE2322F4BA930744BA1307000000
:101F8400B746000093054000130600000325C4F97A
:101F9400EF109071930705002326F4F8832744BAC1
:101FA4006388070283A7418E03A7C700832744BA27
:101FB40093860700B7770A801386C7E1B7670A805C
:101FC4009385C76D13050700EFC0C754EFB0877939
:101FD4008327C4F8232CF4BE930720FE2320F4BAED
:101FE400930704BA13070000B746000093054000A6
:101FF400130600000325C4F9EF10106B93070500C6
:102004002324F4F8832704BA6388070283A7418E44
:1020140003A7C700832704BA93860700B7770A800B
:102024001386C7E1B7670A809385C76D1305070058
:10203400EFC0474EEFB00773832784F8232AF4BE1A
:10204400B7770A80138547E7EFE0977283A7418E3D
:1020540083A7870013850700EFB0D75D930720FEA1
:10206400232EF4B89307C4B913070000B746000041
:1020740093052000130600000325C4F9EF10D06275
:10208400930705002322F4F88327C4B96388070261
:1020940083A7418E03A7C7008327C4B9938607008B
:1020A400B7770A80138687E9B7670A809385C76D77
:1020B40013050700EFC00746EFB0C76A832744F84B
:1020C4002328F4BE832784BF232EF4BE832744BF72
:1020D4002320F4C0832704BF2322F4C09307000401
:1020E4002326F4BEB7770A80138547EFEFE05768DD
:1020F40083A7418E83A7870013850700EFB097530A
:10210400930720FE232CF4B8930784B913860700A1
:10211400B7770A80938547F1032544FEEF9090003A
:10212400930705002320F4F8832784B96388070202
:1021340083A7418E03A7C700832784B9938607002A
:10214400B7770A80138647F2B7670A809385C76D0D
:1021540013050700EFC0073CEFB0C760832704F8FE
:102164002328F4F8930784BF9386070013064000DE
:1021740093050000032504F9EFA08072930705007E
:10218400232EF4F68327C4F76386070283A7418EC0
:1021940003A7C7008326C4F7B7770A80138647F5D9
:1021A400B7670A809385C76D13050700EFC08736AC
:1021B400EFB0475B13000000930744BF938607000A
:1021C4001306400093051000032504F9EFA0406DA9
:1021D40093070500232CF4F6832784F7638607020C
:1021E40083A7418E03A7C700832684F7B7770A80A5
:1021F400138687F9B7670A809385C76D13050700AF
:10220400EFC04731EFB0075613000000930704BF37
:10221400938607001306400093052000032504F964
:10222400EFA0006893070500232AF4F6832744F7F8
:102234006386070283A7418E03A7C700832644F75A
:10224400B7770A801386C7FDB7670A809385C76D81
:1022540013050700EFC0072CEFB0C75013000000B0
:102264009307C4BE9386070013064000930530000D
:10227400032504F9EFA0C062930705002328F4F6B0
:10228400832704F76386070283A7418E03A7C70049
:10229400832604F7B7770A8013860702B7670A8094
:1022A4009385C76D13050700EFC0C726EFB0874BB2
:1022B40013000000B7770A8013854705EFE0574BFA
:1022C40083A7418E83A7870013850700EFB0973655
:1022D400232004FE032704FEB71700006356F716F5
:1022E400EFF087759307050013850700EF70974F8C
:1022F40013070500B7770A8083A507431305070072
:10230400EF70475E9307050013870700B7770A80CD
:1023140083A5474313050700EF705716930705007D
:10232400232AF4B8832584BF832704FE93962700C9
:10233400930744B923200100930800001308000008
:102344001307400013061000032544F9EF805127BA
:10235400930705002326F4F68327C4F66386070251
:1023640083A7418E03A7C7008326C4F6B7770A80E4
:1023740013868707B7670A809385C76D130507001F
:10238400EFC04719EFB0073E13000000EFF0C76A33
:102394009307050013850700EF70D7441307050062
:1023A400B7770A8083A5074313050700EF708753A7
:1023B4009307050013870700B7770A8083A547436F
:1023C40013050700EF70970B93070500232AF4B851
:1023D400832544BF832704FE93962700930744B9BB
:1023E4002320010093080000130800001307400095
:1023F40013061000032544F9EF80911C9307050090
:102404002324F4F6832784F66386070283A7418E88
:1024140003A7C700832684F6B7770A801386470D7F
:10242400B7670A809385C76D13050700EFC0870E51
:10243400EFB0473313000000832704FE938717008F
:102444002320F4FE6FF01FE993070004232EF4BC4D
:10245400930710002320F4BE930710002322F4BE38
:10246400930700042328F4BC93070004232AF4BC34
:1024740093070004232CF4BCB7770A801385071351
:10248400EFE0172F83A7418E83A7870013850700EA
:10249400EFB0571A9306C4BD130704BD930784BE57
:1024A4002320F1009308000013080000938706001E
:1024B4009306000013063000832504F9032544F92C
:1024C400EFB0001F930705002322F4F6832744F698
:1024D4006386070283A7418E03A7C700832644F6B9
:1024E400B7770A8013860715B7670A809385C76D87
:1024F40013050700EFC00702EFB0C7261300000062
:10250400B7770A801385071CEFE0972683A7418ECF
:1025140083A7870013850700EFB0D711930784BE04
:102524009385070013051000EFB04165930705007C
:102534002320F4F6832704F66386070283A7418EDB
:1025440003A7C700832604F6B7770A801386471DBE
:10255400B7670A809385C76D13050700EFB0977BB3
:10256400EFB0472013000000032584BE930784BC0A
:10257400130700009386070013068000B7170000B6
:1025840093852728EFB0010D93070500232EF4F45B
:102594008327C4F56386070283A7418E03A7C70078
:1025A4008326C4F5B7770A801386C71FB7670A80E6
:1025B4009385C76D13050700EFB0D775EFB0871A81
:1025C40013000000032584BE930704BC1307000016
:1025D4009386070013068000B717000093853728F9
:1025E400EFB0410793070500232CF4F4832784F507
:1025F4006386070283A7418E03A7C700832684F559
:10260400B7770A801386C726B7670A809385C76D94
:1026140013050700EFB01770EFB0C71413000000E4
:10262400032704BC832744BC032584BC8325C4BC82
:102634003306A7401308060033380701B386B740B2
:10264400B3870641938607001307060093870600A5
:102654001305070093850700EF60173D1307050076
:10266400938705002328E4F4232AF4F4032604F5CD
:10267400832644F5B7770A801385472DEFE0570F7B
:10268400832784BE13850700EFB011239307050049
:102694002326F4F48327C4F46386070283A7418EB8
:1026A40003A7C7008326C4F4B7770A801386472E8E
:1026B400B7670A809385C76D13050700EFB0976568
:1026C400EFB0470A13000000B7770A8013858730FC
:1026D400EFE0170A232E04FC0327C4FDB7170000FC
:1026E400635EF706832504BF8327C4FD9396270002
:1026F400930704B923200100930800001308000085
:102704001307400013061000032544F9EF20903D01
:10271400930705002324F4F4832784F463860702D3
:1027240083A7418E03A7C700832684F4B7770A8062
:1027340013860731B7670A809385C76D13050700B1
:10274400EFB0575DEFB00702130000008327C4FD0C
:1027540093871700232EF4FC6FF01FF8B7770A80D5
:1027640013850737EFE0D7008327C4BF138507001D
:10277400EF30004C930705002322F4F4832744F43C
:102784006386070283A7418E03A7C700832644F408
:10279400B7770A8013864737B7670A809385C76D72
:1027A40013050700EFB01757EFA0D77B1300000005
:1027B400832704C013850700EF3080479307050083
:1027C4002320F4F4832704F46386070283A7418E4D
:1027D40003A7C700832604F4B7770A8013868739D2
:1027E400B7670A809385C76D13050700EFB097524A
:1027F400EFA0577713000000832744C01385070018
:10280400EF30004393070500232EF4F28327C4F32B
:102814006386070283A7418E03A7C7008326C4F3F8
:10282400B7770A801386C73BB7670A809385C76D5D
:1028340013050700EFB0174EEFA0D7721300000086
:10284400032504F9EF90103993070500232CF4F2C3
:10285400832784F36386070283A7418E03A7C700F7
:10286400832684F3B7770A801386073EB7670A8006
:102874009385C76D13050700EFB0D749EFA0976E96
:1028840013000000032544FEEF50006A930705007F
:10289400232AF4F2832744F36386070283A7418E35
:1028A40003A7C700832644F3B7770A801386873FBC
:1028B400B7670A809385C76D13050700EFB0974586
:1028C400EFA0576A130000000325C4F9EF00C061AC
:1028D400930705002328F4F2832704F36386070291
:1028E40083A7418E03A7C700832604F3B7770A8022
:1028F40013864741B7670A809385C76D13050700A0
:10290400EFB05741EFA017661300000093070000D3
:1029140013850700372300001303034A33016100C2
:102924008320C17E0324817E1301017F6780000020
:10293400130101FE232E1100232C81001304010234
:102944002326A4FE2324B4FE0327C4FE9307100009
:10295400631AF702032784FEB70701009387F7FF82
:102964006312F702138581C2EF70D30BB7E70C80B3
:10297400138687BF938581C2B7A703801385C73C9D
:10298400EFA0D77C130000008320C1010324810140
:102994001301010267800000130101FF23261100C7
:1029A4002324810013040101B70701009385F7FF75
:1029B40013051000EFF0DFF78320C100032481002A
:1029C4001301010167800000130101FF2326110098
:1029D400232481001304010113850190EF004001B9
:1029E400032481008320C1001301010167800000DA
:1029F400130101FF23261100232481001304010184
:102A0400232AA4FE37750A8013058543B735008051
:102A1400938505BE1387418B9387C1C2130640007B
:102A240093060000EFE0D23C032481008320C10020
:102A34001301010167800000130101FF2326110027
:102A44002324810013040101EFF01FF80324810003
:102A54008320C1001301010167800000130101FB01
:102A640023261104232481042322910423202105F5
:102A7400232E3103232C4103232A510323286103EA
:102A84002326710323248103232291032320A103FA
:102A9400232EB101130401051371C1FF232CA100DE
:102AA4000325C701232AA100330505038324070155
:102AB400B38AA400832487013385F4028327C700E3
:102AC4003385A700832707022324F100B387170364
:102AD400032747013307F7002322E1003387E60287
:102AE400B307E500338756033305E50013152500C6
:102AF4003385A5002320A10013952700B309A60060
:102B04002326D100139D26009305000003254100D0
:102B14002328B1003305B5008325C1003309B5026C
:102B2400832D0100930B000033857A0133052501C1
:102B34001315250083258101338BA500138C0D000B
:102B4400938C0900130A000003250B0083250C0055
:102B540097700700E780C01283A50C0097700700E8
:102B6400E780C09523A0AC00130C4C00938C4C0060
:102B7400130A1A00E36A9AFCB38DAD01938B1B0010
:102B840003254101E3E2ABFAB389A90183250101DD
:102B94009385150003258100E3EAA5F6130104FBE0
:102BA400832DC101032D0102832C4102032C8102D8
:102BB400832BC102032B0103832A4103032A8103CC
:102BC4008329C103032901048324410403248104C8
:102BD4008320C1041301010567800000130101FB78
:102BE4002326110423248104232291042320210574
:102BF400232E3103232C4103232A51032328610369
:102C04002326710323248103232291032320A10378
:102C1400232EB10183A7C501232CF100B386D7026B
:102C240083A70501B38BD70003A485013306C4022F
:102C340083A6C5003386C60083A605022328D100D7
:102C4400B386E60283A54501B386D5008325C50076
:102C540003A705002326D100B305D702B305B600A8
:102C6400B30677033306D6001316260083264500E1
:102C740083A606003386C6002322C100939525004F
:102C84000326850003260600330DB6000325050040
:102C9400032C05002324E100931C27009305000066
:102CA4000325C100232AB1003305B5008325810023
:102CB400B304B502832A4100130A000033854B0193
:102CC4003305950013152500B309AC00138B0A00D6
:102CD400930D0D001309000003A5090083250B00C3
:102CE40097700700E780C0F983A50D00976007007F
:102CF400E780C07C23A0AD00130B4B00938D4D00E7
:102D040013091900E36A89FCB38A9A01130A1A00A9
:102D140003258101E364AAFA330D9D018325410152
:102D24009385150003250101E3ECA5F6832DC1016C
:102D3400032D0102832C4102032C8102832BC10247
:102D4400032B0103832A4103032A81038329C1033B
:102D54000329010483244104032481048320C1043E
:102D64001301010567800000130101FB23261104F0
:102D7400232481042322910423202105232E3103BB
:102D8400232C4103232A510323286103232671039F
:102D940023248103232291032320A103232EB101A1
:102DA40083A7C501232CF100B386D70283A70501AD
:102DB400B38BD70003A485013306C40283A6C500E0
:102DC4003386C60083A605022328D100B386E60213
:102DD40083A54501B386D5008325C50003A7050057
:102DE4002326D100B305D702B305B600B306770393
:102DF4003306D60013162600832645003386C60004
:102E04002322C1009395250003268500330DB600C7
:102E1400032C05002324E100931C270093050000E4
:102E24000325C100232AB1003305B50083258100A1
:102E3400B304B502832A4100130A000033854B0111
:102E44003305950013152500B309AC00138B0A0054
:102E5400930D0D001309000003A5090083250B0041
:102E640097700700E780C0E183A50D009760070015
:102E7400E780C06423A0AD00130B4B00938D4D007D
:102E840013091900E36A89FCB38A9A01130A1A0028
:102E940003258101E364AAFA330D9D0183254101D1
:102EA4009385150003250101E3ECA5F6832DC101EB
:102EB400032D0102832C4102032C8102832BC102C6
:102EC400032B0103832A4103032A81038329C103BA
:102ED4000329010483244104032481048320C104BD
:102EE4001301010567800000130101FD232611026F
:102EF4002324810223222103232031031304010309
:102F0400232EA4FC8326C4FD83C68601639C06008D
:102F14000325C4FDEFD04720232E04FC93070000B3
:102F24006F00003097E60C009386060403A60600A3
:102F340083A646001377060493F70600930607005A
:102F4400B3E6F6006384060AEF10C2369306100057
:102F540017460A001306C64E9305E00217450A00F9
:102F64001305C55EEF10922497E70C00938747FF83
:102F740083A707006388070297B70C0083A7C77469
:102F840083A7070083A7C700938607001306E00002
:102F94009305100017450A001305454BEFC0173180
:102FA4006F00000297B70C0083A7077283A707007E
:102FB40083A7C7009385070013050002EFB0C75F1E
:102FC40097B70C0083A7477083A7070083A7C700A0
:102FD40093860700130610019305100017450A0095
:102FE4001305C547EFC0972CEF10822E8327C4FD2D
:102FF40083A747006342F00297460A009386464738
:1030040017460A00130686549305F00217450A0072
:1030140013050548EFA087768327C4FD83A74700DF
:103024009387F7FF0327C4FD2322F7002324F4FE2C
:103034008327C4FD83A7470063D2070297460A008B
:103044009386064717460A00130646509305F00276
:1030540017450A001305C543EFA04772832784FE72
:10306400639E071A97E70C00938707F003A70700EE
:1030740083A747001379070493F90700930709000E
:10308400B3E737016382070AEF10C22293061000E8
:1030940017460A001306C63A9305200317450A008B
:1030A4001305C54AEF10921097E70C00938747EB7E
:1030B40083A707006388070297B70C0083A7C7603C
:1030C40083A7070083A7C700938607001306E000C1
:1030D4009305100017450A0013054537EFC0171D67
:1030E4006F00000297B70C0083A7075E83A7070051
:1030F40083A7C7009385070013050002EFB0C74BF1
:1031040097B70C0083A7475C83A7070083A7C70072
:103114000326C4FD97450A009385853B1385070064
:10312400EFB0473FEF10C21A232604FE6F000003DE
:103134008327C4FD03A787008327C4FE9397270032
:10314400B307F70083A7070013850700EFB0013B1F
:103154008327C4FE938717002326F4FE8327C4FD28
:1031640083A707010327C4FEE364F7FC8327C4FD98
:1031740083A7870013850700EFC0177A8327C4FD50
:1031840023A407008327C4FD83A7C7001385070072
:10319400EFC097788327C4FD23A60700232604FEE7
:1031A4006F0080040327C4FD8327C4FE9387870030
:1031B40093972700B307F70083A707001385070039
:1031C400EFC097750327C4FD8327C4FE9387870048
:1031D40093972700B307F70023A007008327C4FEB3
:1031E400938717002326F4FE0327C4FE9307500099
:1031F400E3FAE7FA0325C4FDEFC01772232E04FC9B
:1032040097B70C0083A7C74C83A707001387F7FF62
:1032140097B70C0083A7C74B23A0E70093070000D0
:10322400138507008320C10203248102032941027C
:10323400832901021301010367800000130101FDCA
:103244002326110223248102232221032320310374
:10325400232E4101232C5101130401039305000083
:1032640017450A0013050528EF009272232EA4FCCB
:103274008327C4FD6382071C97B70C0083A74745C7
:1032840083A7070093B7170093F7F70F232CF4FCD9
:10329400832784FD638A070C97E70C009387C7CCC8
:1032A40003A7070083A74700137A070493FA0700CC
:1032B40093070A00B3E757016384070AEF00927F7C
:1032C4009306100017460A00130686179305D006C6
:1032D40017450A001305C528EF10426D97E70C0047
:1032E400938707C883A707006388070297B70C0072
:1032F40083A7873D83A7070083A7C700938607009A
:103304001306E0009305100017450A001305051481
:10331400EFC0C7796F00000297B70C0083A7C73AC4
:1033240083A7070083A7C70093850700130500023E
:10333400EFB0872897B70C0083A7073983A7070046
:1033440083A7C700938607001306000393051000A4
:1033540017450A001305451AEFC04775EF00527769
:10336400EF5052076F00800D97E70C009387C7BF9B
:1033740003A7070083A74700B71600003379D700D7
:1033840093F9070093070900B3E737016388070A35
:10339400EF0052729306300017460A00130606190E
:1033A4009305200717450A001305851BEF100260DB
:1033B40097E70C009387C7BA83A7070063880702BF
:1033C40097B70C0083A7473083A7070083A7C700DC
:1033D400938607001306E0009305100017450A00C2
:1033E4001305C506EFC0876C6F00000297B70C0089
:1033F40083A7872D83A7070083A7C70093850700AA
:1034040013050002EFB0471B97B70C0083A7C72B27
:1034140083A7070083A7C7009386070013066001EC
:103424009305100017450A001305C510EFC007687F
:10343400EF00126A6F008000130000008320C102B5
:10344400032481020329410283290102032AC101C1
:10345400832A81011301010367800000130101FB2A
:1034640023261104232481042322910423202105EB
:10347400232E3103232C4103232A51031304010572
:103484002326A4FC2324B4FC2320C4FC2322D4FC40
:10349400232EE4FA232A04FC8327C4FC6394070E36
:1034A40097E70C00938747AC03A7070083A747005F
:1034B400B7160000337ED70093FE070093070E0073
:1034C400B3E7D701638A070AEF00D25E93063000A0
:1034D40017460A001306860A9305600217450A0078
:1034E40013050520EF10824C97E70C00938747A73C
:1034F40083A707006388070297B70C0083A7C71C3C
:1035040083A7070083A7C70093860700130600025A
:103514009305100017450A001305C506EFC00759A7
:103524006F00C00297B70C0083A7071A83A7070090
:1035340083A7C70093860700130630019305100084
:1035440017450A0013054506EFC0475697B70C0008
:1035540083A7871783A7070083A7C70017460A0016
:103564001306C60597450A0093858506138507004B
:10357400EFA0577AEF00D2559307E0FD232CF4FC1B
:103584006F00C051832784FC6394070E97E70C00F7
:103594009387879D03A7070083A74700B7160000FA
:1035A4003373D70093F3070093070300B3E777005F
:1035B400638A070AEF0012509306300017460A0088
:1035C4001306C6FB9305800217450A00130545112F
:1035D400EF10C23D97E70C009387879883A70700F5
:1035E4006388070297B70C0083A7070E83A7070019
:1035F40083A7C700938607001306F0019305100004
:1036040017450A00130505FDEFC0474A6F00C002C5
:1036140097B70C0083A7470B83A7070083A7C700AE
:1036240093860700130620019305100017450A002E
:10363400130545FCEFC0874797B70C0083A7C7085D
:1036440083A7070083A7C70017460A001306C6FB13
:1036540097450A009385C5F713850700EFA0976B7C
:10366400EF0012479307F0FD232CF4FC6F00004396
:1036740097E70C009387478F03A7070083A74700AA
:103684001378170093F8070093070800B3E71701AE
:103694006386070AEF0012429306100017460A00D9
:1036A4001306C6F79305A00217450A001305450340
:1036B400EF10C22F97E70C009387878A83A7070030
:1036C4006388070297B70C0083A7070083A7070046
:1036D40083A7C700938607001306E0009305100034
:1036E40017450A00130505F4EFC0473C6F000002BC
:1036F40097B70C0083A747FD83A7070083A7C700DC
:103704009385070013050002EFA0176B97B70C0011
:1037140083A787FB83A7070003A7C700832784FC2D
:1037240083A7471A1386070097450A00938585F0F7
:1037340013050700EFA0175EEF009239832744FCBE
:10374400639C0700832744FC639A070E032704FC49
:103754009307300063F4E70E97E70C009387C78064
:1037640003A7070083A74700B7160000337AD700E2
:1037740093FA070093070A00B3E75701638A070A1D
:10378400EF0052339306300017460A00130606DF93
:103794009305D00217450A00130585F4EF100221A2
:1037A40097D70C009387C77B83A70700638807021A
:1037B40097B70C0083A747F183A7070083A7C70027
:1037C400938607001306E0019305100017450A00CD
:1037D400130585E8EFC0872D6F00C00297B70C0072
:1037E40083A787EE83A7070083A7C70093860700F4
:1037F400130610019305100017450A001305C5E7C9
:10380400EFC0C72A97B70C0083A707EC83A707006C
:1038140083A7C700938607001306B0029305100020
:1038240017450A00130585E6EFC04728EF00522A22
:10383400930720FE232CF4FC6F00402697D70C003E
:103844009387877203A6070083A6470093070600A1
:10385400B3E7D700639A070097B70C0083A707E77D
:1038640083A70700638E0700832704FC93E72700E0
:103874002320F4FC832744FC93E707002322F4FC71
:10388400232E04FC6F0000048327C4FC03A78700D5
:103894008327C4FD93972700B307F70083A4070089
:1038A400032584FCEFE0413D930705006396F40093
:1038B40093071000232AF4FC8327C4FD9387170081
:1038C400232EF4FC8327C4FC83A707010327C4FD2C
:1038D400E36CF7FA832744FD6394070E97D70C0033
:1038E4009387876803A7070083A74700B7160000DC
:1038F4003379D70093F9070093070900B3E7370139
:10390400638A070AEF00121B9306300017460A0069
:103914001306C6C69305900317450A00130545DC34
:10392400EF10C20897D70C009387876383A707001B
:103934006388070297B70C0083A707D983A70700FA
:1039440083A7C700938607001306F00193051000B0
:1039540017450A00130505C8EFC047156F00C002DC
:1039640097B70C0083A747D683A7070083A7C70090
:1039740093860700130620019305100017450A00DB
:10398400130545C7EFC0871297B70C0083A7C7D3A9
:1039940083A7070083A7C700938607001306500276
:1039A4009305100017450A00130505D1EFC0071051
:1039B400EF0012129307F0FD232CF4FC6F00000EAD
:1039C40013050003EFC08774930705002328F4FC54
:1039D400832704FD639807009307A0FF232CF4FCBE
:1039E4006F00C00B832704FD1307100023A2E70018
:1039F400832704FD0327C4FC23A4E700832704FDD5
:103A0400032784FC23A6E700832604FD032704FC84
:103A1400832744FC23A8E60023AAF600832704FD99
:103A240023AE0700832704FD23AC0700832704FD8E
:103A340023A00702832704FD23A20702832704FD92
:103A440023A407020325C4FCEFF00203032584FC2E
:103A5400EFA09161232C04FC832784FC83A74725D2
:103A640083A7C703638E0700832784FC83A74725A6
:103A740083A7C703032504FDE7800700232CA4FCC8
:103A84008327C4FB638807008327C4FB032784FDC3
:103A940023A0E700832704FD6F00C0018327C4FB34
:103AA400638807008327C4FB032784FD23A0E70062
:103AB40093070000138507008320C10403248104B5
:103AC40083244104032901048329C103032A8103B4
:103AD400832A41031301010567800000130101FCDF
:103AE400232E1102232C8102232A210323283103AC
:103AF4002326410323245103130401042326A4FC95
:103B04008326C4FC6392060E97D60C009386C645A2
:103B140003A6060083A64600B71500003377B60057
:103B240093F7060093060700B3E6F600638A060AD5
:103B3400EF0042789306300017460A001306C6BB0E
:103B44009305E00117450A001305C5CFEF0012667F
:103B540097D70C009387C74083A7070063880702A1
:103B640097B70C0083A747B683A7070083A7C700AE
:103B740093860700130660029305100017450A0098
:103B8400130505B8EFB097726F00C00297B70C0029
:103B940083A787B383A7070083A7C700938607007B
:103BA400130690019305100017450A001305C5B7C5
:103BB400EFB0D76F97B70C0083A707B183A70700AF
:103BC40083A7C70017460A001306C6B797450A001D
:103BD4009385C5B813850700EFA0D713EF00426F94
:103BE4009307C0FD6F00002A8327C4FC83A78700C6
:103BF400232EF4FC8327C4FC83A7C700232CF4FCE6
:103C04000325C4FCEF80C1468327C4FC83A7470077
:103C14006342F00297460A00938686B417460A0068
:103C2400130646C29305500217450A00130585B5CD
:103C3400EF90D7348327C4FC83A747009387F7FF0B
:103C44000327C4FC2322F700232AF4FC8327C4FCA3
:103C540083A7470063D2070297460A009386C6B437
:103C640017460A00130606BE9305500217450A00BC
:103C7400130545B1EF90973097D70C009387C72E63
:103C840003A7070083A74700137A070493FA0700E2
:103C940093070A00B3E757016384070AEF008261C0
:103CA4009306100017460A00130646B293056002F5
:103CB40017450A00130505B9EF00524F97D70C00BA
:103CC4009387072A83A707006388070297B70C0026
:103CD40083A7879F83A7070083A7C700938607004E
:103CE4001306E0009305100017450A001305C5AE3E
:103CF400EFB0D75B6F00000297B70C0083A7C79C97
:103D040083A7070083A7C700938507001305000254
:103D1400EFA0970A97B70C0083A7079B83A7070018
:103D240083A7C700832644FD0326C4FC97450A00E5
:103D3400938585AB13850700EFA0C77DEF0042593B
:103D4400832744FD639E07128327C4FC83A70702CD
:103D54006382070297460A00938606AB17460A0059
:103D6400130646AE9305A00217450A00130585A164
:103D7400EF90D72097D70C009387071F03A707005E
:103D840083A747001379070493F9070093070900F1
:103D9400B3E737016382070AEF00C25193061000AC
:103DA40017460A00130686A29305B00217450A00B7
:103DB400130545A9EF00923F97D70C009387471A44
:103DC40083A707006388070297B70C0083A7C78FF0
:103DD40083A7070083A7C700938607001306E000A4
:103DE4009305100017450A001305059FEFB0174C03
:103DF4006F00000297B70C0083A7078D83A7070005
:103E040083A7C7009385070013050002EFA0C77AB4
:103E140097B70C0083A7478B83A7070083A7C70026
:103E24000326C4FC97450A00938545A01385070023
:103E3400EFA0476EEF00C2498327C4FC83A7C700E5
:103E440083A7472583A70704638E07008327C4FC41
:103E540083A7C70083A7472583A707040325C4FCBA
:103E6400E78007000325C4FCEFC0072B232604FCCE
:103E74000325C4FDEFF04F87032584FDEFA00168FF
:103E840093070000138507008320C10303248103E3
:103E94000329410383290103032AC102832A8102DE
:103EA4001301010467800000130101ED23261112A0
:103EB400232481122322211323203113232E411181
:103EC400232C5111232A61112328711123268111D6
:103ED400232491112322A1112320B11113040113CE
:103EE4002326A4FA2320B4FA2322C4FA2324D4FADE
:103EF400232EE4F8232CF4F8232604FC832784FAE5
:103F04006394070E97D70C009387070603A707004F
:103F140083A74700B71600003378D70093F807004B
:103F240093070800B3E71701638A070AEF00823892
:103F34009306300017460A00130646929305A00222
:103F440017450A00130505E7EF00522697D70C0022
:103F54009387070183A707006388070297A70C00CC
:103F640083A7877683A7070083A7C70093860700E4
:103F7400130640029305100017450A001305858EA9
:103F8400EFB0D7326F00C00297A70C0083A7C773A6
:103F940083A7070083A7C700938607001306700151
:103FA4009305100017450A001305458EEFB017302E
:103FB40097A70C0083A7477183A7070083A7C700AF
:103FC40017460A001306068E97450A009385458E08
:103FD40013850700EFA00754EF00822F930730FCEE
:103FE4002324F4FC6F1000288327C4FA6394070E7B
:103FF40097D70C00938747F703A7070083A74700C9
:10400400B71600003373D70093F307009307030038
:10401400B3E77700638A070AEF00C22993063000EA
:1040240017460A00130686839305C00217450A0043
:10403400130545D8EF00921797D70C00938747F2E2
:1040440083A707006388070297A70C0083A7C767A5
:1040540083A7070083A7C7009386070013060002FF
:104064009305100017450A001305C584EFB0172403
:104074006F00C00297A70C0083A7076583A70700FA
:1040840083A7C70093860700130630019305100029
:1040940017450A0013054584EFB0572197A70C0074
:1040A40083A7876283A7070083A7C70017460A0070
:1040B4001306C68397350A009385857F1385070009
:1040C400EFA04745EF00C2209307E0FD2324F4FC52
:1040D4006F10401913050009EFC04703930705004B
:1040E4002326F4FC8327C4FC639807009307A0FFEE
:1040F4002324F4FC6F1000178327C4FC23A60702B3
:10410400032704FA832744FA3367F700631A070086
:1041140013071000930700002320E4FA2322F4FA83
:10412400832744FA639C0700832744FA639A070EA3
:10413400032704FA9307F03F63F4E70E97D70C00C4
:10414400938787E203A7070083A74700B7160000F9
:104154003379D70093F9070093070900B3E73701D0
:10416400638A070AEF0002159306300017360A0027
:104174001306C66E9305B00317450A00130585C3DD
:10418400EF00D20297D70C00938787DD83A707003F
:104194006388070297A70C0083A7075383A7070028
:1041A40083A7C700938607001306E0019305100058
:1041B40017350A001305C574EFB0570F6F00C0021E
:1041C40097A70C0083A7475083A7070083A7C700BE
:1041D40093860700130610019305100017350A0093
:1041E40013050574EFB0970C97A70C0083A7C74D70
:1041F40083A7070083A7C700938607001306F0026E
:104204009305100017350A001305C572EFB0170A9D
:10421400EF00020C930720FE2324F4FC6F108004AB
:10422400832704FA13FA1700832744FA93FA070042
:1042340093070A00B3E7570163800712832704FA40
:1042440013FB2700832744FA93FB070093070B0013
:10425400B3E7770163900702832704FA13FD47004D
:10426400832744FA93FD070093070D00B3E7B701D2
:104274006384070E97D70C00938707CF03A7070023
:1042840083A74700B7160000337CD70093FC0700D0
:1042940093070C00B3E79701638A070AEF008201D2
:1042A4009306300017360A001306465B9305E003B5
:1042B40017450A00130505B0EF00426F97D70C00AD
:1042C400938707CA83A707006388070297A70C0090
:1042D40083A7873F83A7070083A7C70093860700A8
:1042E4001306E0019305100017350A001305456114
:1042F400EFB0C77B6F00C00297A70C0083A7C73C31
:1043040083A7070083A7C70093860700130610013D
:104314009305100017350A0013058560EFB007797F
:1043240097A70C0083A7473A83A7070083A7C70072
:1043340093860700130640069305100017350A00FC
:1043440013054562EFB08776EFF09178930720FE6E
:104354002324F4FC6F001071832704FA93F74700B9
:104364002328F4F8832744FA93F70700232AF4F860
:10437400832604F9032744F993870600B3E7E7008B
:1043840063820712832704FA93F727002324F4F89F
:10439400832744FA93F707002326F4F8832684F846
:1043A4000327C4F893870600B3E7E700638C070E7E
:1043B40097D70C00938747BB03A7070083A7470041
:1043C400B7160000B376D7002320D4F893F707007C
:1043D4002322F4F8832604F8032744F8938706007D
:1043E400B3E7E700638A070AEFF0D16C9306300065
:1043F40017360A00130686469305300417450A004B
:104404001305459BEF00825A97D70C00938747B555
:1044140083A707006388070297A70C0083A7C72A0E
:1044240083A7070083A7C700938607001306E0014C
:104434009305100017350A001305854CEFB0076784
:104444006F00C00297A70C0083A7072883A7070063
:1044540083A7C70093860700130610019305100075
:1044640017350A001305C54BEFB0476497A70C0036
:1044740083A7872583A7070083A7C7009386070020
:10448400130660049305100017350A00130505543C
:10449400EFB0C761EFF0D163930720FE2324F4FC4F
:1044A4006F00505C832704FA93F78700232CF4F6FB
:1044B400832744FA93F70700232EF4F6832684F720
:1044C4000327C4F793870600B3E7E700638807145C
:1044D400832704FA93F707012328F4F6832744FA81
:1044E40093F70700232AF4F6832604F7032744F7F7
:1044F40093870600B3E7E70063980702832704FA6B
:1045040093F707022324F4F6832744FA93F707006A
:104514002326F4F6832684F60327C4F6938706003D
:10452400B3E7E700638C070E97D70C009387C7A304
:1045340003A7070083A74700B7160000B376D70088
:104544002320D4F693F707002322F4F6832604F6F7
:10455400032744F693870600B3E7E700638A070A54
:10456400EFF051559306300017360A001306062F54
:104574009305700417450A001305C583EF00024331
:1045840097D70C009387C79D83A70700638807020A
:1045940097A70C0083A7471383A7070083A7C70027
:1045A400938607001306E0019305100017350A00EF
:1045B40013050535EFB0874F6F00C00297A70C00B5
:1045C40083A7871083A7070083A7C70093860700E4
:1045D400130610019305100017350A00130545341E
:1045E400EFB0C74C97A70C0083A7070E83A707005B
:1045F40083A7C700938607001306E00693051000FF
:1046040017350A0013050541EFB0474AEFF0514C46
:10461400930720FE2324F4FC6F00D044832704FA7C
:1046240093F70708232CF4F4832744FA93F707003D
:10463400232EF4F4832684F50327C4F59387060018
:10464400B3E7E70063820712832704FA93F707109E
:104654002328F4F4832744FA93F70700232AF4F475
:10466400832604F5032744F593870600B3E7E700A0
:10467400638C070E97D70C009387078F03A7070057
:1046840083A74700B7160000B376D7002324D4F4D9
:1046940093F707002326F4F4832684F40327C4F451
:1046A40093870600B3E7E700638A070AEFF09140B7
:1046B4009306300017360A001306461A9305C00401
:1046C40017350A001305056FEF00422E97D70C002B
:1046D4009387078983A707006388070297A70C00BD
:1046E40083A787FE83A7070083A7C70093860700D5
:1046F4001306E0019305100017350A001305452041
:10470400EFB0C73A6F00C00297A70C0083A7C7FB9E
:1047140083A7070083A7C700938607001306100129
:104724009305100017350A001305851FEFB00738ED
:1047340097A70C0083A747F983A7070083A7C7009F
:1047440093860700130600059305100017350A0029
:1047540013054533EFB08735EFF09137930720FE0B
:104764002324F4FC6F001030832704FA93F7072006
:104774002320F4F4832744FA93F707002322F4F464
:10478400832604F4032744F493870600B3E7E70081
:1047940063880714832704FA93F70710232CF4F291
:1047A400832744FA93F70700232EF4F2832684F335
:1047B4000327C4F393870600B3E7E700639807026F
:1047C400832704FA93F707082328F4F2832744FA8B
:1047D40093F70700232AF4F2832604F3032744F310
:1047E40093870600B3E7E700638C070E97C70C00B6
:1047F4009387877703A7070083A74700B7160000AE
:10480400B376D7002324D4F293F707002326F4F2D7
:10481400832684F20327C4F293870600B3E7E700F4
:10482400638A070AEFF011299306300017360A004D
:104834001306C6029305000517350A0013058557AC
:10484400EF00C21697C70C009387877183A70700F0
:104854006388070297A70C0083A707E783A70700CD
:1048640083A7C700938607001306E0019305100091
:1048740017350A001305C508EFB047236F00C002BF
:1048840097A70C0083A747E483A7070083A7C70063
:1048940093860700130610019305100017350A00CC
:1048A40013050508EFB0872097A70C0083A7C7E17D
:1048B40083A7070083A7C700938607001306200772
:1048C4009305100017350A0013050521EFB0071EE4
:1048D400EFF01120930720FE2324F4FC6F009018BE
:1048E4008327C4F963980714832704FA93F787008E
:1048F4002320F4F2832744FA93F707002322F4F2E7
:10490400832604F2032744F293870600B3E7E70003
:1049140063980702832704FA93F70702232CF4F021
:10492400832744FA93F70700232EF4F0832684F1B7
:104934000327C4F193870600B3E7E70063820724E3
:1049440097C70C009387476203A7070083A7470014
:10495400B7160000B376D7002328D4F093F70700E6
:10496400232AF4F0832604F1032744F193870600F5
:10497400B3E7E700638A070AEFF0D1139306300028
:1049840017360A00130686ED9305700517350A00DD
:1049940013054542EF00820197C70C009387475CDB
:1049A40083A707006388070297A70C0083A7C7D1D2
:1049B40083A7070083A7C700938607001306100286
:1049C4009305100017350A0013054518EFB0070EBC
:1049D4006F00C00297A70C0083A707CF83A7070027
:1049E40083A7C700938607001306400193051000B0
:1049F40017350A001305C517EFB0470B97A70C002E
:104A040083A787CC83A7070083A7C70093860700E3
:104A1400130680039305100017350A001305C51605
:104A2400EFB0C708EFF0D10A9307B0FD2324F4FCDC
:104A34006F005003832704FA93F787002324F4F0CC
:104A4400832744FA93F707002326F4F0832684F09F
:104A54000327C4F093870600B3E7E70063920712C5
:104A6400832704FA93F707022320F4F0832744FAF8
:104A740093F707002322F4F0832604F0032744F07D
:104A840093870600B3E7E700639C070E97C70C0003
:104A94009387874D03A7070083A74700B716000035
:104AA400B376D700232CD4EE93F70700232EF4EE2D
:104AB400832684EF0327C4EF93870600B3E7E70058
:104AC400638A070AEFF0017F9306300017360A0065
:104AD4001306C6D89305D00517350A001305852D8E
:104AE400EFF0D16C97C70C009387874783A7070023
:104AF4006388070297A70C0083A707BD83A7070055
:104B040083A7C700938607001306100293051000BD
:104B140017350A0013058503EFA057796F00C0020B
:104B240097A70C0083A747BA83A7070083A7C700EA
:104B340093860700130640019305100017350A00F9
:104B440013050503EFA0977697A70C0083A7C7B7B3
:104B540083A7070083A7C7009386070013062004D2
:104B64009305100017350A001305C505EFA0177447
:104B7400EFF001769307B0FD2324F4FC6F00806E00
:104B84008327C4FA83A7C701032784FA63F0E710D5
:104B940097C70C009387473D03A7070083A74700E7
:104BA400B7160000B376D7002328D4EE93F7070096
:104BB400232AF4EE832604EF032744EF93870600A9
:104BC400B3E7E700638E070AEFF0C16E9306300087
:104BD40017360A00130686C89305200617350A00FF
:104BE4001305451DEFF0915C97C70C009387473779
:104BF40083A707006388070297A70C0083A7C7ACA5
:104C040083A7070083A7C700938607001306400203
:104C14009305100017350A001305C5C4EFA01769E2
:104C24006F00C00297A70C0083A707AA83A70700F9
:104C340083A7C7009386070013067001930510002D
:104C440017350A00130585C4EFA0576697A70C0013
:104C540083A787A783A7070003A7C7008327C4FAEE
:104C640083A7C70193860700032684FA97350A00B1
:104C7400938585F913050700EF90D709EFF0416597
:104C8400930730FC2324F4FC6F00C05D8327C4FC2D
:104C94001307100023A2E7008327C4FC23AE0702F6
:104CA4008327C4FC23A207028327C4FC23AC070286
:104CB4008327C4FC23AE07068327C4FC23A0070470
:104CC4008327C4FC371700001307070F23A4E7004A
:104CD4008326C4FC032704FA832744FA23A8E600A6
:104CE40023AAF6008327C4FC23A407048327C4FC57
:104CF40023AA07028327C4FC23A007088327C4FC34
:104D040023A207088327C4FC23A4070897B70C0031
:104D1400938707A383A70700930500011385070062
:104D2400EF80973693070500138707008327C4FC99
:104D340023A6E7028327C4FC83A7C702639C070E4C
:104D440097C70C009387472203A7070083A7470050
:104D5400B7160000B376D7002324D4EE93F70700E8
:104D64002326F4EE832684EE0327C4EE93870600FD
:104D7400B3E7E700638A070AEFF0C15393063000F4
:104D840017360A00130686AD9305C00717350A00C7
:104D940013054502EFF0914197C70C009387471C18
:104DA40083A707006388070297A70C0083A7C7910E
:104DB40083A7070083A7C700938607001306300262
:104DC4009305100017350A00130505E9EFA0174EE7
:104DD4006F00C00297A70C0083A7078F83A7070063
:104DE40083A7C7009386070013066001930510008C
:104DF40017350A00130585E8EFA0574B97A70C0059
:104E040083A7878C83A7070083A7C70017360A00E8
:104E1400130646E897350A00938585A9138507008C
:104E2400EF90476FEFF0C14A9307A0FF2324F4FCEF
:104E34006F004043232204FC6F0000088327C4FA58
:104E440003A78700832744FC93972700B307F70041
:104E540083A7070083A7471A232CF4FA8327C4FAED
:104E640003A78700832744FC93972700B307F70021
:104E740003A707008327C4FC83A6C702832784FBF8
:104E840093974700B387F6000327871A23A2E70006
:104E94008327C4FC03A7C702832744FC93974700D6
:104EA400B307F7001307100023A0E700832744FC8F
:104EB400938717002322F4FC8327C4FA83A70701EE
:104EC400032744FCE36CF7F68327C4FC032784FA26
:104ED40023ACE7008327C4FC23AE07008327C4FC6C
:104EE4000327C4FA23A4E7028327C4FC0327C4F9D5
:104EF40023A0E7028327C4FC23A807028327C4FA5C
:104F040083A70705638007048327C4FA83A70705DB
:104F140083A7472503A747048327C4FA83A7070564
:104F24000326C4F98325C4FC13850700E7000700A2
:104F340093070500638807009307C0FF2324F4FC4C
:104F44006F00C02C232204FC6F00400B8327C4FA9B
:104F540003A707058327C4FA83A68700832744FC95
:104F640093972700B387F60083A707006300F70829
:104F74008327C4FA03A78700832744FC9397270059
:104F8400B307F70083A70700232EF4FA8327C4FB93
:104F940083A7472583A747046392070297360A002D
:104FA400938606D117360A001306C6E09305100A45
:104FB40017350A00130505D2EF80477C8327C4FB0D
:104FC40083A7472583A747040326C4F98325C4FC84
:104FD4000325C4FBE780070093070500638A0700E5
:104FE4009307C0FF2324F4FC6F0040221300000049
:104FF400832744FC938717002322F4FC8327C4FAF5
:1050040083A70701032744FCE362F7F4832704FA28
:1050140093F707012320F4EE832744FA93F707005C
:105024002322F4EE832604EE032744EE938706003E
:10503400B3E7E700638607068327C4FC83A7070258
:10504400639007068327C4FC83A7070363820702D0
:1050540097360A009386C6C917360A00130686D502
:105064009305C00A17350A001305C5C6EF800771FA
:10507400832584FA13050008EF905159130705009E
:105084008327C4FC23A0E7028327C4FC83A7070269
:10509400639807009307A0FF2324F4FC6F00001714
:1050A4008327C4FA83A747006342F00297360A00B5
:1050B4009386C6C617360A001306C6CF9305500B4F
:1050C40017350A00130505C1EF80476B8327C4FA1F
:1050D40083A74700138717008327C4FA23A2E70096
:1050E4008327C4FA83A7470063D2070297360A00CE
:1050F4009386C6C417360A001306C6CB9305500B15
:1051040017350A00130505BDEF80476797C70C00E4
:10511400938787E503A7070083A7470093762700B3
:10512400232CD4EC93F70700232EF4EC832684ED90
:105134000327C4ED93870600B3E7E700638C070AEF
:10514400EFF041179306100017360A00130606C144
:105154009305700B17350A001305C5C5EFF011054B
:1051640097C70C009387C7DF83A7070063880702EC
:1051740097970C0083A7475583A7070083A7C70009
:10518400938607001306E0009305100017350A0004
:10519400130545BDEFA097116F00000297970C000F
:1051A40083A7875283A7070083A7C70093850700B7
:1051B40013050002EF90474097970C0083A7C75050
:1051C40083A7070003A5C7008327C4FC83A607029F
:1051D4008327C4FC83A7C70203A78700832784FA15
:1051E4000326C4FC97350A009385C5B8EF9087322F
:1051F400EFF0010E832784F963860700832784F97F
:1052040023A007008327C4FC6F00000A232004FCAA
:105214006F0040048327C4FA03A78700832704FC94
:1052240093972700B307F70083A70700232EF4FA08
:105234008327C4FB83A7472583A787048325C4FC4E
:105244000325C4FBE7800700832704FC938717002A
:105254002320F4FC032704FC832744FCE36CF7FAC3
:10526400130000008327C4FC638E07008327C4FC5B
:1052740083A7C70213850700EFA0176A8327C4FC1E
:1052840023A607020325C4FCEFA01769232604FC08
:10529400832784F963880700832784F9032784FC20
:1052A40023A0E70093070000138507008320C112A1
:1052B400032481120329411283290112032AC111F3
:1052C400832A8111032B4111832B0111032CC1105B
:1052D400832C8110032D4110832D01101301011320
:1052E40067800000130101F9232611062324810697
:1052F4002322210723203107232E4105232C510586
:10530400232A610523287105232681052324910579
:105314002322A1052320B10513040107232EA4FA97
:10532400232CB4FA232AC4FA2328D4FA2326E4FA31
:105334002324F4FA232204FB232014FB232004FC5B
:105344008327C4FB6392070E97C70C009387C7C1DA
:1053540003A7070083A74700B7160000337DD700D3
:1053640093FD070093070D00B3E7B701638A070AAB
:10537400EFE051749306300017360A001306C6A4F2
:105384009305D00217350A00130585D7EFF00162A3
:1053940097C70C009387C7BC83A7070063880702DD
:1053A40097970C0083A7473283A7070083A7C700FA
:1053B40093860700130660029305100017350A0050
:1053C400130505A1EFA0876E6F00C00297970C002C
:1053D40083A7872F83A7070083A7C70093860700A7
:1053E400130690019305100017350A001305C5A094
:1053F400EFA0C76B97970C0083A7072D83A707001F
:1054040083A7C70017360A001306C6A097350A00FB
:105414009385C5A113850700EF90C70FEFE0516B8B
:105424009307C0FD6F00007D832784FB6392070E02
:1054340097C70C00938747B303A7070083A74700C8
:10544400B7160000337CD70093FC070093070C00C9
:10545400B3E79701638A070AEFE0D165930630004A
:1054640017360A00130646969305F00217350A000C
:10547400130505C9EFF0815397C70C00938747AE16
:1054840083A707006388070297970C0083A7C723A5
:1054940083A7070083A7C70093860700130630027B
:1054A4009305100017350A0013058598EFA00760CF
:1054B4006F00C00297970C0083A7072183A70700FA
:1054C40083A7C700938607001306600193051000A5
:1054D40017350A0013050598EFA0475D97970C0050
:1054E40083A7871E83A7070083A7C70017360A0070
:1054F4001306C69797350A009385459313850700CD
:10550400EF904701EFE0D15C9307A0FD6F00806E40
:10551400832784FB83A7C70363800710832784FB47
:1055240003A7C7018327C4FB83A7C70083A7C70BAF
:10553400B377F7026382070E97C70C009387C7A25D
:1055440003A7070083A74700B7160000337BD700E3
:1055540093FB070093070B00B3E77701638A070AFD
:10556400EFE051559306300017360A001306C6853E
:105574009305100317350A00130585B8EFF00143AE
:1055840097C70C009387C79D83A70700638807020A
:1055940097970C0083A7471383A7070083A7C70027
:1055A400938607001306D0029305100017350A00EE
:1055B4001305058DEFA0874F6F00C00297970C006D
:1055C40083A7871083A7070083A7C70093860700D4
:1055D400130600029305100017350A001305458DC4
:1055E400EFA0C74C97970C0083A7070E83A707006B
:1055F40083A7C700938607001306100393051000C2
:1056040017350A001305058DEFA0474AEFE0514C0A
:10561400930730FF6F00005E8327C4FB03A7870056
:10562400832784FB83A787026302F70E97C70C00C6
:105634009387879303A7070083A74700B716000043
:10564400337AD70093FA070093070A00B3E75701A8
:10565400638A070AEFE011469306300017260A0012
:10566400130686769305300317350A00130545A9FA
:10567400EFF0C13397C70C009387878E83A7070089
:105684006388070297970C0083A7070483A7070082
:1056940083A7C70093860700130600029305100032
:1056A40017350A0013054586EFA047406F00C00276
:1056B40097970C0083A7470183A7070083A7C70018
:1056C40093860700130630019305100017350A006E
:1056D4001305C585EFA0873D97970C0083A7C7FEE8
:1056E40083A7070083A7C7009386070013067003E8
:1056F4009305100017350A0013058584EFA0073BB6
:10570400EFE0113D9307E0FD6F00C04E832784FB5B
:1057140003A7070183A74701137F072893FF070007
:1057240093070F00B3E7F7016382070E97C70C00D6
:105734009387878303A7070083A74700B716000052
:10574400337ED70093FE070093070E00B3E7D7011B
:10575400638A070AEFE011369306300017260A0021
:10576400130686669305600317350A0013054599E9
:10577400EFF0C12397B70C009387877E83A70700B8
:105784006388070297970C0083A707F483A7070091
:1057940083A7C70093860700130620029305100011
:1057A40017250A001305457DEFA047306F00C0029E
:1057B40097970C0083A747F183A7070083A7C70027
:1057C40093860700130650019305100017250A005D
:1057D4001305C57CEFA0872D97970C0083A7C7EE10
:1057E40083A7070083A7C700938607001306D00486
:1057F4009305100017250A001305C57BEFA0072B9E
:10580400EFE0112D930750FC6F00C03E832784FA0C
:105814006392070E97B70C009387077503A70700D9
:1058240083A74700B71600003373D70093F307002C
:1058340093070300B3E77700638A070AEFE0912731
:105844009306300017260A00130606589305C00372
:1058540017350A001305C58AEFF0411597B70C00F8
:105864009387077083A707006388070297970C0044
:1058740083A787E583A7070083A7C700938607004C
:105884001306E0019305100017250A001305857718
:10589400EFA0C7216F00C00297970C0083A7C7E24F
:1058A40083A7070083A7C700938607001306100188
:1058B4009305100017250A001305C576EFA0071FEE
:1058C40097970C0083A747E083A7070083A7C70027
:1058D40017260A001306467697250A009385055570
:1058E40013850700EF801743EFE0911E930720FE16
:1058F4006F004030832784FB0326C4FA832504FB0E
:1059040013850700EFA0D1219307050063860700E4
:10591400930720FE6F00002E832784FB83A7C70311
:1059240063820702832784FB83A7C701032704FB41
:10593400B307F7002328F4FA832784FB83A7C7035C
:10594400232CF4FA832784FB83A78701232CF4F800
:10595400232E04F88327C4FB83A7C70003A70708E3
:1059640083A74708032584F98325C4F91386050012
:105974009386070063EEC60013860500938607002E
:105984006318D60E930605009307070063F2D70E3B
:1059940097B70C009387475D03A7070083A74700C9
:1059A400B71600003379D70093F90700930709006D
:1059B400B3E73701638A070AEFE0D10F930630009B
:1059C40017260A00130646409305300417250A00DB
:1059D40013050573EFE0917D97B70C009387475843
:1059E40083A707006388070297970C0083A7C7CD96
:1059F40083A7070083A7C700938607001306100236
:105A04009305100017250A0013050564EFA0070A83
:105A14006F00C00297970C0083A707CB83A70700EA
:105A240083A7C7009386070013064001930510005F
:105A340017250A0013058563EFA0470797970C0005
:105A440083A787C883A7070083A7C7009386070097
:105A5400130620039305100017250A001305856219
:105A6400EFA0C704EFE0D1069307B0FF6F008018E2
:105A7400032604FA832544FA0325C4FBEFC0D10F9F
:105A84002324A4FC832784FC63860700832784FCE7
:105A94006F0040168327C4FB83A7C7001385070044
:105AA400EFC0811D2322A4FC232604FC6F004003C5
:105AB4008327C4FB83A7870003A787008327C4FC2D
:105AC40093972700B307F70083A70700032744FC35
:105AD4006304F7028327C4FC938717002326F4FC8E
:105AE4008327C4FB83A7870083A707010327C4FC7C
:105AF400E360F7FC6F008000130000008327C4FB01
:105B040083A7870083A707010327C4FC6362F70206
:105B140097260A009386465A17260A001306465EFD
:105B24009305C00417250A001305855BEF7017451C
:105B3400032744FA930784FB130504FC93880700A6
:105B440013081000832704FA832604003716000084
:105B54001306361F8325C4FBEF90512D2324A4FC88
:105B6400832784FC63860700832784FC6F008008F6
:105B7400832704FC032784FA23A0E700832784FBFC
:105B840083A6C702832744FC83A7471A13974700B9
:105B9400832704FC3387E60023A2E700832704FC61
:105BA400032704FB23A4E700832704FC0327C4FA88
:105BB40023A6E700832784FB13850700EF00406BCF
:105BC400832784FB0327C4FB0327C70023AAE70218
:105BD400832704FC938507000325C4FBEF90117110
:105BE400832744FB638607000325C4FBEF60C1429F
:105BF40093070000138507008320C1060324810650
:105C04000329410683290106032AC105832A810544
:105C1400032B4105832B0105032CC104832C810430
:105C2400032D4104832D0104130101076780000043
:105C3400130101FA232E1104232C8104232A2105A4
:105C44002328310523264105232451051304010685
:105C54002326A4FA232804FC8325C4FA6392050EA0
:105C640097B70C009387473003A7070083A7470023
:105C7400B71500003376B70093F6070093070600C4
:105C8400B3E7D700638A070AEFE0C16293063000E6
:105C940017260A00130646489305500217250A00E2
:105CA4001305C557EFE0915097B70C009387472B26
:105CB40083A707006388070297970C0083A7C7A0F0
:105CC40083A7070083A7C700938607001306300243
:105CD4009305100017250A0013058544EF90175DFE
:105CE4006F00C00297970C0083A7079E83A7070045
:105CF40083A7C7009386070013066001930510006D
:105D040017250A0013050544EF90575A97970C007E
:105D140083A7879B83A7070083A7C70017260A00CA
:105D24001306C64397250A00938585441385070007
:105D3400EF80477EEFE0C1599307A0FD6F0000514B
:105D44008326C4FA83A686022326D4FC8326C4FAB7
:105D540083A646006342D00297260A0093868641B2
:105D640017260A001306864B9305900217250A008E
:105D740013050542EF7097208326C4FA83A64600D4
:105D84009386F6FF0326C4FA2322D6002324D4FCE8
:105D94008326C4FA83A6460063D2060297260A0025
:105DA4009386064117260A00130646479305900278
:105DB40017250A001305C53DEF70571C97B60C0054
:105DC4009386861A03A6060083A646001377060464
:105DD40093F7060093060700B3E6F6006384060A09
:105DE400EFE0414D9306100017260A001306463EC5
:105DF4009305B00217250A0013054542EFE0113B55
:105E040097B70C009387C71583A707006388070219
:105E140097970C0083A7478B83A7070083A7C70026
:105E2400938607001306E0009305100017250A0067
:105E34001305C53AEF9097476F00000297970C003F
:105E440083A7878883A7070083A7C70093850700D4
:105E540013050002EF80477697970C0083A7C78647
:105E640083A7070083A7C700832684FC0326C4FAFC
:105E740097250A009385853713850700EF80876986
:105E8400EFE00145832784FC6390073C8327C4FA31
:105E940083A78704638607068327C4FA03A78700BA
:105EA400B71700009387670F631CF7048327C4FAAE
:105EB40083A7C7072322F4FC832744FC63920702C9
:105EC40097260A009386063417260A001306063519
:105ED4009305A00317250A001305852BEF70170AF5
:105EE400032544FCEFF0DFD42320A4FC0325C4FAEB
:105EF400EFA08722232604FA832704FC6F000035D1
:105F040097B70C009387470603A7070083A74700AA
:105F1400137A070493FA070093070A00B3E75701BB
:105F24006382070AEFE001399306100017260A007E
:105F34001306062A9305000417250A001305052EE7
:105F4400EFE0D12697B70C009387870183A707005A
:105F54006388070297870C0083A7077783A7070046
:105F640083A7C700938607001306E000930510007B
:105F740017250A0013058526EF9057336F0000029A
:105F840097870C0083A7477483A7070083A7C700DC
:105F94009385070013050002EF80076297870C00C2
:105FA40083A7877283A7070083A7C7000326C4FAC1
:105FB40097250A009385452513850700EF808755AB
:105FC400EFE001318327C4FA83A7C703639607125E
:105FD4008327C4FA83A70703232EF4FA232E04FC91
:105FE4006F00800E8327C4FC03A787008327C4FDAA
:105FF40093972700B307F70083A707000327C4FB81
:10600400630CF70A8327C4FC03A787008327C4FD16
:1060140093972700B307F70083A70700232CF4FA0C
:106024008327C4FA83A78704638C0704832784FB2C
:1060340083A7870863860704832784FB83A74725F0
:1060440083A7470A638E0702832784FB83A7472518
:1060540083A6470A8327C4FA03A7C702832784FBBE
:1060640083A7471A93974700B307F70083A7C7008E
:10607400138607008325C4FA032584FBE780060002
:10608400832784FB83A7472583A787048325C4FA32
:10609400032584FBE78007008327C4FA03A7C7020C
:1060A400832784FB83A7471A93974700B307F70016
:1060B40023A407006F008000130000008327C4FDA1
:1060C40093871700232EF4FC8327C4FC83A70701BE
:1060D4000327C4FDE368F7F08327C4FB638E07003E
:1060E4008327C4FB83A7472583A787048325C4FA92
:1060F4000325C4FBE78007008327C4FA83A787032B
:10610400232CF4FC6F008001032584FDEFA0C7005D
:10611400232C04FC832704FB232CF4FC832784FD19
:10612400638A0700832784FD83A707012328F4FAE1
:106134006FF09FFD8327C4FA23AC07028327C4FAB8
:1061440083A7C7032328F4FC8327C4FA83A7C703C0
:10615400639407048327C4FA03A7070183A74701AD
:106164001379070193F9070093070900B3E737018F
:10617400638407028327C4FA83A70702638E070098
:106184008327C4FA83A7070213850700EF90D77803
:106194008327C4FA23A007028327C4FA83A7C7026C
:1061A40013850700EF9057778327C4FA23A60702C5
:1061B4008327C4FA83A70704232AF4FC6F00C003CF
:1061C400832744FD03A70700832744FD83A74700D3
:1061D400938507000325C4FAE7000700832744FDDD
:1061E40083A78700232AF4FA032544FDEF90D7728E
:1061F400832744FB232AF4FC832744FDE39207FC12
:106204008327C4FA83A78704638E07008327C4FA0D
:1062140083A7470413850700EF9017708327C4FAF8
:1062240023A207040325C4FAEF90176F232604FA68
:10623400832704FD63860700032504FDEFF05F9FB9
:106244000325C4FCEFC05FCA930700001385070051
:106254008320C10503248105032941058329010500
:10626400032AC104832A8104130101066780000004
:10627400130101FE232E1100232C810013040102BB
:106284002326A4FE8325C4FE6392050E97B70C0053
:10629400938787CD03A7070083A74700B71500009E
:1062A4003376B70093F6070093070600B3E7D700E9
:1062B400638A070AEFE001009306300017260A00FC
:1062C400130646F79305D00117250A001305450563
:1062D400EFE0C16D97B70C00938787C883A70700C9
:1062E4006388070297870C0083A7073E83A70700EC
:1062F40083A7C70093860700130630029305100096
:1063040017250A00130585F3EF90477A6F00C00242
:1063140097870C0083A7473B83A7070083A7C70081
:1063240093860700130660019305100017250A00E1
:10633400130505F3EF90877797870C0083A7C73879
:1063440083A7070083A7C70017260A001306C6F20F
:1063540097250A00938585F313850700EF80871B33
:10636400EFD011779307A0FD6F0040148326C4FE7D
:1063740083A646006342D00297260A00938646F11C
:1063840017260A001306C6F99305E00117250A002B
:106394001305C5F1EF70873E8326C4FE83A646002D
:1063A400138616008326C4FE23A2C6008326C4FED9
:1063B40083A6460063D2060297260A00938606F156
:1063C40017260A001306C6F59305E00117250A00EF
:1063D4001305C5EDEF70873A97B60C009386C6B8DF
:1063E40003A6060083A646001377060493F7060067
:1063F40093060700B3E6F6006388060AEFD0916BB4
:106404009306100017260A00130646EE9305F001C2
:1064140017250A001305C5F0EFE0415997B70C00A2
:10642400938707B483A707006388070297870C0044
:1064340083A7872983A7070083A7C700938607003C
:106444001306E0009305100017250A001305C5EA9A
:10645400EF90C7656F00000297870C0083A7C726DB
:1064640083A7070083A7C7009385070013050002CD
:10647400EF80871497870C0083A7072583A707005D
:1064840003A7C7008327C4FE83A74700938607009A
:106494000326C4FE97250A00938505E71305070024
:1064A400EF804707EFD0D162930700001385070000
:1064B4008320C101032481011301010267800000CC
:1064C400130101FA232E1104232C8104232A91049D
:1064D400232821052326310513040106232EA4FABB
:1064E400232CB4FA232AC4FA2328D4FA2326E4FA60
:1064F400232E04FC232C04FC232A04FC8327C4FB42
:106504006394070E97B70C00938707A603A70700A9
:1065140083A74700B71600003373D70093F307002F
:1065240093070300B3E77700638A070AEFD0915813
:106534009306300017260A001306C6DF9305A0024F
:1065440017250A001305C5F0EFE0414697B70C0084
:10655400938707A183A707006388070297870C0026
:1065640083A7871683A7070083A7C700938607001E
:10657400130600029305100017250A00130505DC15
:10658400EF90C7526F00C00297870C0083A7C71310
:1065940083A7070083A7C70093860700130630016B
:1065A4009305100017250A00130585DBEF900750AB
:1065B40097870C0083A7471183A7070083A7C70009
:1065C40017260A00130606DB97250A009385C5DB08
:1065D40013850700EF701774EFD0914F9307E0FD18
:1065E4002326F4FC6F00C06B832784FB6394070E9F
:1065F40097B70C009387479703A7070083A7470023
:10660400B71600003378D70093F807009307080003
:10661400B3E71701638A070AEFD0D1499306300024
:1066240017260A00130606D19305C00217250A008F
:10663400130505E2EFE0813797B70C009387479283
:1066440083A707006388070297870C0083A7C707FF
:1066540083A7070083A7C700938607001306E001FA
:106664009305100017250A00130545D2EF9007443F
:106674006F00C00297870C0083A7070583A7070054
:1066840083A7C70093860700130610019305100023
:1066940017250A00130585D1EF90474197870C0011
:1066A40083A7870283A7070083A7C70017260A00CA
:1066B400130606D197250A00938505CD1385070097
:1066C400EF705765EFD0D140930720FE2326F4FCEA
:1066D4006F00005D9305002E13051000EF70C71ABC
:1066E40093070500232EF4FC8327C4FD6398070059
:1066F4009307A0FF2326F4FC6F00805A8327C4FD70
:106704001307100023A2E700232804FC6F00801A5B
:10671400832704FD93972700032744FBB307F7005F
:1067240083A707006392070E97B70C009387C7836C
:1067340003A7070083A74700B71600003379D700E3
:1067440093F9070093070900B3E737016388070A41
:10675400EFD051369306300017260A00130686BD83
:106764009305900317250A00130585CEEFE0012455
:1067740097A70C009387C77E83A707006388070247
:1067840097870C0083A747F483A7070083A7C70054
:10679400938607001306E0019305100017250A00ED
:1067A4001305C5BEEF9087306F00C00297870C00B9
:1067B40083A787F183A7070083A7C70093860700F1
:1067C400130610019305100017250A00130505BED2
:1067D400EF90C72D97870C0083A707EF83A70700C7
:1067E40083A7C700032604FD97250A00938545BEA9
:1067F40013850700EF701752EFD0912D930720FEF9
:106804002326F4FC6F00C049832704FB639A070224
:10681400832704FD93972700032744FBB307F7005E
:1068240083A7070013850700EFE047271307050038
:10683400832784FDB387E700232CF4FC6F00C00694
:10684400832704FD93972700032704FBB307F7006E
:1068540083A70700639A0702832704FD9397270001
:10686400032744FBB307F70083A70700138507003A
:10687400EFE0C72213070500832784FDB387E700F1
:10688400232CF4FC6F004002832704FD9397270018
:10689400032704FBB307F70083A70700032784FD3E
:1068A400B307F700232CF4FC832704FD9387170018
:1068B4002328F4FC032704FD832784FBE36AF7E41D
:1068C400832784FD9387170013850700EF9017042F
:1068D40093070500232AF4FC832744FD63980700EB
:1068E4009307A0FF2326F4FC6F00803B8327C4FD9D
:1068F400032744FD23ACE700232804FC6F000017A2
:10690400832704FB639C0706832704FD93972700D2
:10691400032744FBB307F70083A40700832704FD80
:1069240093972700032744FBB307F70083A70700C7
:1069340013850700EFE08716930705001386070009
:1069440093850400032544FDEFA0C725832704FD98
:1069540093972700032744FBB307F70083A7070097
:1069640013850700EFE0871313070500832744FD11
:10697400B387E700232AF4FC6F00800E832704FD0D
:1069840093972700032704FBB307F70083A70700A7
:10699400639C0706832704FD93972700032744FB82
:1069A400B307F70083A40700832704FD9397270008
:1069B400032744FBB307F70083A7070013850700E9
:1069C400EFE0C70D930705001386070093850400C5
:1069D400032544FDEFA0071D832704FD939727009B
:1069E400032744FBB307F70083A7070013850700B9
:1069F400EFE0C70A13070500832744FDB387E700C8
:106A0400232AF4FC6F00C005832704FD9397270015
:106A1400032744FBB307F70083A60700832704FD7D
:106A240093972700032704FBB307F70083A7070006
:106A34001386070093850600032544FDEFA08716FF
:106A4400832704FD93972700032704FBB307F7006C
:106A540083A70700032744FDB307F700232AF4FCA8
:106A6400832704FD938717002328F4FC032704FDE0
:106A7400832784FBE366F7E8832744FD238007002C
:106A84008327C4FD0327C4FB23A4E7008327C4FB97
:106A940003A707018327C4FD23A6E7008327C4FBBC
:106AA40003A787008327C4FD23AAE7008327C4FD27
:106AB4001307F0FF23A8E72C8327C4FD23AA072C80
:106AC4008327C4FD83A7C7009305400013850700EF
:106AD400EF60975B93070500138707008327C4FDC6
:106AE40023A0E7028327C4FD83A70702638207125A
:106AF4008327C4FD83A7C7009305400013850700BF
:106B0400EF60975893070500138707008327C4FD98
:106B140023A2E7028327C4FD83A74702638A070EE3
:106B24008327C4FD83A7C70093054000138507008E
:106B3400EF60975593070500138707008327C4FD6B
:106B440023AAE7028327C4FD83A747036382070CB4
:106B54008327C4FD83A7C70093054000138507005E
:106B6400EF60975293070500138707008327C4FD3E
:106B740023A8E7028327C4FD83A70703638A0708C2
:106B84008327C4FD83A7C70093054000138507002E
:106B9400EF60974F93070500138707008327C4FD11
:106BA40023A4E7048327C4FD83A78704638207061D
:106BB4008327C4FD83A7C7009305400013850700FE
:106BC400EF60974C93070500138707008327C4FDE4
:106BD40023A6E72C8327C4FD83A7C72C638A070257
:106BE4008327C4FD83A7C70093059002138507007C
:106BF400EF60974993070500138707008327C4FDB7
:106C040023A2E7048327C4FD83A7470463980700EE
:106C14009307A0FF2326F4FC6F0080088327C4FB9E
:106C240083A747006342F00297160A009386C67B47
:106C340017260A001306C6819305B00717150A0024
:106C44001305857CEF6097338327C4FB83A7470034
:106C5400138717008327C4FB23A2E7008327C4FB01
:106C640083A7470063D2070297160A009386467CDF
:106C740017160A001306C67D9305B00717150A00F8
:106C840013058578EF60972F8327C4FA638607007E
:106C94008327C4FA23A007008327C4FD6F00000FD5
:106CA4008327C4FD6382070C8327C4FD83A747049D
:106CB40013850700EF9047468327C4FD23A20704EA
:106CC4008327C4FD83A7C72C13850700EF90C7440F
:106CD4008327C4FD23A6072C8327C4FD83A7870429
:106CE40013850700EF9047438327C4FD23A40704BB
:106CF4008327C4FD83A7470213850700EF90C7418C
:106D04008327C4FD23A207028327C4FD83A70702A8
:106D140013850700EF9047408327C4FD23A0070293
:106D24008327C4FD83A7470313850700EF90C73E5D
:106D34008327C4FD23AA07028327C4FD83A707036F
:106D440013850700EF90473D8327C4FD23A807025E
:106D54008327C4FD83A7870113850700EF90C73BF2
:106D64008327C4FD23AC07000325C4FDEF90C73A75
:106D7400232E04FC8327C4FA638807008327C4FAFC
:106D84000327C4FC23A0E700930700001385070032
:106D94008320C105032481058324410503290105BA
:106DA4008329C1041301010667800000130101B6A1
:106DB400232E1148232C8148232A91482328214932
:106DC400232631492324414923225149232061495F
:106DD400232E7147232C8147232A91472328A14737
:106DE4002326B1471304014A2326A4B82324B4B8A4
:106DF4002322C4B82320D4B8232EE4B6232CF4B61B
:106E0400232A04B7232814B7232804FA8327C4B8F1
:106E1400639C070E97A70C009387071503A7070029
:106E240083A74700B7160000B376D7002324D4B64F
:106E340093F707002326F4B6832684B60327C4B643
:106E440093870600B3E7E700638A070AEFD0814619
:106E54009306300017160A001306466193051003C3
:106E640017250A001305058EEFD0513497A70C009F
:106E74009387070F83A707006388070297870C008F
:106E840083A7878483A7070083A7C7009386070087
:106E9400130600029305100017150A001305855DFB
:106EA400EF80D7406F00C00297870C0083A7C7818B
:106EB40083A7070083A7C700938607001306300142
:106EC4009305100017150A001305055DEF80173EA2
:106ED40097770C0083A7477F83A7070083A7C70082
:106EE40017160A001306865C97150A009385455DFC
:106EF40013850700EF700762EFD0813D9307E0FD33
:106F0400232AF4FA6F009075832744B8639C070E14
:106F140097A70C009387470503A7070083A747009B
:106F2400B7160000B376D7002320D4B693F7070032
:106F34002322F4B6832604B6032744B693870600B7
:106F4400B3E7E700638A070AEFD0C136930630003F
:106F540017160A00130686519305300317150A0005
:106F64001305457EEFD0912497A70C00938747FF24
:106F740083A707006388070297770C0083A7C77469
:106F840083A7070083A7C700938607001306E001C1
:106F94009305100017150A001305C552EF80173129
:106FA4006F00C00297770C0083A7077283A70700BE
:106FB40083A7C700938607001306100193051000EA
:106FC40017150A0013050552EF80572E97770C000A
:106FD40083A7876F83A7070083A7C70017160A0034
:106FE4001306865197150A009385854D138507006E
:106FF400EF704752EFD0C12D930720FE232AF4FAF5
:107004006F00D065832784B86394070E97A70C009C
:10701400938787F503A7070083A74700B7160000E7
:10702400337DD70093FD070093070D00B3E7B70145
:10703400638A070AEFD001289306300017160A0066
:107044001306C6429305500317150A001305856FEE
:10705400EFD0D11597A70C00938787F083A707007B
:107064006388070297770C0083A7076683A7070046
:1070740083A7C700938607001306E0019305100059
:1070840017150A0013050544EF8057226F00C0024C
:1070940097770C0083A7476383A7070083A7C700DC
:1070A40093860700130610019305100017150A00B4
:1070B40013054543EF80971F97770C0083A7C7609C
:1070C40083A7070083A7C70017160A0013064644C0
:1070D40097150A009385C53E13850700EF70874313
:1070E400EFD0011F930720FE232AF4FA6F001057F4
:1070F400832704B763900722832704B86394070E99
:1071040097A70C00938747E603A7070083A74700C8
:10711400B7160000337FD70093FF070093070F00D3
:10712400B3E7F701638A070AEFD0C118930630006A
:1071340017160A00130686339305900317150A00E1
:1071440013054560EFD0910697A70C00938747E19C
:1071540083A707006388070297770C0083A7C756A5
:1071640083A7070083A7C700938607001306E001DF
:107174009305100017150A001305C534EF80171383
:107184006F00C00297770C0083A7075483A70700FA
:1071940083A7C70093860700130610019305100008
:1071A40017150A0013050534EF80571097770C0064
:1071B40083A7875183A7070083A7C70017160A0070
:1071C4001306463697150A009385852F1385070005
:1071D400EF704734EFD0C10F930720FE232AF4FA4F
:1071E4006F00D047232E04FA6F0000128327C4FBDC
:1071F40093972700032704B8B307F70083A7070072
:10720400638E07008327C4FB939727000327C4B723
:10721400B307F70083A707006392070E97A70C0034
:10722400938787D403A7070083A74700B7160000F6
:10723400337ED70093FE070093070E00B3E7D70110
:107244006388070AEFD001079306300017160A0077
:107254001306C6219305D00317150A001305854E9E
:10726400EFD0C17497A70C00938787CF83A707003B
:107274006388070297770C0083A7074583A7070055
:1072840083A7C700938607001306E0019305100047
:1072940017150A0013050523EF8057016F00C0027C
:1072A40097770C0083A7474283A7070083A7C700EB
:1072B40093860700130610019305100017150A00A2
:1072C40013054522EF80877E97770C0083A7C73F7D
:1072D40083A7070083A7C7000326C4FB97150A00EA
:1072E4009385852513850700EF70C722EFC0517E73
:1072F400930720FE232AF4FA6F0050368327C4FB39
:1073040093871700232EF4FA0327C4FB832784B83A
:10731400E36EF7EC232E04FA6F004018232604FAD8
:10732400232C04FA6F0080058327C4B803A78700C1
:107334008327C4FB93972700B307F70003A707002D
:10734400832784FB93972700832644B8B387F600EA
:1073540083A70700B307F74093B7170093F7F70F16
:10736400138707008327C4FAB387E7002326F4FAB8
:10737400832784FB93871700232CF4FA032784FBC9
:10738400832784B8E362F7FA0327C4FA930710004B
:1073940063D0E71097A70C00938707BD03A70700E6
:1073A40083A74700B71600003373D70093F3070091
:1073B40093070300B3E777006386070CEFC0916F70
:1073C4009306300017160A001306460A9305C004F4
:1073D40017150A0013050537EFD0415D97A70C0078
:1073E400938707B883A707006388070297770C0081
:1073F40083A7872D83A7070083A7C7009386070069
:107404001306F0019305100017150A00130545151E
:10741400EF80C7696F00C00297770C0083A7C72A63
:1074240083A7070083A7C7009386070013062001DC
:107434009305100017150A0013058514EF800767DC
:1074440097770C0083A7472883A7070083A6C70064
:107454008327C4B803A787008327C4FB9397270017
:10746400B307F70083A7070083A70717138607004E
:1074740097150A009385051213850600EF70870996
:10748400EFC011659307F0FD232AF4FA6F00101D75
:107494008327C4FB93871700232EF4FA8327C4B8E9
:1074A40083A707010327C4FBE36AF7E6232E04F846
:1074B4009307C4F913860700832584B8032544B8C9
:1074C400EFA011002328A4FA8327C4F92324F4B8D5
:1074D400832704FB2322F4B8232E04FA6F00C0167A
:1074E400232404FA232C04FA6F0080058327C4B8EC
:1074F40003A78700832784FB93972700B307F7002C
:1075040003A707008327C4FB93972700832644B867
:10751400B387F60083A70700B307F74093B71700B4
:1075240093F7F70F13870700832784FAB3E7E7007D
:107534002324F4FA832784FB93871700232CF4FA7B
:107544008327C4B883A70701032784FBE360F7FA02
:10755400832784FA6394070E97A70C009387C7A028
:1075640003A7070083A74700B7160000337CD700A2
:1075740093FC070093070C00B3E79701638A070A9B
:10758400EFC051539306300017160A00130606EE97
:107594009305E00517150A001305C51AEFD001413C
:1075A40097A70C009387C79B83A7070063880702EC
:1075B40097770C0083A7471183A7070083A7C70009
:1075C400938607001306F0019305100017150A00AF
:1075D400130505F9EF80874D6F00C00297770C0003
:1075E40083A7870E83A7070083A7C7009386070096
:1075F400130620019305100017150A00130545F81A
:10760400EF80C74A97770C0083A7070C83A707006E
:1076140083A7C70093860700130630039305100061
:1076240017150A00130545F9EF804748EFC0514A82
:107634009307F0FD232AF4FA6F0050028327C4FB5A
:1076440093871700232EF4FA0327C4FB832784B8F7
:10765400E368F7E89305002E13051000EF60C722D6
:10766400930705002322F4FA832744FA639807005A
:107674009307A0FF232AF4FA6F00407E832744FA7D
:107684001307100023A2E70093054000032584B8E4
:10769400EF60871F9307050013870700832744FAC9
:1076A40023A0E702832744FA83A70702638A070E0D
:1076B40093054000032584B8EF60071D9307050078
:1076C40013870700832744FA23A2E702832744FA97
:1076D40083A747026386070C93054000032584B8FB
:1076E400EF60871A9307050013870700832744FA7E
:1076F40023AAE702832744FA83A747036382070A7E
:1077040093054000032584B8EF600718930705002C
:1077140013870700832744FA23A8E702832744FA40
:1077240083A70703638E070693054000032584B8E7
:10773400EF6087159307050013870700832744FA32
:1077440023A4E704832744FA83A78704638A0704EE
:1077540093054000032584B8EF60071393070500E1
:1077640013870700832744FA23A6E72C832744FAC8
:1077740083A7C72C6386070293059002032584B868
:10778400EF6087109307050013870700832744FAE7
:1077940023A2E704832744FA83A7470463980700D6
:1077A4009307A0FF232AF4FA6F000058832744FAB2
:1077B4000327C4B823A4E700832744FA032784B823
:1077C40023A6E700832744FA032704FB23AAE70040
:1077D400832744FA1307F0FF23A8E72C832744FAEE
:1077E40023AA072C832704B7638A0700832704B8D6
:1077F400639607008327C4B76384074A232E04FAD9
:107804006F0000498327C4FB93972700032744B8DC
:10781400B307F70083A607008327C4FB93972700C9
:107824000327C4B7B307F70083A7070093850700AE
:1078340013850600EFD0115F9307050063860734B4
:107844008327C4FB93972700032704B83307F70063
:10785400832744FA83A607038327C4FB939727004F
:10786400B387F6000327070023A0E7008327C4FBA0
:1078740093972700032704B8B307F70083A60700EC
:10788400832744FA03A747038327C4FB939727005E
:10789400B304F70013850600EF805707930705002C
:1078A40023A0F400832744FA03A747038327C4FBD8
:1078B40093972700B307F70083A607008327C4FB29
:1078C400939727000327C4B7B307F70083A50700DE
:1078D4008327C4FB93972700032704B8B307F70053
:1078E40083A707001386070013850600EF90872BF4
:1078F4008327C4FB939727000327C4B7B307F70074
:1079040083A70700138607008325C4FB032544FAD5
:10791400EFD091559307C4B913870700930600006D
:10792400130600008325C4FB032544FAEF009242AA
:107934002320A4FA832704FA6384070E97970C0084
:107944009387876203A7070083A74700B716000041
:107954003379D70093F9070093070900B3E7370198
:10796400638A070AEFC011159306300017160A0040
:107974001306C6AF9305F00917150A00130585DC35
:10798400EFD0C10297970C009387875D83A7070008
:107994006388070297770C0083A707D383A70700A0
:1079A40083A7C7009386070013066002930510009F
:1079B40017150A00130585C3EF80470F6F00C00237
:1079C40097770C0083A747D083A7070083A7C70036
:1079D40093860700130690019305100017150A00FB
:1079E400130545C3EF80870C97770C0083A7C7CD99
:1079F40083A7070083A7C700938607001306100216
:107A04009305100017150A00130585C2EF80070AB5
:107A1400EFC0110C930750FF232AF4FA6F000044BF
:107A24008325C4FB032544FAEFE081109307050086
:107A34006384070E97970C009387075303A70700E7
:107A440083A74700B7160000337AD70093FA0700DC
:107A540093070A00B3E75701638A070AEFC0910549
:107A64009306300017160A00130646A09305100A61
:107A740017150A00130505CDEFC0517397970C0035
:107A84009387074E83A707006388070297770C0044
:107A940083A787C383A7070083A7C700938607002C
:107AA4001306F0019305100017150A00130585BA93
:107AB400EF70D77F6F00C00297770C0083A7C7C011
:107AC40083A7070083A7C700938607001306200136
:107AD4009305100017150A001305C5B9EF70177D3B
:107AE40097770C0083A747BE83A7070083A7C70027
:107AF400938607001306F0019305100017150A007A
:107B0400130585B8EF70977AEFC0817C930760FD09
:107B1400232AF4FA6F0080349307C4B9138507004D
:107B2400EFE0D1349307050063800704832744FA08
:107B340003A747028327C4FB93972700B306F700E4
:107B4400832744FA03A707028327C4FB93972700DC
:107B54003307F7009307C4B913060700938506009B
:107B640013850700EFE05138832784B7638C07102F
:107B74008327C4FB93972700032784B7B307F70031
:107B840023A007006F00001097970C009387C73D50
:107B940003A7070083A74700B71600009386068053
:107BA400337BD70093FB070093070B00B3E7770100
:107BB4006384070AEFC001709306200017160A00B9
:107BC400130686AE9305200B17150A00130585B717
:107BD400EFC0D15D97970C009387873883A7070080
:107BE4006388070297770C0083A707AE83A7070073
:107BF40083A7C700938607001306E00093051000CF
:107C040017150A001305C5AAEF70576A6F00000222
:107C140097770C0083A747AB83A7070083A7C70008
:107C24009385070013050002EF60171997770C007E
:107C340083A787A983A7070083A7C70093860700A4
:107C44001306B0019305100017150A00130545A784
:107C5400EF70D765EFC0C167832784B7638E0700D1
:107C64008327C4FB93972700032784B7B307F70040
:107C7400130760FD23A0E700930760FD232AF4FAAD
:107C84006F00800A8327C4FB93871700232EF4FA1E
:107C94000327C4FB832784B8E366F7B66F0080002C
:107CA400130000008327C4B883A747006342F0028F
:107CB40097160A00938686A217160A00130686A84A
:107CC4009305B00B17150A00130545A3EF50172BA6
:107CD4008327C4B883A74700138717008327C4B832
:107CE40023A2E7008327C4B883A7470063D207020F
:107CF40097160A00938606A317160A00130686A48D
:107D04009305B00B17150A001305459FEF5017276D
:107D1400832744B763860700832744B723A007005B
:107D2400832744FA6F00C015832744FA83A74702C8
:107D3400638E0704232E04FA6F008004832744FA19
:107D440003A747028327C4FB93972700B307F700D1
:107D540083A7070013850700EF80073C832744FAB5
:107D640003A747028327C4FB93972700B307F700B1
:107D740023A007008327C4FB93871700232EF4FA5C
:107D84000327C4FB832784B8E36AF7FA832744FAFA
:107D940083A7470213850700EF800738832744FA37
:107DA40023A20702832744FA83A707021385070047
:107DB400EF808736832744FA23A00702832744FAF7
:107DC40083A74703638E0704232E04FA6F008004FD
:107DD400832744FA03A747038327C4FB9397270009
:107DE400B307F70083A7070013850700EF80C732A6
:107DF400832744FA03A747038327C4FB93972700E9
:107E0400B307F70023A007008327C4FB9387170059
:107E1400232EF4FA0327C4FB832784B8E36AF7FA12
:107E2400832744FA83A7470313850700EF80C72EEF
:107E3400832744FA23AA0702832744FA83A7070364
:107E440013850700EF80472D832744FA23A80702F0
:107E5400032544FAEF80472C232204FA032504FB6C
:107E6400EF80872B232804FA832744B7638807000D
:107E7400832744B7032744FB23A0E70093070000AC
:107E8400138507008320C149032481498324414980
:107E9400032901498329C148032A8148832A414887
:107EA400032B0148832BC147032C8147832C414773
:107EB400032D0147832DC1461301014A6780000049
:107EC400130101FD2326110223248102130401035B
:107ED4002326A4FE2324B4FE2322C4FE2320D4FE9E
:107EE400232EE4FC232CF4FC232A04FD9308000035
:107EF400032844FD832784FD0327C4FD832604FE51
:107F0400032644FE832584FE0325C4FEEFE01FEA16
:107F140093070500138507008320C102032481020F
:107F24001301010367800000130101FC232E1102D9
:107F3400232C8102232A210323283103130401045F
:107F44002326A4FC8325C4FC6392050E97970C009A
:107F54009387870103A7070083A74700B71500008D
:107F64003376B70093F6070093070600B3E7D7000C
:107F7400638A070AEFC001349306300017060A002B
:107F84001306C67D9305D00217150A001305C59084
:107F9400EFC0D12197970C00938787FC83A7070034
:107FA4006388070297670C0083A7077283A70700FB
:107FB40083A7C700938607001306000293051000E9
:107FC40017050A001305057AEF70572E6F00C002DB
:107FD40097670C0083A7476F83A7070083A7C70091
:107FE40093860700130630019305100017050A0055
:107FF40013058579EF70972B97670C0083A7C76CDF
:1080040083A7070083A7C70017060A00130606798B
:1080140097050A009385C57913850700EF60874F9C
:10802400EFC0012B930740FD6F00806A8326C4FCD8
:1080340083A646006342D00297060A009386867799
:1080440017160A00130646859305F00217050A0061
:1080540013054578EF5087728326C4FC83A6460037
:108064009386F6FF0326C4FC2322D6002322D4FEE3
:108074008326C4FC83A6460063D2060297060A0040
:108084009386467717160A00130606819305F002B5
:1080940017050A0013050574EF50476E97960C00F8
:1080A400938686EC03A6060083A64600137706048F
:1080B40093F7060093060700B3E6F6006388060A02
:1080C400EFC0411F9306100017060A0013068674BA
:1080D4009305000317050A001305057CEFC0110D75
:1080E40097970C009387C7E783A707006388070265
:1080F40097670C0083A7475D83A7070083A7C70082
:10810400938607001306E0009305100017050A0084
:1081140013050571EF7097196F00000297670C0043
:1081240083A7875A83A7070083A7C70093850700FF
:1081340013050002EF60474897670C0083A7C758F0
:1081440083A7070003A5C7008327C4FC83A787036D
:1081540013870700832644FE0326C4FC97050A0000
:108164009385056DEF60073BEFC08116832744FEBE
:10817400639E07548327C4FC83A787002320F4FE4F
:1081840097970C00938747DE03A7070083A7470050
:108194001379070493F9070093070900B3E737013C
:1081A4006382070AEFC001119306100017060A0044
:1081B400130646669305500317050A001305C56D9B
:1081C400EFC0C17E97970C00938787D983A70700D8
:1081D4006388070297670C0083A7074F83A70700EC
:1081E40083A7C700938607001306E00093051000D9
:1081F40017050A001305C562EF70570B6F000002E4
:1082040097670C0083A7474C83A7070083A7C70081
:108214009385070013050002EF60073A97670C0087
:1082240083A7874A83A7070083A7C7000326C4FC44
:1082340097050A009385456313850700EF60872D32
:10824400EFC001098327C4FC83A7070463820702E4
:1082540097060A009386866217060A001306C66309
:108264009305800317050A001305C556EF500751FF
:108274008327C4FC03A747018327C4FC83A7870083
:1082840083A78700630EF7008327C4FC83A74701F5
:1082940013850700EF7057688327C4FC23AA0700DF
:1082A4008327C4FC83A7870113850700EF70D76673
:1082B4008327C4FC23AC07008327C4FC83A7872D32
:1082C40013850700EF7057658327C4FC23AC072C84
:1082D4008327C4FC83A7070213850700EF70D763C5
:1082E4008327C4FC23A007028327C4FC83A7470277
:1082F40063800706232604FE6F0080048327C4FCE2
:1083040003A747028327C4FE93972700B307F70008
:1083140083A7070013850700EF7017608327C4FC49
:1083240003A747028327C4FE93972700B307F700E8
:1083340023A007008327C4FE938717002326F4FE97
:108344008327C4FC83A7C7000327C4FEE368F7FAA6
:108354008327C4FC83A7470213850700EF70D75B0C
:108364008327C4FC23A207028327C4FC83A7070333
:1083740013850700EF70575A8327C4FC23A807020C
:108384008327C4FC83A7470363800706232604FED0
:108394006F0080048327C4FC03A747038327C4FE1C
:1083A40093972700B307F70083A7070013850700F7
:1083B400EF7097568327C4FC03A747038327C4FEA3
:1083C40093972700B307F70023A007008327C4FE71
:1083D400938717002326F4FE8327C4FC83A7C700D2
:1083E4000327C4FEE368F7FA8327C4FC83A7470383
:1083F40013850700EF7057528327C4FC23AA070292
:108404000325C4FCEF00C22E8327C4FC83A7870482
:1084140063800706232604FE6F0080048327C4FCC0
:1084240003A787048327C4FE93972700B307F700A5
:1084340083A7070013850700EF70174E8327C4FC3A
:1084440003A787048327C4FE93972700B307F70085
:1084540023A007008327C4FE938717002326F4FE76
:108464008327C4FC83A7C7000327C4FEE368F7FA85
:108474008327C4FC83A7870413850700EF70D749BB
:108484008327C4FC23A407048327C4FC83A787038E
:108494006380071E232604FE6F00001B8327C4FC91
:1084A40003A7C7038327C4FE93976700B307F700A6
:1084B400232EF4FC8327C4FD83A70701138507003B
:1084C400EF7097458327C4FD23A807008327C4FDC5
:1084D40083A7C70013850700EF7017448327C4FDE3
:1084E40023A60700232404FE6F0000088327C4FD8D
:1084F40003A74701832784FE93975700B307F70028
:1085040083A7470013850700EF7017418327C4FD35
:1085140003A74701832784FE93975700B307F70007
:1085240023A207008327C4FD03A74701832784FEF2
:1085340093975700B307F70083A707001385070035
:10854400EF70973D8327C4FD03A74701832784FE6B
:1085540093975700B307F70023A00700832784FEEF
:10856400938717002324F4FE8327C4FD83A7070001
:10857400032784FEE36CF7F68327C4FD83A7470132
:1085840013850700EF7057398327C4FD23AA07001A
:108594008327C4FD83A78703638E0704232404FE73
:1085A4006F0040048327C4FD03A78703832784FE49
:1085B40093972700B307F70083A70700638E07008C
:1085C4008327C4FD03A78703832784FE939727008B
:1085D400B307F70023A00700832784FE93871700BF
:1085E4002324F4FE8327C4FC83A7C700032784FE47
:1085F400E36AF7FA8327C4FD83A78703138507007B
:10860400EF7097318327C4FD23AC07028327C4FD91
:1086140083A7870013850700EF7017308327C4FDF5
:1086240023A407008327C4FD83A7C702138507007B
:10863400EF70972E8327C4FD23A607028327C4FE69
:10864400938717002326F4FE8327C4FC83A787039C
:108654000327C4FEE364F7E48327C4FC83A7C703AA
:1086640013850700EF70572B8327C4FC23AE070242
:108674008327C4FC83A7470413850700EF70D72919
:108684008327C4FC23A207048327C4FC83A7C70150
:1086940013850700EF7057288327C4FC23AE070017
:1086A4008327C4FC83A7C72C13850700EF70D72644
:1086B4008327C4FC23A6072C0325C4FCEF70D7250D
:1086C400232604FC032504FEEFA01F829307000069
:1086D400138507008320C103032481030329410375
:1086E400832901031301010467800000130101FBC6
:1086F4002326110423248104130401052326A4FE44
:108704002324B4FE2322C4FE2320D4FE232EE4FC1F
:10871400232CF4FC832784FD2328F1008327C4FD44
:108724002326F10023240100232201002320010039
:108734009308000013080000832704FE032744FE67
:10874400832684FE0326C4FE93051000130510003F
:10875400EF10806493070500138507008320C1048C
:10876400032481041301010567800000130101F350
:108774002326110C2324810C2322210D2320310DC7
:10878400232E410B232C510B232A610B2328710B1D
:108794002326810B2324910B2322A10B2320B10B2D
:1087A4001304010D232EA4F6232CB4F6232AC4F6B5
:1087B4002328D4F62326E4F62324F4F6232204F70C
:1087C400232014F7232404FC232404F8832744F6E9
:1087D40023A00700832704F623A0070083270400AF
:1087E40023A007008327440023A00700232204FCBE
:1087F400832744F723800700832784F72380070017
:10880400832784F6638E07008327C4F663860700F4
:10881400930750FD6F0000019307D0FB6F008000A9
:108824009307E0FB232EF4FA8327C4F7639207022D
:1088340097060A009386462417160A001306C6CF25
:108844009305000E17050A0013058523EF401773DF
:10885400832784F76392070297060A009386C62348
:1088640017160A00130646CD9305100E17050A00C5
:1088740013050521EF4097708327C4F6639607021A
:10888400832784F66392070297060A009386C6211B
:1088940017160A00130646CA9305200E17050A0088
:1088A4001305051EEF40976D930710002320F4FC79
:1088B400232C04FA0325C4F7EFC0471E93070500D1
:1088C4009387170013850700EF705704930705007B
:1088D400232AF4FA8325C4F7032544FBEFA0974821
:1088E400930784F81386070097050A009385451DAE
:1088F400032544FBEFE007242324A4FC6F100000AD
:108904001306300097050A009385C51B032584FCD4
:10891400EFC0872193070500638E0702130620002A
:1089240097050A009385451A032584FCEFC0C71FE9
:1089340093070500638007021306700097050A0079
:108944009385C518032584FCEFC0071E9307050013
:10895400639A0740832584FC17050A0013058508DC
:10896400EFC047749307050063840718832784F6D0
:10897400638C07128327C4F663980712832744FC89
:10898400639E071097870C009387075E03A7070071
:1089940083A74700B71600003379D70093F907007F
:1089A40093070900B3E737016382070AEFB0911018
:1089B4009306300017060A001306C6119305800FAC
:1089C40017150A00130545B7EFB0517E97870C00C1
:1089D4009387075983A707006388070297670C00EA
:1089E40083A787CE83A7070083A7C70093860700C2
:1089F4001306E0009305100017050A001305050E81
:108A0400EF70C70A6F00000297670C0083A7C7CBFB
:108A140083A7070083A7C7009385070013050002F7
:108A2400EF50973997670C0083A707CA83A70700FD
:108A340083A7C700032684FC97050A009385050BCA
:108A440013850700EF50172DEFB09108832704F723
:108A54009387C70413850700EFC04704232AA4F8AB
:108A6400832704F71387C704832744F93305F700E2
:108A740013070028832744F9B307F740832684FCAF
:108A840017060A001306860693850700EFA0C7346D
:108A94008327C4FB2326F4FC6F00106C832584FC1D
:108AA400032544F7EFA0877797050A0093854509C6
:108AB400032584FCEFC0075F930705006388070064
:108AC400832704F61307100023A0E70097050A0084
:108AD40093858508032584FCEFC0C75C93070500D4
:108AE40063880700832704001307100023A0E7000E
:108AF400832584FC17050A00130545DBEFC0875A5C
:108B040093070500E39A0754832584FC17050A009C
:108B1400130585F4EFC0075993070500638807120E
:108B240097870C009387474403A7070083A7470050
:108B3400B7160000337AD70093FA070093070A00A8
:108B4400B3E757016382070AEFB0C176930630009A
:108B540017060A00130606F89305101117150A00E4
:108B64001305859DEFB0916497870C009387473F69
:108B740083A707006388070297670C0083A7C7B41D
:108B840083A7070083A7C700938607001306E000A6
:108B94009305100017050A00130545F4EF601771DB
:108BA4006F00000297670C0083A707B283A7070032
:108BB40083A7C7009385070013050002EF50D71F52
:108BC40097670C0083A747B083A7070083A7C70054
:108BD400032684FC97050A00938585FA138507000C
:108BE400EF505713EFB0C16E832704F79387C70480
:108BF40013850700EFB0976A2326A4F8832704F7A8
:108C04001387C7048327C4F83305F7001307002824
:108C14008327C4F8B307F740832684FC17060A00A9
:108C2400130606F693850700EFA0071B930784F845
:108C34001386070097050A00938585E8130500004D
:108C4400EFD0576F2324A4FC6F00504B97870C0080
:108C54009387873103A7070083A74700B71600004F
:108C6400337BD70093FB070093070B00B3E777012F
:108C74006382070AEFB001649306300017060A0006
:108C8400130646E59305901117150A001305C58AC6
:108C9400EFB0D15197870C009387872C83A70700E7
:108CA4006388070297670C0083A707A283A70700BE
:108CB40083A7C700938607001306E00093051000FE
:108CC40017050A00130585E1EF60575E6F00000287
:108CD40097670C0083A7479F83A7070083A7C70054
:108CE4009385070013050002EF50170D97670C00DA
:108CF40083A7879D83A7070083A7C700032684FC57
:108D040097050A00938545EB13850700EF509700FC
:108D1400EFB0015C832704F79387C704138507002A
:108D2400EFB0D7572328A4F8832704F71387C70481
:108D3400832704F93305F70013070028832704F970
:108D4400B307F740832684FC17060A001306C6E619
:108D540093850700EFA047088327C4FB2326F4FC70
:108D64006F00903F1306200097050A00938585E65F
:108D7400032584FCEFB0575B93070500639A070053
:108D840097070A00938747E52324F4FC6F00D02C4F
:108D94001306200097050A00938545E9032584FC02
:108DA400EFB097589307050063800702130620006D
:108DB40097050A009385C5E7032584FCEFB0D756D1
:108DC400930705006390070E032584FCEFB0174D4D
:108DD4009307050093871700232CF4FA032704FC58
:108DE400832784FBB307F7000327840063E2E702C9
:108DF40097060A00938606E417060A001306C6734C
:108E04009305501217050A00130585C7EF4017177D
:108E1400032704FC832784FBB307F7002320F4FC17
:108E2400832584FC032584F7EFA0473F032584F7BB
:108E3400EFB0D7469307050013870700832784F70D
:108E4400B387E700130700022380E700A38007002D
:108E5400032584FCEFB09744130705009307200013
:108E64006312F702930784F81386070097050A0034
:108E7400938505C513050000EFD0D74B2324A4FC2C
:108E84006F00901D930784F81386070097050A0066
:108E9400938505C313050000EFD0D7492324A4FC10
:108EA4006F00D0251306200097050A009385C5D9C5
:108EB400032584FCEFB05747930705006394072C00
:108EC400032584FCEFB0973D1307050093072000AA
:108ED400631AF72A930784F81386070097050A0094
:108EE400938505BE13050000EFD0D7442324A4FCCA
:108EF400832784FC638007021306400097050A0059
:108F04009385C5D4032584FCEFB01742930705006D
:108F14006380071297870C009387070503A7070050
:108F240083A74700B7160000337CD70093FC0700E3
:108F340093070C00B3E797016384070AEFB0813706
:108F44009306300017060A001306C6B8930560138B
:108F540017050A001305455EEFB0512597870C00ED
:108F64009387070083A707006388070297570C00BD
:108F740083A7877583A7070083A7C7009386070085
:108F84001306E0009305100017050A00130505B544
:108F9400EF60D7316F00000297570C0083A7C772A8
:108FA40083A7070083A7C700938507001305000262
:108FB400EF50876097570C0083A7077183A70700BA
:108FC40083A7C70093860700130650029305100079
:108FD40017050A00130505C8EF60572DEFB0412FA0
:108FE400832704F79387C70413850700EFB0172B73
:108FF4002326A4FA832704F71387C7048327C4FA14
:10900400B306F700130700288327C4FAB307F74011
:1090140017060A00130606C4938507001385060085
:10902400EF90975B8327C4FB2326F4FC6F00D012D8
:10903400832704F783A787016380071297870C00AF
:10904400938787F203A7070083A74700B71600009A
:10905400337DD70093FD070093070D00B3E7B701F5
:109064006384070AEFB001259306300017060A004F
:10907400130646A69305E01317050A001305C54B0E
:10908400EFB0D11297870C00938787ED83A7070071
:109094006388070297570C0083A7076383A7070019
:1090A40083A7C700938607001306E000930510000A
:1090B40017050A00130585A2EF60571F6F00000211
:1090C40097570C0083A7476083A7070083A7C700AF
:1090D4009385070013050002EF50074E97570C00C5
:1090E40083A7875E83A7070083A7C700938607002B
:1090F400130610039305100017050A00130505B89D
:10910400EF60D71AEFB0C11C832704F79387C70415
:1091140013850700EFB097182328A4FA832704F7D0
:109124001387C704832704FBB306F700130700283B
:10913400832704FBB307F74017060A00130606B497
:109144009385070013850600EF9017498327C4FB16
:109154002326F4FC6F0050008327440013071000FB
:1091640023A0E700930784F81386070097050A00F5
:109174009385059513050000EFD0D71B2324A4FC89
:109184006F00C0771306D00097050A00938545B297
:10919400032584FCEFB05719930705006394071661
:1091A400832704F783A787016388071297870C0036
:1091B400938787DB03A7070083A74700B716000040
:1091C400B376D700232CD4F493F70700232EF4F4BA
:1091D400832684F50327C4F593870600B3E7E700E5
:1091E4006384070AEFB0010D9306300017060A00E6
:1091F4001306468E9305D01417050A001305C533CC
:10920400EFB0C17A97870C00938787D583A70700AF
:109214006388070297570C0083A7074B83A70700AF
:1092240083A7C700938607001306E0009305100088
:1092340017050A001305858AEF6057076F000002BF
:1092440097570C0083A7474883A7070083A7C70045
:109254009385070013050002EF50073697570C005B
:1092640083A7874683A7070083A7C70093860700C1
:10927400130690039305100017050A00130545A46F
:10928400EF60D702EFB0C104832704F79387C704C4
:1092940013850700EFB09700232CA4F8832704F765
:1092A4001387C704832784F9B306F700130700283C
:1092B400832784F9B307F74017060A00130646A06C
:1092C4009385070013850600EF9017318327C4FBAD
:1092D4002326F4FC6F004068832744001307100022
:1092E40023A0E700930784F81386070097F5090085
:1092F4009385057D13050000EFD0D7032324A4FC38
:109304006F00C05F1306F00097050A009385059F60
:10931400032584FCEFB057019307050063920716F9
:10932400832784F66398071297870C009387C7C333
:1093340003A7070083A74700B7160000B376D7003A
:109344002328D4F493F70700232AF4F4832604F59E
:10935400032744F593870600B3E7E7006384070A0D
:10936400EFA051759306300017F6090013068676B0
:109374009305B01517050A001305051CEFB001632A
:1093840097870C009387C7BD83A7070063880702EC
:1093940097570C0083A7473383A7070083A7C70009
:1093A400938607001306E0009305100017F50900E3
:1093B4001305C572EF60876F6F00000297570C00AA
:1093C40083A7873083A7070083A7C7009385070077
:1093D40013050002EF50471E97570C0083A7C72EB2
:1093E40083A7070083A7C7009386070013062003FB
:1093F4009305100017050A0013054591EF60076BEC
:10940400EFA0116D832704F79387C7041385070022
:10941400EFB0C768232EA4F8832704F71387C70483
:109424008327C4F9B306F700130700288327C4F978
:10943400B307F74017060A001306468D9385070005
:1094440013850600EF9057198327C4FB2326F4FCE9
:109454006F008050832744F61307100023A0E70011
:10946400930784F81386070097F5090093854565EB
:1094740013050000EFD0076C2324A4FC6F00004800
:109484001306400197050A009385858B032584FC08
:10949400EFB0876993070500639C0728832784F648
:1094A4006398071297870C00938707AC03A70700FC
:1094B40083A74700B7160000B376D7002324D4F45B
:1094C40093F707002326F4F4832684F40327C4F4D3
:1094D40093870600B3E7E7006384070AEFA0915D72
:1094E4009306300017F609001306C65E930580162E
:1094F40017050A0013054504EFB0414B97870C008C
:10950400938707A683A707006388070297570C0071
:1095140083A7871B83A7070083A7C7009386070039
:109524001306E0009305100017F509001305055B09
:10953400EF60C7576F00000297570C0083A7C71846
:1095440083A7070083A7C7009385070013050002BC
:10955400EF50870697570C0083A7071783A70700C8
:1095640083A7C700938607001306700393051000B2
:1095740017F509001305457EEF604753EFA05155D9
:10958400832704F79387C70413850700EFB00751B7
:109594002320A4FA832704F71387C704832704FA34
:1095A400B306F70013070028832704FAB307F7402C
:1095B40017F609001306467A9385070013850600FB
:1095C400EF9097018327C4FB2326F4FC6F00C03877
:1095D400832744F683A707006398071297870C0034
:1095E4009387879803A7070083A74700B71600004F
:1095F400B376D7002320D4F493F707002322F4F49E
:10960400832604F4032744F493870600B3E7E700B2
:109614006384070AEFA0114A9306300017F6090085
:109624001306464B9305F01617050A001305C5F0FB
:10963400EFB0C13797870C009387879283A7070001
:109644006388070297570C0083A7070883A70700BE
:1096540083A7C700938607001306E0009305100054
:1096640017F5090013058547EF6047446F000002B2
:1096740097570C0083A7470583A7070083A7C70054
:109684009385070013050002EF40177397570C00EA
:1096940083A7870383A7070083A7C70093860700D0
:1096A400130600059305100017F509001305456E10
:1096B400EF60C73FEFA0D141832704F79387C70426
:1096C40013850700EFB0873D2322A4FA832704F70C
:1096D4001387C704832744FAB306F7001307002847
:1096E400832744FAB307F74017F609001306466ABE
:1096F4009385070013850600EF90076E8327C4FB4C
:109704002326F4FC6F004025930710002322F4FC69
:10971400930784F81386070097F509009385453A63
:1097240013050000EFD007412324A4FC6F00001DA3
:1097340097870C009387478303A7070083A74700F5
:10974400B7160000B376D700232CD4F293F70700A2
:10975400232EF4F2832684F30327C4F393870600AD
:10976400B3E7E7006382070AEFA0D1349306300021
:1097740017F60900130606369305B01717050A00F5
:10978400130585DBEFB0812297770C009387477D23
:1097940083A707006388070297570C0083A7C7F2C3
:1097A40083A7070083A7C700938607001306E0007A
:1097B4009305100017F5090013054532EF60072FD4
:1097C4006F00000297570C0083A707F083A70700D8
:1097D40083A7C7009385070013050002EF40D75DF8
:1097E40097570C0083A747EE83A7070083A7C700FA
:1097F400032684FC97F509009385053C138507002F
:10980400EF405751EFA0D12C832704F79387C70467
:1098140013850700EFB087282324A4FA832704F7CD
:109824001387C704832784FA3305F7001307002836
:10983400832784FAB307F740832684FC17F60900CC
:109844001306863793850700EF9007598327C4FBD7
:109854002326F4FC6F004010032584FCEFB007249A
:109864009307050093871700232CF4FA032704FCBD
:10987400832784FBB307F7000327840063E2E7022E
:1098840097F609009386063B17060A001306C6CA14
:109894009305F01717F509001305851EEF30176EB1
:1098A400032704FC832784FBB307F7002320F4FC7D
:1098B400832584FC032584F7EF905716032584F74A
:1098C400EFB0C71D9307050013870700832784F7AC
:1098D400B387E700130700022380E700A380070093
:1098E400930784F81386070097F509009385451DAF
:1098F40013050000EFD007242324A4FC832784FC51
:10990400638407006FE0DFFF232604FC032584F74C
:10991400EFB0C7182320A4FC832704FC638C070240
:10992400832704FC9387F7FF032784F7B307F70023
:1099340003C7070093070002631EF700832704FC94
:109944009387F7FF032784F7B307F7002380070003
:109954006F00800013000000032544FBEF60C77B09
:10996400232A04FA8327C4FC138507008320C10C2F
:109974000324810C0329410C8329010C032AC10B04
:10998400832A810B032B410B832B010B032CC10A6C
:10999400832C810A032D410A832D010A1301010D31
:1099A40067800000130101FD232611022324810294
:1099B40013040103232EA4FC8327C4FD83A7870378
:1099C400638A071E232604FE6F00401C8327C4FD00
:1099D40003A7C7038327C4FE93976700B307F70061
:1099E4002322F4FE832744FE83A7C70213850700BE
:1099F400EF608772832744FE23A60702832744FE71
:109A040003A6070383A6470393070600B3E7D7001B
:109A140063960716832744FE83A70701138507006F
:109A2400EF60876F832744FE23A80700832744FE43
:109A340083A7C70013850700EF60076E832744FEE2
:109A440023A60700232404FE6F000008832744FE96
:109A540003A74701832784FE93975700B307F700B2
:109A640083A7470013850700EF60076B832744FE35
:109A740003A74701832784FE93975700B307F70092
:109A840023A20700832744FE03A74701832784FEFC
:109A940093975700B307F70083A7070013850700C0
:109AA400EF608767832744FE03A74701832784FE6B
:109AB40093975700B307F70023A00700832784FE7A
:109AC400938717002324F4FE832744FE83A707000B
:109AD400032784FEE36CF7F6832744FE83A747013C
:109AE40013850700EF604763832744FE23AA07001A
:109AF400232404FE6F004004832744FE03A7870346
:109B0400832784FE93972700B307F70083A70700F2
:109B1400638E0700832744FE03A78703832784FEFD
:109B240093972700B307F70023A00700832784FE39
:109B3400938717002324F4FE8327C4FD83A7C7005B
:109B4400032784FEE36AF7FA832744FE83A7870387
:109B540013850700EF60475C832744FE23AC0702AC
:109B6400832744FE83A7870013850700EF60C75A45
:109B7400832744FE23A407006F0080001300000025
:109B84008327C4FE938717002326F4FE8327C4FD8E
:109B940083A787030327C4FEE36AF7E28327C4FD90
:109BA40083A7C70313850700EF6007578327C4FD06
:109BB40023AE0702130000008320C10203248102A4
:109BC4001301010367800000130101FD2326110224
:109BD4002324810213040103232EA4FC8327C4FD40
:109BE40003A7072D9307F0FF6318F7008327C4FD2D
:109BF40083A78703638807188327C4FD83A7070403
:109C04006382070297F609009386C61D17060A00A9
:109C1400130686939305C01B17F50900130545E643
:109C2400EF30D7350325C4FDEFF0DFD78327C4FD1C
:109C340023AC07028327C4FD1307F0FF23A8E72CF6
:109C4400232604FE6F0080128327C4FD03A7870424
:109C54008327C4FE93972700B307F70083A7070061
:109C640013850700EF60474B8327C4FD03A78704D0
:109C74008327C4FE93972700B307F70023A00700A8
:109C84008327C4FD83A647040327C4FE9307070064
:109C940093972700B387E70093973700B387E700CC
:109CA400B387F6001306900293050000138507009E
:109CB400EF7007138327C4FD83A787016382070A14
:109CC4008327C4FD03A747028327C4FE9397270075
:109CD400B307F70083A7070013850700EF60C743A6
:109CE4008327C4FD03A747028327C4FE9397270055
:109CF400B307F70023A007008327C4FD03A70702C7
:109D04008327C4FE93972700B307F70023A0070017
:109D14008327C4FD03A747038327C4FE9397270023
:109D2400B307F70083A7070013850700EF60C73E5A
:109D34008327C4FD03A747038327C4FE9397270003
:109D4400B307F70023A007008327C4FD03A7070375
:109D54008327C4FE93972700B307F70023A00700C7
:109D64008327C4FE938717002326F4FE8327C4FDAC
:109D740083A7C7000327C4FEE368F7EC8327C4FD69
:109D840023860704130000008320C10203248102F8
:109D940013010103678000001301018B2326117452
:109DA400232481742322917423202175232E31735B
:109DB400232C4173232A517323286173232671733F
:109DC40023248173232291732320A173232EB17141
:109DD40013040175232EA494232CB494232AC4942D
:109DE4002328D4942326E4942324F494232204954E
:109DF40023201495232804962326049623240496CA
:109E040023220496232C04FA232C04F8232A04FA8C
:109E1400232804FA232204FA9305000017F5090005
:109E2400130505FEEFA0413E232AA4F88327849559
:109E340063860700930750FF6F008000930710FFAD
:109E44002328F4F8832744956394070E97770C002E
:109E54009387871103A7070083A74700B71600005D
:109E64003379D70093F9070093070900B3E7370163
:109E7400638A070AEFA001449306300017F609002D
:109E8400130646C59305A01F17F509001305856D34
:109E9400EFA0D13197770C009387870C83A7070035
:109EA4006388070297570C0083A7078283A70700DC
:109EB40083A7C700938607001306000293051000CA
:109EC40017F50900130545F5EF50573E6F00C00222
:109ED40097470C0083A7477F83A7070083A7C70082
:109EE40093860700130630019305100017F5090047
:109EF4001305C5F4EF50973B97470C0083A7C77C25
:109F040083A7070083A7C70017F60900130646F4C2
:109F140097F50900938505F513850700EF40875FE2
:109F2400EFA0013B930740FD232EF4FA6F10D019E4
:109F3400832704956388070E8327C4946394070ECC
:109F440097770C009387470203A7070083A747006E
:109F5400B7160000337AD70093FA070093070A0074
:109F6400B3E75701638A070AEFA0C13493063000B0
:109F740017F60900130606B69305C01F17F5090066
:109F84001305455EEFA0912297770C00938747FD58
:109F940083A707006388070297470C0083A7C7724B
:109FA40083A7070083A7C700938607001306E00171
:109FB4009305100017F50900130505EBEF50172F53
:109FC4006F00C00297470C0083A7077083A70700A0
:109FD40083A7C7009386070013061001930510009A
:109FE40017F50900130545EAEF50572C97470C0065
:109FF40083A7876D83A7070083A7C70017F6090007
:10A004001306C6E997F509009385C5E5138507008E
:10A01400EF404750EFA0C12B930720FE232EF4FA04
:10A024006F10900A832704956398070E8327C494BE
:10A034006384070E97770C00938707F303A7070041
:10A0440083A74700B7160000337BD70093FB0700B4
:10A0540093070B00B3E77701638A070AEFA0812512
:10A064009306300017F609001306C6A69305E01FF1
:10A0740017F509001305054FEFA0511397770C004E
:10A08400938707EE83A707006388070297470C00AE
:10A0940083A7876383A7070083A7C7009386070066
:10A0A4001306E0019305100017F509001305C5DB3D
:10A0B400EF50D71F6F00C00297470C0083A7C760FB
:10A0C40083A7070083A7C700938607001306100120
:10A0D4009305100017F50900130505DBEF50171D54
:10A0E40097470C0083A7475E83A7070083A7C70091
:10A0F40017F60900130646DD97F50900938585D602
:10A1040013850700EF400741EFA0811C930720FE51
:10A11400232EF4FA6F10407B8327C4006398070E44
:10A12400832704016384070E97770C009387C7E3A2
:10A1340003A7070083A74700B7160000337CD700A6
:10A1440093FC070093070C00B3E79701638A070A9F
:10A15400EFA041169306300017F609001306869700
:10A164009305102017F509001305C53FEFA011044E
:10A1740097770C009387C7DE83A7070063880702DD
:10A1840097470C0083A7475483A7070083A7C700FA
:10A19400938607001306E0019305100017F50900E4
:10A1A400130585CCEF5097106F00C00297470C0041
:10A1B40083A7875183A7070083A7C7009386070057
:10A1C400130610019305100017F509001305C5CBFC
:10A1D400EF50D70D97470C0083A7074F83A70700BD
:10A1E40083A7C70017F609001306C6D097F5090020
:10A1F400938545C713850700EF40C731EFA0410D94
:10A20400930720FE232EF4FA6F10006C83274495E5
:10A2140083A707046384070E97770C009387C7D43A
:10A2240003A7070083A74700B7160000337DD700B4
:10A2340093FD070093070D00B3E7B701638A070A8C
:10A24400EFA041079306300017F60900130686882D
:10A254009305402017F509001305C530EFA00175DB
:10A2640097770C009387C7CF83A7070063880702FB
:10A2740097470C0083A7474583A7070083A7C70018
:10A2840093860700130620029305100017F50900B2
:10A29400130505C9EF5097016F00C00297470C00E2
:10A2A40083A7874283A7070083A7C7009386070075
:10A2B400130650019305100017F50900130585C80E
:10A2C400EF50C77E97470C0083A7074083A707007A
:10A2D40083A7C700938607001306C00193051000E7
:10A2E40017F50900130585C7EF50477CEF90517EA1
:10A2F400930750FC232EF4FA6F10005D83274495D6
:10A3040083A78701639807108327449583A747028F
:10A31400639207108327449583A7C702639C070EA3
:10A3240097770C00938747C403A7070083A74700C8
:10A33400B7160000B376D700232CD49293F7070006
:10A34400232EF492832684930327C49393870600D1
:10A35400B3E7E700638A070AEF90D17593063000EC
:10A3640017E60900130606779305702017F5090010
:10A374001305451FEFA0816397770C00938747BEB1
:10A3840083A707006388070297470C0083A7C73396
:10A3940083A7070083A7C70093860700130600025C
:10A3A4009305100017F50900130505A7EF50077072
:10A3B4006F00C00297470C0083A7073183A70700EB
:10A3C40083A7C70093860700130630019305100086
:10A3D40017F50900130585A6EF50476D97470C0044
:10A3E40083A7872E83A7070083A7C7009386070048
:10A3F4001306A0089305100017F50900130505B806
:10A40400EF50C76AEF90D16C930740FD232EF4FA06
:10A414006F10804B8327449583A7870163900710AF
:10A4240083278495639C070E97770C009387C7B3A3
:10A4340003A7070083A74700B7160000B376D70029
:10A444002328D49293F70700232AF49283260493B3
:10A454000327449393870600B3E7E700638A070A58
:10A46400EF9051659306300017E6090013068666DF
:10A474009305002117F509001305C50EEFA001533C
:10A4840097770C009387C7AD83A7070063880702FB
:10A4940097470C0083A7472383A7070083A7C70018
:10A4A40093860700130620029305100017F5090090
:10A4B400130505A7EF50875F6F00C00297470C0094
:10A4C40083A7872083A7070083A7C7009386070075
:10A4D400130650019305100017F50900130585A60E
:10A4E400EF50C75C97470C0083A7071E83A707009C
:10A4F40083A7C70093860700130630039305100053
:10A5040017F50900130545B0EF50475AEF90515C19
:10A51400930750FC232EF4FA6F10003B83274495D5
:10A5240083A747006342F00297F60900938606B1B9
:10A5340017F60900130606039305502117E50900D1
:10A5440013050554EF308723832744952386070496
:10A554008327449583A7C70113850700EF50D73B92
:10A564008327449523AE0700832744F96380070AB1
:10A5740083278494638A070003258494EFA00752F9
:10A58400930705006F008000930700002326F4F86A
:10A59400032544F9EFA08750130705008327C4F867
:10A5A400B307F700938727002326F4F80325C4F89C
:10A5B400EF50D735930705002322F4FA832744FA92
:10A5C4002380070083278494638A07028325849465
:10A5D400032544FAEF801779032544FAEFA0074CCA
:10A5E4009307050013870700832744FA3387E7009E
:10A5F400930700022300F700A3000700832544F912
:10A60400032544FAEF8097416F00C00083278494A8
:10A614002322F4FA832744FA63860708032544FABD
:10A62400EFA0C7472326A4FA8327C4FA93870720F9
:10A634002324F4F8032584F8EF50572D93070500DD
:10A64400138707008327449523AEE70083274495A7
:10A6540083A5C701930644961307049713064497EA
:10A66400832784F82324F100930784962322F1009E
:10A674009307C4962320F10093880600130807006B
:10A68400832784950327C49583264495032544FA98
:10A69400EFE0CF8D232EA4FA8327C4FB6384070045
:10A6A4006F10C01C97770C009387078C03A70700D3
:10A6B40083A74700937647002324D49293F7070097
:10A6C4002326F492832684920327C4929387060058
:10A6D400B3E7E7006386070AEF90D13D93061000C5
:10A6E40017F60900130686979305A02317F50900AA
:10A6F400130545E7EFA0812B97770C0093874786D6
:10A7040083A707006388070297470C0083A7C7FB4A
:10A7140083A7070083A7C700938607001306E000FA
:10A724009305100017E509001305453BEF50073862
:10A734006F00000297470C0083A707F983A707005F
:10A7440083A7C7009385070013050002EF30D7667F
:10A7540097470C0083A747F783A7070003A7C70001
:10A764008327449583A7C7011386070097F509003B
:10A774009385458F13050700EF30D759EF90513576
:10A78400032744968327449523A8E7008327449608
:10A794006382070E97670C009387077D03A7070062
:10A7A40083A74700B716000093860680B376D700C8
:10A7B4002320D49293F707002322F4928326049251
:10A7C4000327449293870600B3E7E7006384070AEC
:10A7D400EF90512E9306200017F609001306C68A3F
:10A7E4009305202417F509001305C5D7EFA0011C14
:10A7F40097670C009387C77683A7070063880702CF
:10A8040097470C0083A747EC83A7070083A7C700DB
:10A81400938607001306E0009305100017E509006E
:10A824001305C52BEF5087286F00000297470C00D3
:10A8340083A787E983A7070083A7C7009385070039
:10A8440013050002EF30575797470C0083A7C7E75B
:10A8540083A7070083A7C700938607001306200574
:10A864009305100017F5090013058582EF5007249E
:10A87400EF9011268327049563900702832744955C
:10A8840083A7C7002328F4948327449583A747010B
:10A894002326F4946F000003232004969307049660
:10A8A40013860700832504950325C494EF70414162
:10A8B400232CA4FA832704962328F494832784FB67
:10A8C4002326F49403254495EFF00FB0232A04FAC9
:10A8D4006F00D0248327449503A74701832744FBB3
:10A8E40093972700B307F70083A707002320F4F802
:10A8F400232004FA232604FA6F0040038327C4FAB2
:10A90400939727000327C494B307F70083A707008E
:10A91400032704F86316F700930710002320F4FAC2
:10A924008327C4FA938717002326F4FA0327C4FA6B
:10A9340083270495E364F7FC832704FAE380071C68
:10A944008327C49663860724832704F803A7070D87
:10A9540083A7470D93760708232CD49093F7070019
:10A96400232EF490832684910327C49193870600B1
:10A97400B3E7E700639E072097670C009387C75EE1
:10A9840003A7070083A74700B7160000B376D700D4
:10A994002328D49093F70700232AF4908326049164
:10A9A4000327449193870600B3E7E7006384070A0B
:10A9B400EF9051109306300017E609001306861134
:10A9C4009305802617F509001305C5B9EF90117E8C
:10A9D40097670C009387C75883A70700638807020B
:10A9E40097470C0083A747CE83A7070083A7C70018
:10A9F400938607001306E0009305100017E509008D
:10AA04001305C50DEF50870A6F00000297470C002D
:10AA140083A787CB83A7070083A7C7009385070075
:10AA240013050002EF30573997470C0083A7C7C9B5
:10AA340083A7070083A7C7009386070013060008AF
:10AA44009305100017E509001305C569EF500706C3
:10AA5400EF901108832744959387C7041385070053
:10AA6400EFA0C703232EA4F6832744951387C704B6
:10AA74008327C4F7B306F700130700288327C4F716
:10AA8400B307F74017E609001306C6659385070068
:10AA940013850600EF80473497670C009387C74CF3
:10AAA40003A7070083A74700B7160000B376D700B3
:10AAB4002324D49093F707002326F49083268490CC
:10AAC4000327C49093870600B3E7E700638C070A63
:10AAD400EF90417E9306300017E60900130686FFC7
:10AAE4009305902617F509001305C5A7EF90116C7F
:10AAF40097670C009387C74683A7070063880702FC
:10AB040097470C0083A747BC83A7070083A7C70008
:10AB1400938607001306E0019305100017E509006A
:10AB240013058564EF4097786F00C00297470C00C7
:10AB340083A787B983A7070083A7C7009386070065
:10AB4400130610019305100017E509001305C563EA
:10AB5400EF40D77597470C0083A707B783A7070073
:10AB640003A7C700832704F883A7C7161386070023
:10AB740097E509009385856213050700EF3097195F
:10AB8400EF900175832704F9232EF4FA6F00D04463
:10AB9400832704FB938717002328F4FA832744951B
:10ABA40083A7C702639007768327449583A7870109
:10ABB400638A072097670C009387073B03A7070066
:10ABC40083A74700B7160000B376D7002320D4909C
:10ABD40093F707002322F4908326049003274490DC
:10ABE40093870600B3E7E7006384070AEF90816C5C
:10ABF4009306300017E609001306C6ED9305602896
:10AC040017F5090013050596EF90515A97670C0044
:10AC14009387073583A707006388070297470C00CB
:10AC240083A787AA83A7070083A7C7009386070083
:10AC34001306E0009305100017E50900130505EA63
:10AC4400EF40D7666F00000297470C0083A7C7A7A1
:10AC540083A7070083A7C700938507001305000295
:10AC6400EF30971597470C0083A707A683A7070023
:10AC740083A7C70093860700130690059305100069
:10AC840017E509001305055AEF405762EF90416438
:10AC9400832744959387C70413850700EF901760B3
:10ACA400232AA4F6832744951387C704832744F7EC
:10ACB400B306F70013070028832744F7B307F740C8
:10ACC40017E6090013060656938507001385060048
:10ACD400EF80871097670C009387072903A7070065
:10ACE40083A74700B7160000B376D700232CD48E71
:10ACF40093F70700232EF48E8326848F0327C48FB3
:10AD040093870600B3E7E7006388070AEF90815A48
:10AD14009306300017E609001306C6DB9305902856
:10AD240017F5090013050584EF90514897670C0047
:10AD34009387072383A707006388070297470C00BC
:10AD440083A7879883A7070083A7C7009386070074
:10AD5400130670029305100017E509001305455208
:10AD6400EF40D7546F00C00297470C0083A7C795E4
:10AD740083A7070083A7C700938607001306A001D3
:10AD84009305100017E5090013050552EF4017520B
:10AD940097470C0083A7479383A7070003A7C7001F
:10ADA400832744959387C7049305070013850700F9
:10ADB400EF30D711EF90C1519307D0FF232EF4FA4F
:10ADC4006F0090218327449503A74702832744FB00
:10ADD40093972700B307F70083A707006388072228
:10ADE4008327449503A74703832744FB93972700AE
:10ADF400B307F70083A70700639A072097670C003F
:10AE04009387871603A7070083A74700B716000098
:10AE1400B376D7002328D48E93F70700232AF48E21
:10AE24008326048F0327448F93870600B3E7E70044
:10AE34006384070AEF9001489306300017E609007F
:10AE4400130646C99305A02B17E509001305857160
:10AE5400EF90D13597670C009387871083A707007D
:10AE64006388070297470C0083A7078683A7070018
:10AE740083A7C700938607001306E000930510001C
:10AE840017E50900130585C5EF4057426F0000021E
:10AE940097470C0083A7478383A7070083A7C700AE
:10AEA4009385070013050002EF30077197470C00E4
:10AEB40083A7878183A7070083A7C700938607001A
:10AEC400130600069305100017E509001305853FD6
:10AED400EF40D73DEF90C13F832744959387C70444
:10AEE40013850700EF90973B232CA4F68327449502
:10AEF4001387C704832784F7B306F70013070028D2
:10AF0400832784F7B307F74017E609001306863B47
:10AF14009385070013850600EF70176C97670C0084
:10AF24009387870403A7070083A74700B716000089
:10AF3400B376D7002324D48E93F707002326F48E08
:10AF44008326848E0327C48E93870600B3E7E70025
:10AF54006388070AEF9001369306300017E609006C
:10AF6400130646B79305D02B17E509001305855F33
:10AF7400EF90D12397670C00938787FE83A7070080
:10AF84006388070297370C0083A7077483A7070019
:10AF940083A7C70093860700130670029305100069
:10AFA40017E509001305C52DEF4057306F00C002A7
:10AFB40097370C0083A7477183A7070083A7C700AF
:10AFC400938607001306A0019305100017E50900F6
:10AFD4001305852DEF40972D97370C0083A7C76E77
:10AFE40083A7070003A7C700832744959387C70453
:10AFF4009305070013850700EF30476DEF90412D4F
:10B004009307D0FF232EF4FA6F00007D8327449525
:10B0140003A74703832744FB93972700B307F7004D
:10B0240083A70700638E070C97670C009387C7F309
:10B0340003A7070083A74700937617002320D48E25
:10B0440093F707002322F48E8326048E0327448E6D
:10B0540093870600B3E7E700638A072AEF90812508
:10B064009306100017E609001306062C9305302CEE
:10B0740017E509001305054FEF90511397670C006E
:10B08400938707EE83A707006388070297370C00AE
:10B0940083A7876383A7070083A7C7009386070056
:10B0A4001306E0009305100017E50900130505A336
:10B0B400EF40D71F6F00000297370C0083A7C760CB
:10B0C40083A7070083A7C700938507001305000221
:10B0D400EF30874E97370C0083A7075F83A70700DD
:10B0E40083A7C700032644FB97E5090093854524FD
:10B0F40013850700EF300742EF90811D6F00002198
:10B10400832784956380071083274400638C070E8C
:10B1140097670C00938747E503A7070083A74700B9
:10B12400B7160000B376D700232CD48C93F707000E
:10B13400232EF48C8326848D0327C48D93870600E5
:10B14400B3E7E700638A070AEF90C116930630005D
:10B1540017E60900130606989305F02E17E5090073
:10B1640013054540EF90910497670C00938747DFE0
:10B1740083A707006388070297370C0083A7C75487
:10B1840083A7070083A7C70093860700130650020E
:10B194009305100017E509001305C51BEF401711AF
:10B1A4006F00C00297370C0083A7075283A70700DC
:10B1B40083A7C70093860700130680019305100038
:10B1C40017E509001305851BEF40570E97370C0050
:10B1D40083A7874F83A7070083A7C7009386070029
:10B1E4001306D0049305100017E509001305C51ACA
:10B1F400EF40D70BEF90C10D9307F0FE232EF4FA26
:10B204006F00805D97670C00938707D603A707003C
:10B2140083A74700B7160000B376D7002328D48C41
:10B2240093F70700232AF48C8326048D0327448D87
:10B2340093870600B3E7E700638C070AEF90810762
:10B244009306300017E609001306C6889305702F8D
:10B2540017E5090013050531EF90417597670C0058
:10B26400938707D083A707006388070297370C00EA
:10B2740083A7874583A7070083A7C7009386070092
:10B284001306F0019305100017E509001305C51511
:10B29400EF40D7016F00C00297370C0083A7C74265
:10B2A40083A7070083A7C70093860700130620011E
:10B2B4009305100017E5090013050515EF40077FF6
:10B2C40097370C0083A7474083A7070003A7C7004D
:10B2D400832704F883A7C7161386070097E5090098
:10B2E4009385C51313050700EF30C722EF80517E05
:10B2F400930760FD232EF4FA6F00004E1300000044
:10B304006F000001130000006F00800013000000B4
:10B31400832744FB93871700232AF4FA8327449551
:10B3240083A7C700032744FB6366F7DA032704FBFC
:10B3340083270495637CF70E97670C009387C7C235
:10B3440003A7070083A74700B7160000B376D7000A
:10B354002324D48C93F707002326F48C8326848C2F
:10B364000327C48C93870600B3E7E700638A070AC0
:10B37400EF8051749306300017D6090013068675C2
:10B384009305603117E509001305C51DEF900162AF
:10B3940097670C009387C7BC83A7070063880702DD
:10B3A40097370C0083A7473283A7070083A7C700FA
:10B3B400938607001306E0019305100017E50900C2
:10B3C400130585DAEF40876E6F00C00297370C00D3
:10B3D40083A7872F83A7070083A7C7009386070047
:10B3E400130610019305100017E509001305C5D9CC
:10B3F400EF40C76B97370C0083A7072D83A707007F
:10B4040083A7C70093860700130640069305100020
:10B4140017E509001305C504EF404769EF80516B38
:10B42400832704F9232EF4FA6F00003B8327449505
:10B4340023A8072C832744951307400023AAE72C4D
:10B444008327049763880700832744951307200004
:10B4540023AAE72C8327C495638C0700832784954C
:10B4640063980700832744951307100023AAE72C49
:10B474008327449583A787036382070297E609001D
:10B484009386860417E609001306C60D93058032D9
:10B4940017D509001305C55EEF20472E8327449571
:10B4A40003A7472D930740006306F700232E04FAF1
:10B4B4006F00003E232A04FA6F0000168327449588
:10B4C40083A7C702638A070C8327449503A78702CF
:10B4D4008327449523ACE7028327449583A78703F6
:10B4E400638607148327449503A74701832744FBF6
:10B4F40093972700B307F70083A707002322F4F8E4
:10B504008327449583A787039305000413850700C5
:10B51400EF20873793070500138707008327449597
:10B5240023AEE702232E04F86F00C005832744F8F6
:10B5340083A7472503A8C70C832744F883A6871944
:10B544008327449503A7C7028327C4F99397270049
:10B55400B307F70083A507008327449503A7C70310
:10B564008327C4F993976700B307F700138607008E
:10B5740013850600E70008008327C4F993871700A2
:10B58400232EF4F88327449583A787030327C4F95C
:10B59400E36EF7F86F0080098327449503A74703F8
:10B5A400832744FB93972700B307F70083A707007B
:10B5B400638E0704832544FB03254495EFA0C11241
:10B5C400130705008327449523ACE702832744959A
:10B5D40083A78703638007068327449583A787038C
:10B5E4009305000413850700EF20072A930705003D
:10B5F400138707008327449523AEE702832544FB82
:10B6040003254495EFA0910F6F00C002832744FBEC
:10B6140093871700232AF4FA8327449583A7C70046
:10B62400032744FBE36CF7E86F00000113000000FC
:10B634006F008000130000008327449583A7C70090
:10B64400032744FB636CF70E97670C009387C7913D
:10B6540003A7070083A74700B7160000B376D700F7
:10B664002320D48C93F707002322F48C8326048CA4
:10B674000327448C93870600B3E7E700638A070A2D
:10B68400EF8051439306300017D609001306864411
:10B694009305303617E509001305C5ECEF90013129
:10B6A40097670C009387C78B83A7070063880702FB
:10B6B40097370C0083A7470183A7070083A7C70018
:10B6C400938607001306F0019305100017E509009F
:10B6D400130585D1EF40873D6F00C00297370C00FA
:10B6E40083A787FE83A7070083A7C7009386070065
:10B6F400130620019305100017E509001305C5D0B2
:10B70400EF40C73A97370C0083A707FC83A70700CD
:10B7140083A7C70093860700130630039305100020
:10B7240017E50900130505DCEF404738EF80513A6F
:10B73400930760FD232EF4FA6F00000A232404FA11
:10B744006F0000088327449583A6C7008327449588
:10B7540003A7C703832784FA93976700B304F7000A
:10B764009305000113850600EF20071293070500D7
:10B7740023A6F4028327449583A7C702639C070288
:10B78400232A04FA6F000002032644FB832584FA6B
:10B7940003254495EF101222832744FB9387170057
:10B7A400232AF4FA8327449583A7C700032744FB7D
:10B7B400E36CF7FC832784FA938717002324F4FAB5
:10B7C4008327449583A78703032784FAE36CF7F65A
:10B7D400232E04FA6F00C00B03254495EFE08F9CE1
:10B7E4008327449523A00704232A04FA6F00C00684
:10B7F4008327449583A78701638A07048327449595
:10B8040003A74702832744FB93972700B307F70056
:10B8140083A7070013850700EF401710832744957B
:10B8240003A74702832744FB93972700B307F70036
:10B8340023A007008327449503A70702832744FB1B
:10B8440093972700B307F70023A00700832744FB3F
:10B8540093871700232AF4FA8327449583A7C70004
:10B86400032744FBE366F7F86F0080001300000031
:10B87400032744FA832784946306F700032544FAD4
:10B88400EF409709832744951307E0FF23A8E72C8B
:10B894008327449583A7470063D2070297E60900EC
:10B8A400938686C717E609001306C6CB9305B038FE
:10B8B40017D509001305C51CEF10576C032584FB2D
:10B8C400EF409705232C04FA8327C400638A0700FA
:10B8D4008327C4008325040103254495E7800700DA
:10B8E4008327C4FB138507008320C1740324817458
:10B8F40083244174032901748329C173032A817346
:10B90400832A4173032B0173832BC172032C81722D
:10B91400832C4172032D0172832DC17113010175B2
:10B9240067800000130101FB2326110423248104F2
:10B934002322210523203105232E4103232C5103E7
:10B94400232A6103232871032326810323249103DB
:10B9540013040105232EA4FA232CB4FA232AC4FACF
:10B96400232604FC232404FC832684FB6394060E10
:10B9740097570C009387475F03A7070083A74700E7
:10B98400B7160000337CD70093FC070093070C0024
:10B99400B3E79701638A070AEF80D1119306300059
:10B9A40017E609001306C6BD9305000317E5090051
:10B9B400130585F0EF80917F97570C009387475AC2
:10B9C40083A707006388070297370C0083A7C7CFB4
:10B9D40083A7070083A7C700938607001306E00127
:10B9E4009305100017E50900130505BAEF40070C8D
:10B9F4006F00C00297370C0083A707CD83A7070009
:10BA040083A7C7009386070013061001930510004F
:10BA140017E50900130545B9EF40470997370C00AE
:10BA240083A787CA83A7070083A7C70017E609006F
:10BA34001306C6B897E509009385C5B913850700B1
:10BA4400EF20572DEF80D108930720FE2324F4FC28
:10BA54006F0090108326C4FB6394060E97570C0066
:10BA64009387875003A7070083A74700B7160000F2
:10BA7400337FD70093FF070093070F00B3E7F70165
:10BA8400638A070AEF8011039306300017E6090062
:10BA9400130606AF9305200317E509001305C5E156
:10BAA400EF80D17097570C009387874B83A70700CB
:10BAB4006388070297370C0083A707C183A7070091
:10BAC40083A7C7009386070013060002930510009E
:10BAD40017E50900130545B0EF30577D6F00C0022C
:10BAE40097370C0083A747BE83A7070083A7C70027
:10BAF40093860700130630019305100017E509002B
:10BB04001305C5AFEF30977A97370C0083A7C7BBEF
:10BB140083A7070083A7C70017E60900130646AFEB
:10BB240097E50900938505AB13850700EF20971E61
:10BB3400EF80017A930740FD2324F4FC6F00D001C9
:10BB44008326C4FB83A6C6006394060E97570C0095
:10BB54009387874103A7070083A74700B716000010
:10BB6400337ED70093FE070093070E00B3E7D70197
:10BB7400638A070AEF8001749306300017E6090010
:10BB8400130606A09305400317E509001305C5D263
:10BB9400EF80D16197570C009387873C83A70700F8
:10BBA4006388070297370C0083A707B283A70700AF
:10BBB40083A7C700938607001306000293051000AD
:10BBC40017E50900130545A1EF30576E6F00C00259
:10BBD40097370C0083A747AF83A7070083A7C70045
:10BBE40093860700130630019305100017E509003A
:10BBF4001305C5A0EF30976B97370C0083A7C7AC2C
:10BC040083A7070083A7C700938607001306A00233
:10BC14009305100017E509001305C5A0EF30176957
:10BC2400EF80016B930740FD2324F4FC6F00C07286
:10BC34008326C4FB03A6062D9306F0FF6314D60ED9
:10BC440097570C009387473203A7070083A7470041
:10BC5400B71600003373D70093F30700930703006C
:10BC6400B3E77700638A070AEF80C1649306300064
:10BC740017E609001306C6909305700317E509003B
:10BC8400130585C3EF80915297570C009387472D76
:10BC940083A707006388070297370C0083A7C7A20E
:10BCA40083A7070083A7C700938607001306B00283
:10BCB4009305100017E5090013058599EF30175F08
:10BCC4006F00C00297370C0083A707A083A7070063
:10BCD40083A7C700938607001306E00193051000AD
:10BCE40017E5090013058599EF30575C97370C0069
:10BCF40083A7879D83A7070083A7C70093860700B0
:10BD04001306E0049305100017E5090013050599CF
:10BD1400EF30D759EF80C15B930730FD2324F4FC47
:10BD24006F0080638326C4FB83A6062D6384060EFE
:10BD340097570C009387472303A7070083A747005F
:10BD4400B71600003378D70093F80700930708006C
:10BD5400B3E71701638A070AEF80C15593063000E1
:10BD640017E609001306C6819305B00317E5090019
:10BD7400130585B4EF80914397570C009387471EB2
:10BD840083A707006388070297370C0083A7C7932C
:10BD940083A7070083A7C700938607001306B00292
:10BDA4009305100017E509001305858AEF30175035
:10BDB4006F00C00297370C0083A7079183A7070081
:10BDC40083A7C700938607001306E00193051000BC
:10BDD40017E509001305858AEF30574D97370C0096
:10BDE40083A7878E83A7070083A7C70093860700CE
:10BDF400130670029305100017E509001305058F5B
:10BE0400EF30D74AEF80C14C930730FD2324F4FC74
:10BE14006F0080548326C4FB83A6C602639A060E71
:10BE24008326C4FB83A6C62C6394060E97560C0087
:10BE34009386861303A6060083A64600B715000062
:10BE44003377B60093F7060093060700B3E6F600CF
:10BE5400638A060AEF8001469306300017D609006C
:10BE6400130606729305E00317E509001305C5A43C
:10BE7400EF80D13397570C009387870E83A7070071
:10BE84006388070297370C0083A7078483A70700FA
:10BE940083A7C700938607001306B002930510001A
:10BEA40017D509001305C57AEF3057406F00C0025B
:10BEB40097370C0083A7478183A7070083A7C70090
:10BEC400938607001306E0019305100017D50900B7
:10BED4001305C57AEF30973D97270C0083A7C77EDB
:10BEE40083A7070083A7C700938607001306D0041F
:10BEF4009305100017E509001305C581EF30173BC2
:10BF0400EF80013D930730FD2324F4FC6F00C0440F
:10BF14009305000213051000EF101717930705008F
:10BF24002326F4FC8327C4FC6394070E97570C0064
:10BF34009387870303A7070083A74700B71600006A
:10BF4400337BD70093FB070093070B00B3E777011C
:10BF5400638A070AEF8001369306300017D609007A
:10BF6400130606629305500417E509001305C594EA
:10BF7400EF80D12397570C00938787FE83A7070090
:10BF84006388070297270C0083A7077483A7070019
:10BF940083A7C70093860700130630029305100099
:10BFA40017D509001305057CEF3057306F00C00228
:10BFB40097270C0083A7477183A7070083A7C700AF
:10BFC40093860700130660019305100017D5090036
:10BFD4001305857BEF30972D97270C0083A7C76E39
:10BFE40083A7070083A7C700938607001306700280
:10BFF4009305100017D509001305857AEF30172B28
:10C00400EF80012D9307A0FF2324F4FC6F00C034BC
:10C014008327C4FC1307100023A2E700232204FC97
:10C024006F00C0038327C4FB03A7C703832744FC13
:10C0340093976700B307F70083A7C700832584FBA2
:10C0440013850700EF70073A930705006382070220
:10C05400832744FC938717002322F4FC8327C4FB23
:10C0640083A78703032744FCE36EF7FA6F0080007D
:10C07400130000008327C4FB83A78703032744FC22
:10C084006362F70E97570C00938707EE03A7070028
:10C0940083A74700B7160000337AD70093FA070046
:10C0A40093070A00B3E757016388070AEF808120EA
:10C0B4009306300017D609001306864C9305E00456
:10C0C40017D509001305457FEF80510E97570C00D3
:10C0D400938707E983A707006388070297270C0063
:10C0E40083A7875E83A7070083A7C70093860700FB
:10C0F400130640029305100017D509001305C56CFB
:10C10400EF30D71A6F00C00297270C0083A7C75BD4
:10C1140083A7070083A7C70093860700130670014F
:10C124009305100017D509001305856CEF30171817
:10C1340097270C0083A7475983A7070083A7C70045
:10C14400032684FB97D509009385056C13850700A6
:10C15400EF20473CEF80C117930720FD2324F4FC14
:10C164006F00801F8327C4FB03A7C703832744FCF6
:10C17400939767003307F7008327C4FC23A8E700DD
:10C184008327C4FC83A7070103A7C7008327C4FC34
:10C1940023AAE7008327C4FB03A787008327C4FCE3
:10C1A40023A4E7008327C4FC0327C4FB23A6E700DA
:10C1B4008327C4FC83A7070183A707009305800195
:10C1C40013850700EF10476C9307050013870700DA
:10C1D4008327C4FC23ACE7008327C4FC83A787011F
:10C1E4006394070E97570C00938707D803A707009B
:10C1F40083A74700B71600003379D70093F90700E7
:10C2040093070900B3E73701638A070AEF80810ABD
:10C214009306300017D60900130686369305900559
:10C2240017D5090013054569EF80417897570C002D
:10C23400938707D383A707006388070297270C0017
:10C2440083A7874883A7070083A7C70093860700AF
:10C25400130630029305100017D509001305855005
:10C26400EF30D7046F00C00297270C0083A7C7459F
:10C2740083A7070083A7C7009386070013066001FE
:10C284009305100017D5090013050550EF30170268
:10C2940097270C0083A7474383A7070083A7C700FA
:10C2A40017D609001306865997D509009385853258
:10C2B40013850700EF200726EF8081019307A0FF75
:10C2C4002324F4FC6F0040098327C4FB83A74700A1
:10C2D4006342F00297D609009386465817D60900A0
:10C2E4001306865D9305C00517D509001305055986
:10C2F400EF10C7488327C4FB03A707048327C4FCA4
:10C3040023AEE7008327C4FB0327C4FC23A0E70470
:10C314008327C4FB83A74700138717008327C4FB25
:10C3240023A2E7008327C4FB83A7470063D2070245
:10C3340097D609009386465617D609001306C657A2
:10C344009305F00517D5090013054553EF1007436E
:10C35400232404FC6F0040038327C4FC638E07007E
:10C364008327C4FC83A7870113850700EF30D75ABE
:10C374008327C4FC23AC07000325C4FCEF30D75942
:10C38400232604FC232604FC832744FB638807003C
:10C39400832744FB032784FC23A0E7008327C4FCF2
:10C3A400138507008320C104032481040329410465
:10C3B40083290104032AC103832A8103032B410334
:10C3C400832B0103032CC102832C81021301010579
:10C3D40067800000130101FD23261102232481023A
:10C3E400232221032320310313040103232EA4FC5D
:10C3F4008325C4FD6392050E97570C009387C7B637
:10C4040003A7070083A74700B71500003376B700DA
:10C4140093F6070093070600B3E7D700638A070A79
:10C42400EF7051699306300017D609001306064AC7
:10C434009305100217D509001305455DEF800157D8
:10C4440097570C009387C7B183A707006388070237
:10C4540097270C0083A7472783A7070083A7C70054
:10C46400938607001306F0019305100017D5090001
:10C4740013054546EF3087636F00C00297270C0011
:10C4840083A7872483A7070083A7C7009386070091
:10C49400130620019305100017D5090013058545DF
:10C4A400EF30C76097270C0083A7072283A70700F4
:10C4B40083A7C70017D609001306064597D50900B8
:10C4C4009385C54513850700EF20C704EF705160BD
:10C4D400930700FD6F00003B8326C4FD83A646003E
:10C4E4006342D00297D609009386864317D6090083
:10C4F4001306C6519305200217D5090013050544F8
:10C50400EF10C7278326C4FD83A646009386F6FF53
:10C514000326C4FD2322D6002322D4FE8326C4FD91
:10C5240083A6460063D2060297D609009386C642C4
:10C5340017D609001306864D9305200217D5090066
:10C544001305C53FEF10872397560C009386C6A1A9
:10C5540003A6060083A646001377060493F7060095
:10C5640093060700B3E6F6006384060AEF7091545D
:10C574009306100017D609001306064093053002EF
:10C5840017D5090013058548EF80414297570C00E1
:10C594009387079D83A707006388070297270C00EA
:10C5A40083A7871283A7070083A7C7009386070082
:10C5B4001306E0009305100017D509001305853C08
:10C5C400EF30C74E6F00000297270C0083A7C70FF8
:10C5D40083A7070083A7C7009385070013050002FC
:10C5E400EF10977D97270C0083A7070E83A70700FA
:10C5F40083A7C700832644FE0326C4FD97D50900FC
:10C604009385453913850700EF10D770EF70514CAF
:10C61400832744FE6396072697570C009387C79495
:10C6240003A7070083A747001379070493F90700BA
:10C6340093070900B3E737016382070AEF70914754
:10C644009306100017D609001306063393057002EB
:10C6540017D509001305853BEF80413597570C002A
:10C664009387079083A707006388070297270C0026
:10C6740083A7870583A7070083A7C70093860700BE
:10C684001306E0009305100017D509001305852F44
:10C69400EF30C7416F00000297270C0083A7C70241
:10C6A40083A7070083A7C70093850700130500022B
:10C6B400EF10977097270C0083A7070183A7070043
:10C6C40083A7C7000326C4FD97D509009385052ECB
:10C6D40013850700EF101764EF70913F8327C4FDA3
:10C6E40083A7C7002320F4FE832704FE6392070276
:10C6F40097D609009386862C17D6090013060631AF
:10C704009305900217D5090013054523EF10070779
:10C71400832704FE83A747006342F00297D60900EB
:10C724009386C62A17D609001306462E9305C0021F
:10C7340017D5090013058520EF104704832704FE4D
:10C7440083A707040327C4FD631EF700832704FEA1
:10C7540083A7070403A7C701832704FE23A0E704D4
:10C764006F008005832704FE83A707042324F4FEB7
:10C774006F000001832784FE83A7C7012324F4FEEE
:10C78400832784FE83A7C701638A0700832784FE67
:10C7940083A7C7010327C4FDE31EF7FC832784FE98
:10C7A40083A7C701638A07008327C4FD03A7C701C2
:10C7B400832784FE23AEE7008327C4FD83A7870174
:10C7C400638C0704232604FE6F00C0038327C4FD83
:10C7D40083A687010327C4FE9307070093971700D6
:10C7E400B387E70093973700B387F60083A7070161
:10C7F40013850700EF20C16A8327C4FE93871700BF
:10C804002326F4FE8327C4FD83A7070183A707001B
:10C814000327C4FEE36CF7FA8327C4FD23AA0700A9
:10C824008327C4FD23A807008327C4FD83A78701AA
:10C8340013850700EF30570E8327C4FD23AC070090
:10C844000325C4FDEF30570D232E04FC832704FE7B
:10C8540083A7470063D2070297D609009386061977
:10C8640017D609001306861A9305A00317D50900E5
:10C874001305C50CEF009770032504FEEFB0CFEA53
:10C8840093070000138507008320C102032481025B
:10C894000329410283290102130101036780000077
:10C8A400130101F7232611082324810823222109D7
:10C8B40023203109232E4107232C5107232A610702
:10C8C4002328710723268107232491072322A10704
:10C8D4002320B10713040109232EA4F8232CB4F850
:10C8E400232AC4F82328D4F88326C4F96392060EB5
:10C8F40097470C009387476703A7070083A7470060
:10C90400B7160000337ED70093FE070093070E008E
:10C91400B3E7D701638A070AEF70D1199306300091
:10C9240017D609001306C60F9305C00217D50900D0
:10C934001305C54BEF80810797470C009387476227
:10C9440083A707006388070297270C0083A7C7D72C
:10C9540083A7070083A7C700938607001306F00187
:10C964009305100017D509001305050CEF300714C3
:10C974006F00C00297270C0083A707D583A7070081
:10C9840083A7C700938607001306200193051000B0
:10C9940017D509001305450BEF30471197270C00F5
:10C9A40083A787D283A7070083A7C70017D60900E8
:10C9B4001306C60A97D509009385850B13850700CE
:10C9C400EF105735EF70D110930700FD6F009037CB
:10C9D4008326C4F983A6060183A60600032684F9E8
:10C9E4006368D60E97470C009387075803A7070080
:10C9F40083A74700B71600003373D70093F30700EB
:10CA040093070300B3E777006380070CEF70910A84
:10CA14009306300017D60900130686009305E0023A
:10CA240017D509001305853CEF70517897470C0022
:10CA34009387075383A707006388070297270C008F
:10CA440083A787C883A7070083A7C7009386070027
:10CA5400130620029305100017D50900130585015C
:10CA6400EF30C7046F00C00297270C0083A7C7C527
:10CA740083A7070083A7C700938607001306500106
:10CA84009305100017D5090013050501EF300702BF
:10CA940097270C0083A747C383A7070003A7C700F2
:10CAA4008327C4F983A7070183A70700832684F992
:10CAB4001386070097D50900938585FF13050700A2
:10CAC400EF105725EF70D1009307F0FC6F0090270B
:10CAD4008326C4F983A686016392060E97470C0049
:10CAE4009387874803A7070083A74700B71600006A
:10CAF4003378D70093F8070093070800B3E71701CA
:10CB0400638A070AEF70017B9306300017D6090089
:10CB1400130606F19305300317D509001305052DF7
:10CB2400EF70D16897470C009387874383A707006A
:10CB34006388070297270C0083A707B983A7070018
:10CB440083A7C700938607001306F001930510001E
:10CB540017D50900130545EDEF2057756F00C00286
:10CB640097270C0083A747B683A7070083A7C700AE
:10CB740093860700130620019305100017D50900BA
:10CB8400130585ECEF20977297270C0083A7C7B392
:10CB940083A7070083A7C700938607001306F00244
:10CBA4009305100017D50900130545F3EF201770FE
:10CBB400EF700172930700FD6F00D0188326C4F94B
:10CBC40083A6060103A64601832684F9939656009C
:10CBD400B306D600232CD4FA832684FB03A686004E
:10CBE400B7F6FFFF938646E6B306D60093B6160063
:10CBF40093F6F60F232AD4FA97460C009386C6368A
:10CC040003A5060083A5460093060500B3E6B60017
:10CC140063860614232204FC832684FB03A6860170
:10CC240093061000630AD600832684FB03A68601BC
:10CC340093062000631CD600832604F9638806004B
:10CC4400832604F983A606002322D4FC232004FCB3
:10CC5400832604F9638E0600032644F993064000F4
:10CC64006318D600832604F983A606002320D4FC87
:10CC740097460C009386462F03A6060083A646001B
:10CC84001377160093F7060093060700B3E6F60041
:10CC94006386060CEF7001629306100017D6090034
:10CCA4001306C6E69305500417D5090013050514A9
:10CCB400EF70D14F97470C009387872A83A707000B
:10CCC4006388070297270C0083A707A083A70700A0
:10CCD40083A7C700938607001306E000930510009E
:10CCE40017D50900130505E3EF20575C6F00000218
:10CCF40097270C0083A7479D83A7070083A7C70036
:10CD04009385070013050002EF10170B97270C00FB
:10CD140083A7879B83A7070003A5C7008327C4F9BC
:10CD240003A64701832784FB03A70700832704FC8A
:10CD34002322F100832744FC2320F100832804F9F3
:10CD4400032844F9832744FB832684F997D50900F3
:10CD5400938545DDEF10077CEF708157832704F935
:10CD6400638C070E832744FB6388070E97470C00E8
:10CD74009387871F03A7070083A74700B716000000
:10CD8400B376D7002324D4F893F707002326F4F8C6
:10CD9400832684F80327C4F893870600B3E7E700E3
:10CDA4006388070AEF7001519306300017D6090013
:10CDB400130606C79305C00417D509001305050318
:10CDC400EF70D13E97470C009387871983A707001C
:10CDD4006388070297270C0083A7078F83A70700A0
:10CDE40083A7C7009386070013062002930510004B
:10CDF40017D50900130545DAEF20574B6F00C00221
:10CE040097270C0083A7478C83A7070083A7C70035
:10CE140093860700130650019305100017D50900E7
:10CE24001305C5D9EF20974897270C0083A7C78916
:10CE340083A7070083A7C700032684F997D50900B1
:10CE4400938545D913850700EF10C76CEF704148EF
:10CE54009307E0FC6F00006F832704F9639C070EBF
:10CE6400832744FB6398070E832784FB03A787016A
:10CE7400930710006300F70E97470C009387C70EC3
:10CE840003A7070083A74700B7160000337DD70028
:10CE940093FD070093070D00B3E7B7016388070A02
:10CEA400EF7041419306300017D60900130646B7C8
:10CEB4009305200517D50900130545F3EF70112FCD
:10CEC40097470C009387C70983A707006388070265
:10CED40097170C0083A7477F83A7070083A7C70082
:10CEE40093860700130620029305100017D5090046
:10CEF400130585CAEF20973B6F00C00297170C00FB
:10CF040083A7877C83A7070083A7C70093860700AE
:10CF1400130650019305100017D50900130505CA1F
:10CF2400EF20D73897170C0083A7077A83A7070049
:10CF340083A7C700032684F997D50900938505CDF7
:10CF440013850700EF10075DEF7081389307E0FC4D
:10CF54006F00405F832744F96394070E832744FBE3
:10CF64006380070E97470C009387070003A7070009
:10CF740083A74700B7160000337CD70093FC070053
:10CF840093070C00B3E797016388070AEF708132B7
:10CF94009306300017D60900130686A89305B0053A
:10CFA40017D50900130585E4EF70512097470C004D
:10CFB400938707FB83A707006388070297170C0072
:10CFC40083A7877083A7070083A7C70093860700FA
:10CFD400130610029305100017D509001305C5C6E2
:10CFE400EF20D72C6F00C00297170C0083A7C76DE2
:10CFF40083A7070083A7C700938607001306400191
:10D004009305100017D50900130545C6EF20172A0C
:10D0140097170C0083A7476B83A7070083A7C70054
:10D02400032684F997D509009385C5C513850700A0
:10D03400EF10474EEF70C1299307D0FC6F0080506A
:10D04400832784FB03A78701930730006316F70E39
:10D05400832704F96392070E97470C009387C7F060
:10D0640003A7070083A74700B7160000337BD70048
:10D0740093FB070093070B00B3E77701638A070A62
:10D08400EF7041239306300017D609001306469922
:10D094009305F00517D50900130545D5EF70111157
:10D0A40097470C009387C7EB83A7070063880702A1
:10D0B40097170C0083A7476183A7070083A7C700BE
:10D0C40093860700130600029305100017D5090084
:10D0D400130585BEEF20971D6F00C00297170C0043
:10D0E40083A7875E83A7070083A7C70093860700EB
:10D0F400130630019305100017D50900130505BE6A
:10D10400EF20D71A97170C0083A7075C83A70700A3
:10D1140083A7C700938607001306A0029305100097
:10D1240017D509001305C5BCEF205718EF70411A35
:10D13400930770FD6F000041832784FB03A78701D9
:10D14400930710006302F702832784FB03A7870178
:10D1540093072000630AF700832784FB03A7870152
:10D1640093073000631AF70E832744FB6392072268
:10D17400032744F993074000630CF72097470C00FA
:10D18400938787DE03A7070083A74700B71600002D
:10D19400337AD70093FA070093070A00B3E75701DD
:10D1A4006388070AEF7001119306300017D609004F
:10D1B400130606879305500617D50900130505C302
:10D1C400EF70C17E97470C00938787D983A7070028
:10D1D4006388070297170C0083A7074F83A70700EC
:10D1E40083A7C70093860700130610029305100057
:10D1F40017D50900130545A5EF20570B6F00C00292
:10D2040097170C0083A7474C83A7070083A7C70081
:10D2140093860700130640019305100017D50900F3
:10D224001305C5A4EF20970897170C0083A7C749D7
:10D2340083A7070083A7C700032684F997D50900AD
:10D244009385C5AD13850700EF10C72CEF70410817
:10D254009307D0FC6F00002F832784FB83A7C701AB
:10D26400638A0712832744F9232EF4FA0327C4FBA5
:10D2740093073000B377F702639C07000327C4FBCE
:10D2840093073000B357F70293972700232EF4FA3D
:10D29400832784FB83A7C7010327C4FB630CF70E12
:10D2A40097470C00938747CC03A7070083A7470041
:10D2B400B71600003379D70093F9070093070900E4
:10D2C400B3E737016382070CEF60D17E9306300029
:10D2D40017C609001306C6749305000717D509007D
:10D2E4001305C5B0EF70816C97470C00938747C74F
:10D2F40083A707006388070297170C0083A7C73C1E
:10D3040083A7070083A7C7009386070013061002AC
:10D314009305100017D5090013050593EF2007792D
:10D324006F00C00297170C0083A7073A83A7070072
:10D3340083A7C700938607001306400193051000D6
:10D3440017D5090013058592EF20477697170C002F
:10D3540083A7873783A7070003A5C700832784FB18
:10D3640083A60700832784FB03A70700832784FB86
:10D3740083A7C701032684F997D509009385459EA1
:10D38400EF104719EF60D1749307D0FC6F00801B36
:10D39400130000008327C4F983A68701032784F9B7
:10D3A4009307070093971700B387E7009397370015
:10D3B400B387F6002328F4FA8327C4F983A7470028
:10D3C4006342F00297D609009386C69C17D60900DB
:10D3D4001306C6A19305700717D509001305459DCB
:10D3E400EF00C739832704FB23AA0700832704F926
:10D3F4006380070E832784FB03A78701930710002C
:10D404006318F700832704F983A707006382070CD6
:10D41400832704FB83A7070113850700EF10512816
:10D42400832704FB23A80700032544F9EF10817622
:10D434002326A4FC0327C4FC9307F00763F6E70044
:10D44400930700082326F4FC832744F92324F4FCDF
:10D45400032784FC8327C4FC6376F7008327C4FC7A
:10D464002324F4FC832584FC0325C4FCEF10111A47
:10D474002326A4FA8327C4FA639C07028327C4F9EA
:10D4840083A7470063D2070297D6090093860694C0
:10D4940017D60900130686959305E00817D50900E9
:10D4A40013050591EF00872D9307A0FF6F008009F6
:10D4B400032644F9832504F90325C4FAEF30876E63
:10D4C400832704FB0327C4FA23A8E7006F00C001E5
:10D4D400832704FB83A7070113850700EF10511C62
:10D4E400832704FB23A80700832744F92320F4F8A7
:10D4F400232204F8832704FB832604F8032744F833
:10D5040023A0D70023A2E700832704FB13071000FE
:10D5140023AAE7008327C4F983A7470063D207023D
:10D5240097D609009386868A17D609001306068CB7
:10D534009305400A17D5090013058587EF000724D2
:10D5440093070000138507008320C1080324810882
:10D554000329410883290108032AC107832A810773
:10D56400032B4107832B0107032CC106832C81065F
:10D57400032D4106832D0106130101096780000074
:10D58400130101FD2326810213040103232EA4FCAD
:10D59400232CB4FC6F0040028327C4FD2326F4FE31
:10D5A400032784FD8327C4FDB377F702232EF4FCFD
:10D5B4008327C4FE232CF4FC8327C4FDE39E07FCCD
:10D5C400832784FD138507000324C102130101038B
:10D5D40067800000130101FE232E1100232C81001B
:10D5E400130401022326A4FE2324B4FE0327C4FE4D
:10D5F400832784FE6376F7008327C4FE6F00C0048C
:10D60400832784FE6398070297C609009386467FA2
:10D6140017D60900130606129305500417C509000E
:10D624001305C57EEF008715832784FE9387F7FFD4
:10D634002324F4FE0327C4FE832784FEB377F70272
:10D64400E39407FE832784FE138507008320C1012A
:10D65400032481011301010267800000130101FE0C
:10D66400232E8100130401022326A4FE2324B4FEE6
:10D674002322C4FE032784FE8327C4FEB377F70264
:10D68400639E0700032744FE832784FEB377F702D3
:10D6940063960700930710006F0080009307000053
:10D6A400138507000324C1011301010267800000F0
:10D6B400130101E12326111E2324811E2322911E1E
:10D6C4002320211F232E311D232C411D232A511DCC
:10D6D4002328611D2326711D2324811D2322911DCE
:10D6E4002320A11D232EB11B1304011F2326A4F004
:10D6F4002324B4F02322C4F02320D4F0232EE4EE18
:10D70400232CF4EE232A04EF232814EF93070100BB
:10D714002322F4E2232A04FA832744FB2328F4FA7D
:10D72400832704FB2326F4FA232A04F6832744F7E9
:10D734002328F4F6832704F72326F4F6232404FA93
:10D74400832784FA232EF4FA8327C4FB232CF4FAC8
:10D75400232C04F8232404F6832784F083A70701E9
:10D7640083A7070013871700930707009387F7FF22
:10D774002322F4F6130F0700930F00009357BF0101
:10D7840093935F00B3E3770013135F00130907005B
:10D79400930900009357B901939E5900B3EED70142
:10D7A400131E5900931727009387F70093D7470058
:10D7B400939747003301F140930781009387370023
:10D7C40093D72700939727002320F4F6832784F028
:10D7D40083A7070103A70700832744EFB307F700D4
:10D7E40013871700930707009387F7FF232EF4F49A
:10D7F400130C0700930C00009357BC01939A5C0030
:10D80400B3EA5701131A5C00130D0700930D0000CF
:10D814009357BD01939B5D00B3EB7701131B5D0030
:10D82400931727009387F70093D7470093974700F0
:10D834003301F140930781009387370093D7270082
:10D8440093972700232CF4F48327C4F0639A070EDC
:10D8540097370C009387477103A7070083A74700F6
:10D86400B7160000B376D7002324D4EE93F707004D
:10D874002326F4EE832684EE0327C4EE9387060062
:10D88400B3E7E700638A070AEF60D122930630000A
:10D8940017C609001306C6599305400717D5090092
:10D8A400130585E7EF70811097370C009387476B5A
:10D8B40083A707006388070297170C0083A7C7E0B4
:10D8C40083A7070083A7C700938607001306600297
:10D8D4009305100017C5090013050556EF20071D11
:10D8E4006F00C00297170C0083A707DE83A7070009
:10D8F40083A7C700938607001306900193051000C1
:10D9040017C509001305C555EF20471A97170C00D2
:10D9140083A787DB83A7070083A7C70017C609006F
:10D924001306C65597C509009385C5561385070088
:10D93400EF00573EEF60D1199307C0FD6F204054AC
:10D94400832784F0639A070E97370C009387C76187
:10D9540003A7070083A74700B7160000B376D700D4
:10D964002320D4EE93F707002322F4EE832604EE5B
:10D97400032744EE93870600B3E7E700638A070AA8
:10D98400EF6051139306300017C609001306464A88
:10D994009305600717D50900130505D8EF70010139
:10D9A40097370C009387C75B83A707006388070238
:10D9B40097170C0083A747D183A7070083A7C70045
:10D9C400938607001306F0019305100017C509009C
:10D9D4001305854CEF20870D6F00C00297170C00CC
:10D9E40083A787CE83A7070083A7C7009386070072
:10D9F400130620019305100017C509001305C54B34
:10DA0400EF20C70A97170C0083A707CC83A707004A
:10DA140083A7C70017C609001306464B97C509001C
:10DA24009385454713850700EF00D72EEF60510A11
:10DA3400930700FD6F20C0448327C4F003A7870029
:10DA4400832784F083A78700630AF70E97370C00B7
:10DA54009387875103A7070083A74700B7160000E1
:10DA6400B376D700232CD4EC93F70700232EF4ECE1
:10DA7400832684ED0327C4ED93870600B3E7E7000C
:10DA8400638A070AEF6011039306300017C6090082
:10DA94001306063A9305800717D509001305C5C771
:10DAA400EF60D17097370C009387874B83A70700EB
:10DAB4006388070297170C0083A707C183A7070091
:10DAC40083A7C7009386070013060002930510007E
:10DAD40017C509001305C540EF10577D6F00C0023C
:10DAE40097170C0083A747BE83A7070083A7C70027
:10DAF40093860700130630019305100017C509002B
:10DB040013054540EF10977A97170C0083A7C7BBFE
:10DB140083A7070083A7C700938607001306700333
:10DB24009305100017C509001305053FEF1017787A
:10DB3400EF60017A9307E0FD6F208034032604EF41
:10DB4400832544EF0325C4F0EF401103232CA4F8EC
:10DB5400832784F963860700832784F96F20403282
:10DB6400832744F0639A070E97370C009387C73FC7
:10DB740003A7070083A74700B7160000B376D700B2
:10DB84002328D4EC93F70700232AF4EC832604ED2E
:10DB9400032744ED93870600B3E7E700638A070A87
:10DBA400EF6041719306300017C60900130646283A
:10DBB4009305100817D50900130505B6EF60115F2A
:10DBC40097370C009387C73983A707006388070238
:10DBD40097170C0083A747AF83A7070083A7C70045
:10DBE40093860700130670029305100017C50900F9
:10DBF40013050536EF10976B6F00C00297170C00E2
:10DC040083A787AC83A7070083A7C7009386070071
:10DC14001306A0019305100017C509001305C535A7
:10DC2400EF10D76897170C0083A707AA83A70700EC
:10DC340083A7C70017C609001306C63597C5090090
:10DC44009385452513850700EF00D70CEF604168E5
:10DC54009307B0FC6F20C0228327C4F083A7C700BA
:10DC640003A74702832744F0637AF70E97370C0023
:10DC74009387872F03A7070083A74700B7160000E1
:10DC8400B376D7002324D4EC93F707002326F4ECCF
:10DC9400832684EC0327C4EC93870600B3E7E700EC
:10DCA400638A070AEF6001619306300017C6090012
:10DCB400130606189305200817D509001305C5A5F2
:10DCC400EF60D14E97370C009387872983A707000D
:10DCD4006388070297170C0083A7079F83A7070091
:10DCE40083A7C700938607001306700293051000EC
:10DCF40017C509001305C525EF10575B6F00C00257
:10DD040097170C0083A7479C83A7070083A7C70026
:10DD1400938607001306A0019305100017C5090098
:10DD240013058525EF10975897170C0083A7C799FB
:10DD340083A7070083A7C700938607001306200361
:10DD44009305100017C509001305C525EF101756D4
:10DD5400EF6001589307B0FC6F2080128327C4F052
:10DD640083A7C70003A747029307300063F2E702C3
:10DD740097C609009386462617D609001306C69946
:10DD84009305700817C5090013054508EFF0161F21
:10DD94008327C4F083A7C70013850700EF30D16D34
:10DDA4002324A4F6832704F0638E0704832704F056
:10DDB40083A707002326F4FA032744F093071000EF
:10DDC40063FAE700832704F09387470083A70700DB
:10DDD4006F008000930700002328F4FA032744F01F
:10DDE4009307200063FAE700832704F093878700F2
:10DDF40083A707006F00800093070000232AF4FA2A
:10DE04006F000001232604FA232804FA232A04FAC3
:10DE14008327C4EF83A707002326F4F6032744F0DF
:10DE24009307100063FAE7008327C4EF9387470042
:10DE340083A707006F008000930710002328F4F6DF
:10DE4400032744F09307200063FAE7008327C4EF15
:10DE54009387870083A707006F0080009307100053
:10DE6400232AF4F68327C4F6638A0700832704F77A
:10DE740063860700832744F7639A070E97370C00DD
:10DE84009387870E03A7070083A74700B7160000F0
:10DE9400B376D7002320D4EC93F707002322F4ECC5
:10DEA400832604EC032744EC93870600B3E7E700DA
:10DEB400638A070AEF6001409306300017C6090021
:10DEC400130606F79305C00917D509001305C58481
:10DED400EF60D12D97370C009387870883A707003D
:10DEE4006388070297070C0083A7077E83A70700B0
:10DEF40083A7C700938607001306900293051000BA
:10DF040017C509001305C510EF10573A6F00C0027A
:10DF140097070C0083A7477B83A7070083A7C70045
:10DF2400938607001306C0019305100017C5090066
:10DF34001305C510EF10973797070C0083A7C77810
:10DF440083A7070083A7C70017C609001306061195
:10DF540097C50900938505F413850700EF00875BD7
:10DF6400EF600137930710FC6F1090718327C4F0A2
:10DF740083A7C70083A7C702232AF4F4032744F026
:10DF84009307100063FAE7008327C4F083A7C70050
:10DF940083A707036F008000930710002328F4F47D
:10DFA400032744F09307200063FAE7008327C4F0B3
:10DFB40083A7C70083A747036F008000930710005F
:10DFC4002326F4F48327C4F083A7C70083A7870319
:10DFD4002324F4F4832784EF63880776832784EF6C
:10DFE40083A70700232CF4FA032744F093071000B7
:10DFF40063FAE700832784EF9387470083A707002A
:10E004006F00800093071000232EF4FA032744F0D6
:10E014009307200063FAE700832784EF9387870040
:10E0240083A707006F008000930710002324F4FAED
:10E03400032784FB8327C4FB3307F702832784FA6F
:10E044003307F702832784F463FAE70E97370C004B
:10E05400938787F103A7070083A74700B71600003B
:10E06400B376D700232CD4EA93F70700232EF4EADF
:10E07400832684EB0327C4EB93870600B3E7E7000A
:10E08400638A070AEF6001239306300017C609006C
:10E09400130606DA9305C00A17C509001305C567F8
:10E0A400EF60D11097370C00938787EB83A70700A5
:10E0B4006388070297070C0083A7076183A70700FB
:10E0C40083A7C700938607001306800293051000F8
:10E0D40017C509001305C5FBEF10571D6F00C002DB
:10E0E40097070C0083A7475E83A7070083A7C70091
:10E0F400938607001306B0019305100017C50900A5
:10E104001305C5FBEF10971A97070C0083A7C75B8D
:10E1140083A7070083A7C700938607001306D003CD
:10E124009305100017C50900130505FBEF10171818
:10E13400EF60011A9307A0FC6F109054032784FB2F
:10E14400832744F563FAE70E97370C009387C7E1FA
:10E1540003A7070083A74700B7160000B376D700CC
:10E164002328D4EA93F70700232AF4EA832604EB4E
:10E17400032744EB93870600B3E7E700638A070AA3
:10E18400EF6041139306300017C60900130646CA10
:10E194009305000B17C5090013050558EF6011011D
:10E1A40097370C009387C7DB83A7070063880702B0
:10E1B40097070C0083A7475183A7070083A7C700CD
:10E1C40093860700130670029305100017C5090013
:10E1D400130585F4EF10970D6F00C00297070C002C
:10E1E40083A7874E83A7070083A7C70093860700EA
:10E1F4001306A0019305100017C50900130545F483
:10E20400EF10D70A97070C0083A7074C83A70700D2
:10E2140083A7C700938607001306300393051000F5
:10E2240017C50900130585F3EF105708EF60410A7D
:10E23400930790FC6F10D044032744F09307100019
:10E2440063F0E7100327C4FB832704F563FAE70EA2
:10E2540097370C00938747D103A7070083A747008C
:10E26400B7160000B376D7002324D4EA93F7070047
:10E274002326F4EA832684EA0327C4EA9387060064
:10E28400B3E7E700638A070AEF60C1029306300030
:10E2940017C609001306C6B99305500B17C5090024
:10E2A40013058547EF60817097370C00938747CB40
:10E2B40083A707006388070297070C0083A7C7405A
:10E2C40083A7070083A7C70093860700130670027D
:10E2D4009305100017C50900130505E4EF10077D29
:10E2E4006F00C00297070C0083A7073E83A70700AF
:10E2F40083A7C700938607001306A00193051000A7
:10E3040017C509001305C5E3EF10477A97070C00FA
:10E3140083A7873B83A7070083A7C70093860700CB
:10E32400130630039305100017C50900130545E6CD
:10E33400EF10C777EF50D179930790FC6F105034EA
:10E34400032744F09307200063F0E710032784FABF
:10E354008327C4F463FAE70E97370C009387C7C08A
:10E3640003A7070083A74700B7160000B376D700BA
:10E374002320D4EA93F707002322F4EA832604EA4D
:10E38400032744EA93870600B3E7E700638A070A92
:10E39400EF5051729306300017C60900130646A9C0
:10E3A4009305A00B17C5090013050537EF6001603D
:10E3B40097370C009387C7BA83A7070063880702BF
:10E3C40097070C0083A7473083A7070083A7C700DC
:10E3D40093860700130670029305100017C5090001
:10E3E400130585D3EF10876C6F00C00297070C00EC
:10E3F40083A7872D83A7070083A7C70093860700F9
:10E404001306A0019305100017C50900130545D391
:10E41400EF10C76997070C0083A7072B83A7070092
:10E4240083A7C700938607001306300393051000E3
:10E4340017C50900130505D9EF104767EF50516957
:10E44400930790FC6F10D0230327C4F6832784FB23
:10E45400B377F702638A070E97370C009387C7B028
:10E4640003A7070083A74700B7160000B376D700B9
:10E47400232CD4E893F70700232EF4E8832684E9B9
:10E484000327C4E993870600B3E7E700638A070A12
:10E49400EF5051629306300017C6090013064699DF
:10E4A4009305200C17C5090013050527EF600150DB
:10E4B40097370C009387C7AA83A7070063880702CE
:10E4C40097070C0083A7472083A7070083A7C700EB
:10E4D40093860700130680029305100017C50900F0
:10E4E400130505BBEF10875C6F00C00297070C0093
:10E4F40083A7871D83A7070083A7C7009386070008
:10E504001306B0019305100017C50900130505BBD8
:10E51400EF10C75997070C0083A7071B83A70700B1
:10E5240083A7C70017C60900130606CD97C50900BF
:10E534009385459613850700EFF0D67DEF5051592A
:10E544009307A0FC6F10D013032704F78327C4FBA1
:10E55400B377F702638A070E97370C009387C7A037
:10E5640003A7070083A74700B7160000B376D700B8
:10E574002328D4E893F70700232AF4E8832604E940
:10E58400032744E993870600B3E7E700638A070A91
:10E59400EF5051529306300017C6090013064689FE
:10E5A4009305400C17C5090013050517EF600140DA
:10E5B40097370C009387C79A83A7070063880702DD
:10E5C40097070C0083A7471083A7070083A7C700FA
:10E5D40093860700130680029305100017C50900EF
:10E5E400130505ABEF10874C6F00C00297070C00B2
:10E5F40083A7870D83A7070083A7C7009386070017
:10E604001306B0019305100017C50900130505ABE7
:10E61400EF10C74997070C0083A7070B83A70700D0
:10E6240083A7C70017C609001306C6BE97C509000D
:10E634009385458613850700EFF0D66DEF50514959
:10E644009307A0FC6F10D003032744F7832784FAB1
:10E65400B377F702638A070E97370C009387C79046
:10E6640003A7070083A74700B7160000B376D700B7
:10E674002324D4E893F707002326F4E8832684E8C8
:10E684000327C4E893870600B3E7E700638A070A11
:10E69400EF5051429306300017B60900130646792D
:10E6A4009305600C17C5090013050507EF600130D9
:10E6B40097370C009387C78A83A7070063880702EC
:10E6C40097070C0083A7470083A7070083A7C70009
:10E6D40093860700130680029305100017C50900EE
:10E6E4001305059BEF10873C6F00C00297070C00D1
:10E6F40083A787FD83A7070083A7C7009386070026
:10E704001306B0019305100017C509001305059BF6
:10E71400EF10C73997070C0083A707FB83A70700EF
:10E7240083A7C70017C60900130686B097B509006A
:10E734009385457613850700EFF0D65DEF50513988
:10E744009307A0FC6F10C073832784F083A707018D
:10E7540083A70702638C0714832784F083A7070128
:10E7640083A7470263840714832784F083A70701E0
:10E7740083A78702638C0712832784EF63800704CF
:10E78400832784F083A7070183A70702032784FB59
:10E794006316F702832784F083A7070183A7470240
:10E7A4000327C4FB631CF700832784F083A70701B6
:10E7B40083A78702032784FA6300F77697270C0060
:10E7C4009387877A03A7070083A74700B71600003B
:10E7D400B376D7002320D4E893F707002322F4E884
:10E7E400832604E8032744E893870600B3E7E70099
:10E7F400638A070AEF50112C9306300017B60900FC
:10E80400130606639305300D17C509001305C5F0FB
:10E81400EF60C11997270C009387877483A70700BB
:10E824006388070297070C0083A707EA83A70700FA
:10E8340083A7C70093860700130680029305100080
:10E8440017C509001305C584EF1047266F00C002E1
:10E8540097070C0083A747E783A7070083A7C70090
:10E86400938607001306B0019305100017C509002D
:10E874001305C584EF10872397070C0083A7C7E40B
:10E8840083A7070083A7C70017C609001306069CC1
:10E8940097B509009385056013850700EFF0964747
:10E8A400EF5011239307A0FC6F10805D832784EF42
:10E8B40063960766832784F683A7C703232AF4F89D
:10E8C400832744F96396070093071000232AF4F87A
:10E8D40097270C009387476903A7070083A747007E
:10E8E40093761700232CD4E693F70700232EF4E63F
:10E8F400832684E70327C4E793870600B3E7E7008A
:10E904006382070AEF50111B9306100017C6090013
:10E914001306C69D9305E00E17C509001305C5DF50
:10E92400EF60C10897270C009387876383A70700CC
:10E934006388070297070C0083A707D983A70700FA
:10E9440083A7C700938607001306E0009305100011
:10E9540017C509001305059AEF1047156F0000024B
:10E9640097070C0083A747D683A7070083A7C70090
:10E974009385070013050002EFF0164497070C0077
:10E9840083A787D483A7070083A7C700032644F976
:10E9940097C509009385059713850700EFF096370F
:10E9A400EF5011138325C4F6032544F9EFE05FBD4E
:10E9B4002322A4F4832504F7032544F9EFE05FBC84
:10E9C4002320A4F4832544F7032544F9EFE05FBB37
:10E9D400232EA4F20327C4F6832744F4B356F70284
:10E9E400032744F5832744F4B357F70293850700BC
:10E9F40013850600EFE01FBE232CA4FA032784FB33
:10EA0400832744F4B307F702232CF4FA032744F0D2
:10EA14009307100063F0E704032704F7832704F443
:10EA2400B356F702032704F5832704F4B357F70218
:10EA34009385070013850600EFE0DFB9232EA4FABF
:10EA44000327C4FB832704F4B307F702232EF4FA45
:10EA54006F00C00093071000232EF4FA032744F03C
:10EA64009307200063F0E704032744F78327C4F3E4
:10EA7400B356F7020327C4F48327C4F3B357F7024A
:10EA84009385070013850600EFE0DFB42324A4FA7E
:10EA9400032784FA8327C4F3B307F7022324F4FA81
:10EAA4006F00C019930710002324F4FA6F000019B3
:10EAB400832784FA93F71700639A0702832784FA5B
:10EAC40093D71700032644F7938507000325C4F35F
:10EAD400EFE0DFB893070500638A0700832784FA11
:10EAE40093D717002324F4FA6F0040158327C4FB3F
:10EAF40093F71700639A07028327C4FB93D7170081
:10EB0400032604F793850700032504F4EFE01FB5FB
:10EB140093070500638A07008327C4FB93D7170074
:10EB2400232EF4FA6F008011832784FB93F71700D8
:10EB3400639A0702832784FB93D717000326C4F63E
:10EB440093850700032544F4EFE05FB193070500C4
:10EB5400638A0700832784FB93D71700232CF4FAD6
:10EB64006F00C00D032784FA9307100063F4E702D3
:10EB74000327C4F3832744F463EEE7000327C4F3B5
:10EB8400832704F463E8E700930710002324F4FACE
:10EB94006F00C00A0327C4FB9307100063F4E70265
:10EBA400032704F48327C4F363EEE700032704F484
:10EBB400832744F463E8E70093071000232EF4FA54
:10EBC4006F00C007032784FB9307100063F4E70278
:10EBD400032744F4832704F463EEE700032744F493
:10EBE4008327C4F363E8E70093071000232CF4FAA7
:10EBF4006F00C004032784FA9307100063F8E7004A
:10EC0400930710002324F4FA6F0000030327C4FBC6
:10EC14009307100063F8E70093071000232EF4FA1B
:10EC24006F008001032784FB9307100063F8E7005B
:10EC340093071000232CF4FA13000000032784FB2D
:10EC44008327C4FB3307F702832784FAB307F70249
:10EC5400032784F4E36EF7E4832744F993972700AA
:10EC6400232CF4F28327C4F083A7C70083A74701AA
:10EC7400232AF4F20327C4F6832784FBB357F7024D
:10EC84002328F4F8032704F78327C4FBB357F702B8
:10EC94002326F4F8032744F7832784FAB357F702AB
:10ECA4002324F4F86F000022032784FA832744F80E
:10ECB400B377F70263980704032784FA832744F899
:10ECC400B357F702032644F7938507000325C4F3DB
:10ECD400EFE0DF989307050063860702032784FAB1
:10ECE400832744F8B357F7022324F4FA032784F85C
:10ECF400832744F8B307F7022324F4F8232204F803
:10ED04006F00800C0327C4FB832744F8B377F70212
:10ED1400639807040327C4FB832744F8B357F70217
:10ED2400032604F793850700032504F4EFE01F93FB
:10ED340093070500638607020327C4FB832744F86F
:10ED4400B357F702232EF4FA0327C4F8832744F8B1
:10ED5400B307F7022326F4F8232204F86F00C00651
:10ED6400032784FB832744F8B377F70263980704E7
:10ED7400032784FB832744F8B357F7020326C4F61A
:10ED840093850700032544F4EFE05F8D93070500A6
:10ED940063860702032784FB832744F8B357F702EB
:10EDA400232CF4FA032704F9832744F8B307F70262
:10EDB4002328F4F8232204F86F000001832744F881
:10EDC4009387F7FF2322F4F8032744F893071000EE
:10EDD400E3ECE7EC832744F8639407006F00800EAC
:10EDE400032784FA9307100063F2E704032784FAE5
:10EDF400832784FB63ECE702032784FA8327C4FB9D
:10EE040063E6E702032784FB8327C4FBB307F70207
:10EE1400032784F363ECE700930710002324F4FA38
:10EE2400832744F72324F4F86F00C0090327C4FBA5
:10EE34009307100063F2E7040327C4FB832784FAD3
:10EE440063ECE7020327C4FB832784FB63E6E70242
:10EE5400032784FA832784FBB307F702032784F389
:10EE640063ECE70093071000232EF4FA832704F7DA
:10EE74002326F4F86F000005032784FB9307100092
:10EE840063FEE708032784FB8327C4FB63E8E708E2
:10EE9400032784FB832784FA63E2E7080327C4FB80
:10EEA400832784FAB307F702032784F363E8E706AA
:10EEB40093071000232CF4FA8327C4F62328F4F8CC
:10EEC40013000000032704F98327C4F83307F7026B
:10EED400832784F8B307F702032744F3B357F702F1
:10EEE4002322F4F8032744F89307100063F8E70299
:10EEF400032784FB8327C4FB3307F702832784FAA1
:10EF04003307F702832644F8832784F3B387F60292
:10EF1400E3ECE7EA6F0080001300000097270C0081
:10EF24009387870403A7070083A7470093761700F6
:10EF34002328D4E693F70700232AF4E6832604E77C
:10EF4400032744E793870600B3E7E7006380070ECF
:10EF5400EF5041369306100017B609001306063920
:10EF64009305101C17B509001305057BEF501124F8
:10EF740097270C009387C7FE83A7070063880702BF
:10EF840097F70B0083A7477483A7070083A7C700DD
:10EF9400938607001306E0009305100017B50900D7
:10EFA40013054535EF0097306F00000297F70B000B
:10EFB40083A7877183A7070083A7C70093850700EA
:10EFC40013050002EFF0465F97F70B0083A7C76FA6
:10EFD40083A7070003A5C700832784F003A647017E
:10EFE4000327C4F6832784FBB356F702032704F7E9
:10EFF4008327C4FBB355F702032744F7832784FA16
:10F00400B357F7022320F100938805001388060004
:10F01400832784FA0327C4FB832684FB97B509005E
:10F0240093854530EFF0064FEF50812A032784FB88
:10F034008327C4FB3307F702832784FAB307F70255
:10F04400032784F46372F70297B609009386863225
:10F0540017B609001306466C9305901C17B50900F2
:10F064001305C5DAEFE08671032784FB832744F593
:10F0740063F2E70297B609009386C63217B6090011
:10F08400130686699305A01C17B50900130505D856
:10F09400EFE0C66E0327C4FB832704F563F2E7029F
:10F0A40097B609009386863117B609001306C6661B
:10F0B4009305B01C17B50900130545D5EFE0066CA0
:10F0C400032784FA8327C4F463F2E70297B609009E
:10F0D4009386463017B60900130606649305C01CD0
:10F0E40017B50900130585D2EFE046690327C4F676
:10F0F400832784FBB377F7026382070297B609007C
:10F104009386C62E17B60900130606619305F01CF4
:10F1140017B50900130585CFEFE04666032704F70A
:10F124008327C4FBB377F7026382070297B609000B
:10F134009386462D17B609001306065E9305001D37
:10F1440017B50900130585CCEFE04663032744F7A0
:10F15400832784FAB377F7026382070297B609001C
:10F164009386C62B17B609001306065B9305101D7C
:10F1740017B50900130585C9EFE04660232204FA98
:10F18400232004FA232E04F86F009010832784F0C0
:10F1940083A7070103A747018327C4F9939757005F
:10F1A400B307F7002324F4F2832784F083A68701AE
:10F1B4000327C4F99307070093971700B387E70061
:10F1C40093973700B387F6002322F4F2832744F29F
:10F1D40083A74701639A070E97270C009387C7D824
:10F1E40003A7070083A74700B7160000B376D7002C
:10F1F4002324D4E693F707002326F4E6832684E643
:10F204000327C4E693870600B3E7E7006388070A89
:10F21400EF50410A9306300017B60900130646C1A1
:10F224009305C01D17B509001305054FEF5001786C
:10F2340097270C009387C7D283A707006388070228
:10F2440097F70B0083A7474883A7070083A7C70046
:10F2540093860700130640029305100017B50900B2
:10F264001305451DEF0097046F00C00297F70B00CC
:10F2740083A7874583A7070083A7C7009386070052
:10F28400130670019305100017B509001305051D39
:10F29400EF00D70197F70B0083A7074383A7070065
:10F2A40083A7C7000326C4F997B509009385851C75
:10F2B40013850700EFF00626EF5081019307C0FC89
:10F2C400232CF4F86F00903B832784F203A7870173
:10F2D40093072000630AF702832784F203A78700B9
:10F2E400B71700009387C719630EF778832784F252
:10F2F40003A78701930710006316F778832744F266
:10F3040083A7070163800778832744F283A7070153
:10F3140083A70700232EF4F0832784F203A7870131
:10F32400930720006316F73E232004F86F00800340
:10F334008327C4F183A7870203A78700832704F8E0
:10F3440093972700B307F70003A707008327C4F0A8
:10F3540083A7C7006304F702832704F89387170081
:10F364002320F4F88327C4F183A7870283A7070126
:10F37400032704F8E36EF7FA6F008000130000001F
:10F384008327C4F183A7870283A70701032704F80F
:10F394006362F70297B609009386461017B6090010
:10F3A400130686379305901E17B50900130505A6A5
:10F3B400EFE0C63C8327C4F183A7870203A7870035
:10F3C400832704F893972700B307F70083A7070060
:10F3D40083A78708639A071097270C009387C7B8F9
:10F3E40003A7070083A74700B7160000B376D7002A
:10F3F4002320D4E693F707002322F4E6832604E6C9
:10F40400032744E693870600B3E7E7006388070C05
:10F41400EF40516A9306300017B60900130646A15F
:10F424009305901E17B509001305052FEF500158D9
:10F4340097270C009387C7B283A707006388070246
:10F4440097F70B0083A7472883A7070083A7C70064
:10F4540093860700130620029305100017B50900D0
:10F4640013050506EF0087646F00C00297F70B00D1
:10F4740083A7872583A7070083A7C7009386070070
:10F48400130650019305100017B5090013058505EF
:10F49400EF00C76197F70B0083A7072383A7070033
:10F4A40083A6C7008327C4F183A7870203A7870025
:10F4B400832704F893972700B307F70083A707006F
:10F4C40083A707171386070097B5090093850503DB
:10F4D40013850600EFF00604EF40915F930750FC9C
:10F4E400232CF4F86F0090198327C4F103A7470471
:10F4F400832704F893972700B307F70083A707002F
:10F5040093F72700639C070E97270C009387C7A5E2
:10F5140003A7070083A74700B7160000B376D700F8
:10F52400232CD4E493F70700232EF4E4832684E504
:10F534000327C4E593870600B3E7E700638A070A55
:10F54400EF4051579306300017B609001306468E54
:10F554009305901E17B509001305051CEF500145CE
:10F5640097270C009387C79F83A707006388070228
:10F5740097F70B0083A7471583A7070083A7C70046
:10F58400938607001306B0029305100017B509000F
:10F59400130505F9EF0087516F00C00297F70B00C0
:10F5A40083A7871283A7070083A7C7009386070052
:10F5B4001306E0019305100017B50900130505F9BA
:10F5C400EF00C74E97F70B0083A7071083A7070028
:10F5D40083A7C700938607001306F0029305100063
:10F5E40017B50900130585F8EF00474CEF40514E5D
:10F5F400930760FF232CF4F86F0050088327C4F1AD
:10F6040003A74704832704F893972700B307F70059
:10F6140083A7070093F71700639C073A97270C000A
:10F624009387879403A7070083A74700B7160000B2
:10F63400B376D7002328D4E493F70700232AF4E40D
:10F64400832604E5032744E593870600B3E7E70030
:10F65400638A070AEF4011469306300017A6090093
:10F664001306067D9305901E17B509001305C50AF8
:10F67400EF50C13397270C009387878E83A7070029
:10F684006388070297F70B0083A7070483A7070083
:10F6940083A7C70093860700130630029305100062
:10F6A40017B50900130585EFEF0047406F00C0024E
:10F6B40097F70B0083A7470183A7070083A7C70019
:10F6C40093860700130660019305100017B509001F
:10F6D400130505EFEF00873D97F70B0083A7C7FEDF
:10F6E40083A7070083A7C700938607001306F002C9
:10F6F4009305100017B50900130505EEEF00073B4D
:10F70400EF40113D930780FD232CF4F86F00007740
:10F714008327C4F183A7C703638A07108327C4F12F
:10F7240003A7C7018327C4F083A7C70083A7C70B18
:10F73400B377F702638C070E97270C009387C78271
:10F7440003A7070083A74700B7160000B376D700C6
:10F754002324D4E493F707002326F4E4832684E4E3
:10F764000327C4E493870600B3E7E700638A070A24
:10F77400EF4051349306300017A609001306466B78
:10F784009305D01E17B50900130505F9EF500122A2
:10F7940097170C009387C77C83A707006388070229
:10F7A40097F70B0083A747F283A7070083A7C70037
:10F7B400938607001306D0029305100017B50900BD
:10F7C400130585E4EF00872E6F00C00297F70B0046
:10F7D40083A787EF83A7070083A7C7009386070043
:10F7E400130600029305100017B509001305C5E4BC
:10F7F400EF00C72B97F70B0083A707ED83A707003C
:10F8040083A7C7009386070013061003930510000F
:10F8140017B50900130585E4EF004729EF40512B84
:10F82400930730FF232CF4F86F0040658327C4F15D
:10F8340083A7C703638607040327C4F1832744F21D
:10F8440083A707010327C70323A0E7008327C4F185
:10F8540083A7C7012320F4E4232204E4832744F28A
:10F86400832604E4032744E423A4D70023A6E70063
:10F874008327C4F183A7C703232EF4F06F0080010C
:10F88400832744F2930600001307000023A4D70043
:10F8940023A6E7008327C4F183A78701232CF4E27E
:10F8A400232E04E28327C4F083A7C70003A7070815
:10F8B40083A74708032584E38325C4E3138605004F
:10F8C4009386070063EEC60013860500938607003F
:10F8D4006310D610930605009307070063FAD70E4A
:10F8E40097170C009387476803A7070083A747006F
:10F8F400B7160000B376D7002328D4E293F70700A5
:10F90400232AF4E2832604E3032744E393870600CF
:10F91400B3E7E7006388070AEF40D1199306300084
:10F9240017A609001306C6509305801F17B50900D2
:10F93400130585DEEF50810797170C009387476204
:10F9440083A707006388070297F70B0083A7C7D72D
:10F9540083A7070083A7C700938607001306100236
:10F964009305100017B50900130585D2EF0007149D
:10F974006F00C00297F70B0083A707D583A7070082
:10F9840083A7C70093860700130640019305100060
:10F9940017B50900130505D2EF00471197F70B00BF
:10F9A40083A787D283A7070083A7C7000326C4F9C8
:10F9B40097B50900938585D113850700EFE0963547
:10F9C400EF4011119307B0FF232CF4F86F00004BA4
:10F9D400832704FA138717002320E4FA0327C4F1CA
:10F9E400832604F693972700B387F60023A0E70045
:10F9F4008327C4F113850700EF609F878327C4F131
:10FA040083A74703639807008327C4F1032784F679
:10FA140023AAE7028327C4F183A74703638E07045D
:10FA24008327C4F183A7470303A7871A8327C4F056
:10FA340083A7C70083A7871A6300F704832744FAC0
:10FA4400138717002322E4FA93972700032784F5EA
:10FA5400B307F7001306C4F19388070013080000E6
:10FA6400930700009306000013070000930510009D
:10FA74000325C4F0EFB090498327C4F1032784F62B
:10FA840023AAE7028327C4F993871700232EF4F8E7
:10FA9400832784F083A7070183A707000327C4F9FA
:10FAA4006366F7EE832744EF63860702832744FAED
:10FAB40093972700032784F53307F700832744EF40
:10FAC4009397270013860700832504EF1305070087
:10FAD400EF10470D032744FA832744EFB307F700D9
:10FAE40013860700032744FA832744EFB307F7007C
:10FAF40063860700832784F56F0080009307000066
:10FB0400032704FA832604F6130504F293880600F7
:10FB140013080700130706008326040037160000A5
:10FB24001306061F8325C4F0EFF05030232CA4F8ED
:10FB3400832784F963920734832704F2371700007C
:10FB44001307071F23ACE704832704F2032784F079
:10FB540023A4E700832704F2032784FB23A2E702FC
:10FB6400832704F20327C4FB23A4E702832704F2B8
:10FB7400032784FA23A6E702832704F2032744F029
:10FB840023AEE702832704F28326C4F6032784FB0B
:10FB940033D7E60223A6E700832704F2832604F77B
:10FBA4000327C4FB33D7E60223A8E700832704F224
:10FBB400832644F7032784FA33D7E60223AAE7000F
:10FBC400832704F20327C4FA23ACE700832704F253
:10FBD400032704FB23AEE700832704F2032744FB37
:10FBE40023A0E702832784F083A7C700832584F634
:10FBF40013850700EF7001772328A4F2832704F309
:10FC040063D2070297B60900938606B017B60900B7
:10FC1400130686B09305602317A509001305051F75
:10FC2400EFD0D635832704F2032704F323A8E7068D
:10FC3400832784F083A7070183A6C702832704F3DD
:10FC440013974700832704F23387E60023A0E700D5
:10FC5400832784F083A7070103A7070093070700FE
:10FC640093971700B387E70093973700832404F230
:10FC740013850700EF0087499307050023A0F404C8
:10FC8400232E04F86F00C017832704F283A6070409
:10FC94000327C4F99307070093971700B387E70076
:10FCA40093973700B387F6002326F4F2832784F072
:10FCB40083A687010327C4F99307070093971700C6
:10FCC400B387E70093973700B387F60003A70700CD
:10FCD40083A74700232EE4F68327C4F72324F4E202
:10FCE400232604E28327C4F2832684E20327C4E2A2
:10FCF40023A0D70023A2E700832784F083A68701EB
:10FD04000327C4F99307070093971700B387E70005
:10FD140093973700B387F60003A7870083A7C7002C
:10FD24008326C4F223A4E60023A6F600832784F0E6
:10FD340083A687010327C4F9930707009397170045
:10FD4400B387E70093973700B387F60083A70701CB
:10FD5400639807008327C4F223A807006F00800973
:10FD64000325C4F7EFE01063232CA4F6032784F7DC
:10FD74009307F00763F6E70093070008232CF4F6D3
:10FD84000327C4F7832784F76376F700832784F770
:10FD9400232EF4F68325C4F7032584F7EFF0000738
:10FDA400130705008327C4F223A8E7008327C4F2BE
:10FDB40003A50701832784F083A687010327C4F9D9
:10FDC4009307070093971700B387E70093973700CB
:10FDD400B387F60083A607018327C4F203A70700AD
:10FDE40083A747009307070013860700938506003F
:10FDF400EF00575B8327C4F993871700232EF4F889
:10FE0400832784F083A7070183A707000327C4F986
:10FE1400E36CF7E6832704F223AE0704032584F09A
:10FE2400EF30020F97F70B0083A7478A83A70700D9
:10FE340063880702832704F283A747061385070014
:10FE4400EF60016F032584F0EF30820C832704F206
:10FE540083A7470683A7C705032784F023A0E700E9
:10FE6400832704F2938507000325C4F0EFF01048BC
:10FE7400232C04F86F00800013000000832784F90A
:10FE8400032144E213850700130104E18320C11E0A
:10FE94000324811E8324411E0329011E8329C11DBD
:10FEA400032A811D832A411D032B011D832BC11CA1
:10FEB400032C811C832C411C032D011C832DC11B8D
:10FEC4001301011F67800000130101FE232E11009E
:10FED400232C8100130401022326A4FE2324B4FE50
:10FEE4002322C4FE832684FE6396060E8326C4FE64
:10FEF4006382060E97170C009387070703A7070072
:10FF040083A74700B71600003373D70093F30700A5
:10FF140093070300B3E77700638A070AEF40813948
:10FF24009306300017B609001306C6819305700FB7
:10FF340017B509001305C58CEF40512797170C001E
:10FF44009387070283A707006388070297E70B00DC
:10FF540083A7877783A7070083A7C7009386070033
:10FF64001306E0019305100017A509001305057E8B
:10FF7400EFF0D6336F00C00297E70B0083A7C77476
:10FF840083A7070083A7C700938607001306100101
:10FF94009305100017A509001305457DEFF01631F0
:10FFA40097E70B0083A7477283A7070083A7C700BF
:10FFB40017A609001306C67C97A509009385C57E7C
:10FFC40013850700EFE00655EF408130930720FECC
:10FFD4006F004021832684FE6386060E8326C4FEBA
:10FFE4006392060E97170C00938707F803A7070080
:0CFFF40083A74700B71600003378D70041
:02000004800179
:1000000093F8070093070800B3E71701638A070A0C
:10001000EF40812A9306300017A609001306C67226
:100020009305A00F17A509001305C57DEF405118D2
:1000300097170C00938707F383A7070063880702CD
:1000400097E70B0083A7876883A7070083A7C700EC
:10005000938607001306E0019305100017A5090019
:100060001305056FEFF0D6246F00C00297E70B0071
:1000700083A7C76583A7070083A7C70093860700E8
:10008000130610019305100017A509001305456E0E
:10009000EFF0162297E70B0083A7476383A70700BB
:1000A00083A7C70017A609001306867097A5090045
:1000B0009385C56F13850700EFE00646EF40812169
:1000C000930720FE6F004012832644FE6396060EBF
:1000D0008326C4FE6392060E97160C00938606E9EB
:1000E00003A6060083A64600B71500003377B600C6
:1000F00093F7060093060700B3E6F600638A060A44
:10010000EF40811B9306300017A609001306C66353
:100110009305D00F17A509001305C56EEF405109CF
:1001200097170C00938707E483A7070063880702EB
:1001300097E70B0083A7875983A7070083A7C7000A
:10014000938607001306E0019305100017A5090028
:1001500013050560EFF0D6156F00C00297E70B009E
:1001600083A7C75683A7070083A7C7009386070006
:10017000130610019305100017A509001305455F2C
:10018000EFF0161397E70B0083A7475483A70700E8
:1001900083A7C70017A609001306066497A50900E0
:1001A0009385C56013850700EFE00637EF408112A5
:1001B000930720FE6F004003832784FE638A0700B5
:1001C000832784FE17E70B00130787A323A0E7000C
:1001D000832744FE63880700832744FE130710002B
:1001E00023A0E70093070000138507008320C101C7
:1001F000032481011301010267800000130101F84B
:10020000232E1106232C8106232A210723283107B8
:100210002326410723245107232261072320710746
:10022000232E8105232C9105232AA1052328B1051E
:10023000130401082326A4FA2324B4FA2322C4FABF
:100240002320D4FA232EE4F88327C4FA6392070EFE
:1002500097170C00938787D103A7070083A7470050
:10026000B71600003378D70093F80700930708000B
:10027000B3E71701638A070AEF40010493063000D1
:1002800017A60900130646599305700217A5090021
:100290001305457AEF40C17197170C00938787CCFF
:1002A00083A707006388070297E70B0083A707422D
:1002B00083A7070083A7C7009386070013061002D1
:1002C0009305100017A5090013058555EFF0467E2C
:1002D0006F00C00297E70B0083A7473F83A7070083
:1002E00083A7C700938607001306400193051000FB
:1002F00017A5090013050555EFF0867B97E70B005E
:1003000083A7C73C83A7070083A7C70017A60900D8
:100310001306C65497A509009385855513850700D4
:10032000EFE0861FEF30117B930700FE6F00D006D1
:10033000930744FB13060000938507001305100084
:10034000EFF0DFB8832744FB0327C4FA630AF70EF4
:1003500097170C00938787C103A7070083A747005F
:10036000B7160000B376D7002328D4F893F7070018
:10037000232AF4F8832604F9032744F99387060017
:10038000B3E7E700638A070AEF3011739306300082
:1003900017A60900130646489305A00217A50900F1
:1003A00013054569EF40C16097170C00938787BB21
:1003B00083A707006388070297E70B0083A707312D
:1003C00083A7070083A7C7009386070013061002C0
:1003D0009305100017A5090013058544EFF0466D3D
:1003E0006F00C00297E70B0083A7472E83A7070083
:1003F00083A7C700938607001306400193051000EA
:1004000017A5090013050544EFF0866A97E70B006E
:1004100083A7C72B83A7070083A7C700938607007E
:100420001306D0029305100017A509001305854493
:10043000EFF00668EF30116A930700FE6F00C07599
:10044000032784FAB7F7FFFF93870770B307F70016
:10045000130700026360F7741397270097A709003A
:1004600093870755B307F70003A7070097A709006D
:1004700093870754B307F700678007009307D000FE
:10048000232CF4FA832704FA638A0710032744FA1B
:10049000832784FB637AF70E97170C00938707ADC9
:1004A00003A7070083A74700B7160000B376D7005D
:1004B0002324D4F893F707002326F4F8832684F83E
:1004C0000327C4F893870600B3E7E700638A070AA7
:1004D000EF30915E9306300017A609001306C6336D
:1004E0009305200317A509001305C554EF40414C9F
:1004F00097170C00938707A783A707006388070255
:1005000097E70B0083A7871C83A7070083A7C70073
:10051000938607001306E0019305100017A5090054
:1005200013054538EFF0C6586F00C00297E70B007F
:1005300083A7C71983A7070083A7C700938607006F
:10054000130610019305100017A509001305853740
:10055000EFF0065697E70B0083A7471783A707001E
:1005600083A7C700832684FB032644FA97A50900C6
:100570009385853613850700EFD0167AEF309155B5
:10058000930720FE6F004061032684FB97A50900B6
:1005900093850538032504FAEF0007618327C4F922
:1005A000638807008327C4F9032784FB23A0E7009F
:1005B000930700006F00405E93072005232EF4FA96
:1005C000832704FA63820710032744FA8327C4FBB6
:1005D0006372F70E97170C009387479903A70700DC
:1005E00083A74700B7160000337DD70093FD0700AF
:1005F00093070D00B3E7B701638A070AEF30D14BC9
:100600009306300017A60900130606219305600320
:1006100017A5090013050542EF40813997170C0013
:100620009387479483A707006388070297E70B0027
:1006300083A7C70983A7070083A7C700938607007E
:100640001306E0019305100017A509001305852581
:10065000EFF006466F00C00297E70B0083A707077D
:1006600083A7070083A7C70093860700130610011E
:100670009305100017A509001305C524EFF04643A4
:1006800097E70B0083A7870483A7070083A7C7000A
:100690008326C4FB032644FA97A509009385C52346
:1006A00013850700EFD05667EF30D142930720FE45
:1006B0006F00804E0326C4FB97A50900938545264D
:1006C000032504FAEF00474E8327C4F96388070027
:1006D0008327C4F90327C4FB23A0E7009307000086
:1006E0006F00804B9307C0012320F4FC832704FA9A
:1006F00063820710032744FA832704FC6372F70E12
:1007000097170C009387878603A7070083A74700E6
:10071000B7160000337CD70093FC070093070C004A
:10072000B3E79701638A070AEF3011399306300067
:1007300017A609001306460E9305100817A5090011
:100740001305452FEF40C12697170C00938787812B
:1007500083A707006388070297E70B0083A707F7C3
:1007600083A7070083A7C700938607001306E0014D
:100770009305100017A509001305C512EFF04633C5
:100780006F00C00297E70B0083A747F483A7070019
:1007900083A7C70093860700130610019305100076
:1007A00017A5090013050512EFF0863097E70B0037
:1007B00083A7C7F183A7070083A7C700832604FC8C
:1007C000032644FA97A509009385051113850700B0
:1007D000EFD09654EF301130930720FE6F00C03BEE
:1007E000032604FC97A509009385C518032504FA80
:1007F000EF00873B8327C4F9638807008327C4F988
:10080000032704FC23A0E700930700006F00C03813
:10081000930710012322F4FC832704FA6382071054
:10082000032744FA832744FC6372F70E97070C00F2
:100830009387C77303A7070083A74700B716000075
:10084000337BD70093FB070093070B00B3E77701D7
:10085000638A070AEF3051269306300017A6090075
:10086000130686FB9305400817A509001305851C90
:10087000EF40011497070C009387C76E83A707000A
:100880006388070297E70B0083A747E483A7070065
:1008900083A7C700938607001306E00193051000A5
:1008A00017A5090013050500EFF086206F00C002B0
:1008B00097E70B0083A787E183A7070083A7C700FB
:1008C00093860700130610019305100017A5090071
:1008D000130545FFEFF0C61D97E70B0083A707DF61
:1008E00083A7070083A7C700832644FC032644FA96
:1008F00097A50900938545FE13850700EFD0D641E3
:10090000EF30511D930720FE6F000029032644FCA1
:1009100097A509009385C507032504FAEF00C728AA
:100920008327C4F9638807008327C4F9032744FC9D
:1009300023A0E700930700006F0000269307100034
:100940002324F4FC832704FA63820710032744FA64
:10095000832784FC6372F70E97070C009387076167
:1009600003A7070083A74700B7160000337AD70014
:1009700093FA070093070A00B3E75701638A070A4F
:10098000EF3091139306300017A609001306C6E84E
:100990009305C00817A509001305C509EF404101DB
:1009A00097070C009387075C83A7070063880702FB
:1009B00097E70B0083A787D183A7070083A7C7000A
:1009C000938607001306E0019305100017A50900A0
:1009D000130545EDEFF0C60D6F00C00297E70B0061
:1009E00083A7C7CE83A7070083A7C7009386070006
:1009F000130610019305100017A50900130585ECD7
:100A0000EFF0060B97E70B0083A747CC83A70700FF
:100A100083A7C700832684FC032644FA97A5090010
:100A2000938585EB13850700EFD0162FEF30910AE1
:100A3000930720FE6F004016032684FC97A509004B
:100A4000938545F6032504FAEF0007168327C4F9BA
:100A5000638807008327C4F9032784FC23A0E700E9
:100A6000930700006F004013930750002326F4FC07
:100A7000832704FA63820710032744FA8327C4FC00
:100A80006372F70E97070C009387474E03A7070082
:100A900083A74700B71600003379D70093F9070002
:100AA00093070900B3E73701638A070AEF30D100E3
:100AB0009306300017A60900130606D69305000911
:100AC00017A50900130505F7EF30916E97070C0085
:100AD0009387474983A707006388070297E70B00BE
:100AE00083A7C7BE83A7070083A7C7009386070015
:100AF0001306E0019305100017A50900130585DA18
:100B0000EFE0167B6F00C00297E70B0083A707BCDE
:100B100083A7070083A7C700938607001306100169
:100B20009305100017A509001305C5D9EFE0567805
:100B300097E70B0083A787B983A7070083A7C700A0
:100B40008326C4FC032644FA97A509009385C5D8DB
:100B500013850700EFD0561CEF30C177930720FEB6
:100B60006F0080030326C4FC97A509009385C5E3A5
:100B7000032504FAEF0047038327C4F963880700BD
:100B80008327C4F90327C4FC23A0E70093070000D0
:100B90006F008000930720FE138507008320C107A4
:100BA000032481070329410783290107032AC1067A
:100BB000832A8106032B4106832B0106032CC105E2
:100BC000832C8105032D4105832D010513010108A7
:100BD00067800000130101FC232E1102232C8102E7
:100BE000232A21032328310313040104232EA4FC08
:100BF0002328B4FC232AC4FC232CD4FC2326E4FCA5
:100C00002324F4FC232404FE232604FE8327C4FDAE
:100C10006392070E97070C009387473503A70700D9
:100C200083A74700B7160000337ED70093FE070066
:100C300093070E00B3E7D701638A070AEF30C16755
:100C40009306300017A60900130606E093059002EC
:100C500017A50900130585F0EF30915597070C0093
:100C60009387473083A707006388070297E70B0045
:100C700083A7C7A583A7070083A7C700938607009C
:100C8000130610029305100017A50900130545DC93
:100C9000EFE016626F00C00297E70B0083A707A37F
:100CA00083A7070083A7C7009386070013064001A8
:100CB0009305100017A509001305C5DBEFE0565F8B
:100CC00097E70B0083A787A083A7070083A7C70028
:100CD00017A60900130686DB97A50900938545DC56
:100CE00013850700EFD05603EF30C15E930700FE77
:100CF0006F004037832784FD6396070E8327C4FC6B
:100D00006382070E97070C009387472603A7070007
:100D100083A74700B71600003373D70093F307008B
:100D200093070300B3E77700638A070AEF30C158DF
:100D30009306300017A60900130606D19305B002EA
:100D400017A50900130585E1EF30914697070C00C0
:100D50009387472183A707006388070297E70B0063
:100D600083A7C79683A7070083A7C70093860700BA
:100D70001306E0019305100017A50900130585D29D
:100D8000EFE016536F00C00297E70B0083A70794AC
:100D900083A7070083A7C7009386070013061001E7
:100DA0009305100017A509001305C5D1EFE05650B3
:100DB00097E70B0083A7879183A7070083A7C70046
:100DC00017A60900130646D197A50900938545CDBE
:100DD00013850700EFD04674EF30C14F930720FE14
:100DE0006F004028832784FC6396070E8327C4FC8A
:100DF0006392070E97070C009387471703A7070016
:100E000083A74700B71600003378D70093F8070090
:100E100093070800B3E71701638A070AEF30C14957
:100E20009306300017A60900130606C29305C002F8
:100E300017A50900130585D2EF30913797070C00ED
:100E40009387471283A707006388070297E70B0081
:100E500083A7C78783A7070083A7C70093860700D8
:100E60001306E0019305100017A50900130585C3BB
:100E7000EFE016446F00C00297E70B0083A70785D9
:100E800083A7070083A7C7009386070013061001F6
:100E90009305100017A509001305C5C2EFE05641E0
:100EA00097E70B0083A7878283A7070083A7C70064
:100EB00017A609001306C6C497A50900938545BE69
:100EC00013850700EFD04665EF30C140930720FE41
:100ED0006F004019930704FE130600009385070076
:100EE00013051000EFE09FFE832704FE0327C4FDD7
:100EF0006302F70E97070C009387470703A70700C5
:100F000083A74700B71600003379D70093F907008D
:100F100093070900B3E73701638A070AEF30C13945
:100F20009306300017A60900130606B29305F002D7
:100F300017A50900130585C2EF30912797070C000C
:100F40009387470283A707006388070297D70B00A0
:100F500083A7C77783A7070083A7C70093860700E7
:100F6000130610029305100017A50900130545AEDE
:100F7000EFE016346F00C00297D70B0083A7077508
:100F800083A7070083A7C7009386070013064001C5
:100F90009305100017A509001305C5ADEFE0563104
:100FA00097D70B0083A7877283A7070083A7C70083
:100FB000938607001306F0029305100017A5090099
:100FC0001305C5B6EFE0D62EEF30C130930700FE13
:100FD0006F004009EF80C10F2322A4FE832744FE47
:100FE00063860700832744FE6F00C007032504FDC6
:100FF000832544FDEF70D120930705002324F4FEE0
:10100000832784FE639607009307F0FF6F00800537
:101010008327C4FC63800702832684FD0326C4FC67
:10102000032504FD832544FDEF705103930705005C
:101030002326F4FE832784FC63880700032784FEAD
:10104000832784FC23A0E7008327C4FE6346F000C7
:10105000832784FD63960700930700006F008000DC
:101060009307F0FF138507008320C1030324810346
:101070000329410383290103130101046780000050
:10108000130101812326117E2324817E2322217FC7
:101090002320317F232E417D232C517D232A617D06
:1010A0002328717D2326817D2324917D2322A17D08
:1010B0002320B17D1304017F130101F8232EA4A482
:1010C000232CB4A4232AC4A42328D4A42326E4A430
:1010D0008327C4A56392070E97070C00938707E93F
:1010E00003A7070083A74700B71600003378D7008F
:1010F00093F8070093070800B3E71701638A070A0C
:10110000EF30811B9306300017A60900130646A690
:101110009305E00317A50900130505D3EF30510926
:1011200097070C00938707E483A7070063880702EB
:1011300097D70B0083A7875983A7070083A7C7000A
:10114000938607001306F0019305100017A5090008
:10115000130585A2EFE0D6156F00C00297D70B00EC
:1011600083A7C75683A7070083A7C70093860700F6
:10117000130620019305100017A509001305C5A14A
:10118000EFE0161397D70B0083A7475483A70700F8
:1011900083A7C70017A60900130646A197A5090053
:1011A000938505A213850700EFD00637EF30811233
:1011B0009307F0FD6F70D075032784A5B717000063
:1011C0009387B70563E8E704032784A5B7170000F2
:1011D0006374F7006F709073032784A5B7F7FFFF60
:1011E0003307F7009307B00563F4E7006F701072E0
:1011F0001317270097A70900938707AEB307F700D7
:1012000003A7070097A70900938707ADB307F70067
:1012100067800700032784A5B74700009387070E60
:101220006314F7006F70C0676F70506E93074000D3
:101230002326F4EA832704A563880710032744A51F
:101240008327C4EA637AF70E97070C00938707D2C7
:1012500003A7070083A74700B7160000B376D7009F
:101260002320D4A493F707002322F4A4832604A404
:10127000032744A493870600B3E7E700638A070ABD
:10128000EF3081039306300017A609001306468E3F
:101290009305300417A50900130505BBEF30417114
:1012A00097070C00938707CC83A707006388070282
:1012B00097D70B0083A7874183A7070083A7C700A1
:1012C000938607001306E0019305100017A5090097
:1012D0001305458FEFE0C67D6F00C00297D70B0066
:1012E00083A7C73E83A7070083A7C700938607008D
:1012F000130610019305100017A509001305858E2C
:10130000EFE0067B97D70B0083A7473C83A7070036
:1013100083A7C7008326C4EA032644A597A509002E
:101320009385858D13850700EFD0061FEF20917AF6
:10133000930720FE6F70D05D8327C4A503A787089D
:10134000832704A523A0E7008327C4A4638807009C
:101350008327C4A40327C4EA23A0E700930700005F
:101360006F70105B930780002328F4E4832704A5A3
:10137000638C0710032744A5832704E5637AF70EDF
:1013800097070C00938787BE03A7070083A7470032
:10139000B7160000B376D700232CD4A293F707002A
:1013A000232EF4A2832684A30327C4A393870600D5
:1013B000B3E7E700638A070AEF2011709306300055
:1013C000179609001306C67A9305500417A509005D
:1013D000130585A7EF30C15D97070C00938787B889
:1013E00083A707006388070297D70B0083A7072E00
:1013F00083A7070083A7C700938607001306E001B1
:1014000093051000179509001305C57BEFE0466AA8
:101410006F00C00297D70B0083A7472B83A7070055
:1014200083A7C700938607001306100193051000D9
:10143000179509001305057BEFE0866797D70B002A
:1014400083A7C72883A7070083A7C700832604E5CF
:10145000032644A5979509009385057A138507000F
:10146000EFD0860BEF201167930720FE6F70504A74
:101470008327C4A503A7870083A7C700832604A5E5
:1014800023A0E60023A2F6008327C4A463880700F4
:101490008327C4A4032704E523A0E70093070000E3
:1014A0006F70104793074000232AF4E4832704A5B4
:1014B00063880710032744A5832744E5637AF70E62
:1014C00097070C00938787AA03A7070083A7470005
:1014D000B7160000B376D7002328D4A293F70700ED
:1014E000232AF4A2832604A3032744A39387060098
:1014F000B3E7E700638A070AEF20115C9306300028
:10150000179609001306C6669305700417A509000F
:1015100013058593EF30C14997070C00938787A483
:1015200083A707006388070297D70B0083A7071AD2
:1015300083A7070083A7C700938607001306E0016F
:1015400093051000179509001305C567EFE046568F
:101550006F00C00297D70B0083A7471783A7070028
:1015600083A7C70093860700130610019305100098
:101570001795090013050567EFE0865397D70B0011
:1015800083A7C71483A7070083A7C700832644E562
:10159000032644A5979509009385056613850700E2
:1015A000EFC09677EF201153930720FE6F705036EF
:1015B0008327C4A503A70701832704A523A0E70069
:1015C0008327C4A4638807008327C4A4032744E5B2
:1015D00023A0E700930700006F709033930740004B
:1015E000232CF4E4832704A563880710032744A56C
:1015F000832784E5637AF70E97070C009387079794
:1016000003A7070083A74700B7160000B376D700EB
:101610002324D4A293F707002326F4A2832684A2CE
:101620000327C4A293870600B3E7E700638A070A8B
:10163000EF20914893063000179609001306465391
:101640009305900417A5090013050580EF30413676
:1016500097070C009387079183A707006388070209
:1016600097D70B0083A7870683A7070083A7C70028
:10167000938607001306E0019305100017950900F3
:1016800013054554EFE0C6426F00C00297D70B0028
:1016900083A7C70383A7070083A7C7009386070014
:1016A00013061001930510001795090013058553C3
:1016B000EFE0064097D70B0083A7470183A70700F9
:1016C00083A7C700832684E5032644A597950900D0
:1016D0009385855213850700EFC01664EF20913F74
:1016E000930720FE6F70D0228327C4A503A747016C
:1016F000832704A523A0E7008327C4A463880700E9
:101700008327C4A4032784E523A0E70093070000F0
:101710006F70102093074000232EF4E4832704A564
:1017200063880710032744A58327C4E5637AF70E6F
:1017300097070C009387878303A7070083A74700B9
:10174000B7160000B376D7002320D4A293F7070082
:101750002322F4A2832604A2032744A2938706002F
:10176000B3E7E700638A070AEF20113593063000DC
:10177000179609001306C63F9305B0041795090094
:101780001305856CEF30C12297F70B009387877D97
:1017900083A707006388070297D70B0083A707F387
:1017A00083A7070083A7C700938607001306E001FD
:1017B00093051000179509001305C540EFE0462F6B
:1017C0006F00C00297D70B0083A747F083A70700DD
:1017D00083A7C70093860700130610019305100026
:1017E0001795090013050540EFE0862C97D70B00ED
:1017F00083A7C7ED83A7070083A7C7008326C4E597
:10180000032644A5979509009385053F1385070096
:10181000EFC09650EF20112C930720FE6F70500FF1
:101820008327C4A503A74702832704A523A0E700B5
:101830008327C4A4638807008327C4A40327C4E5BF
:1018400023A0E700930700006F70900C8327C4A5C6
:1018500083A787032322F4E6930740002320F4E6BE
:10186000832704A563860710032744A5832704E67E
:10187000637AF70E97F70B009387476F03A707006C
:1018800083A74700B7160000B376D700232CD4A057
:1018900093F70700232EF4A0832684A10327C4A175
:1018A00093870600B3E7E700638A070AEF20D12099
:1018B00093063000179609001306862B9305F00552
:1018C0001795090013054558EF30810E97F70B0067
:1018D0009387476983A707006388070297D70B00A0
:1018E00083A7C7DE83A7070083A7C70093860700E7
:1018F0001306E00193051000179509001305852CC8
:10190000EFE0061B6F00C00297D70B0083A707DC30
:1019100083A7070083A7C70093860700130610015B
:1019200093051000179509001305C52BEFE0461825
:1019300097D70B0083A787D983A7070083A7C70082
:10194000832604E6032644A5979509009385C52AB6
:1019500013850700EFC0563CEF20D117930720FEF8
:101960006F70007B832704A5032744E623A0E700CC
:101970008327C4A4638807008327C4A4032704E63D
:1019800023A0E700930700006F7080789307C000E2
:101990002324F4E6832704A563820712032744A5C2
:1019A000832784E6637AF70E97F70B009387075C2B
:1019B00003A7070083A74700B7160000B376D70038
:1019C0002328D4A093F70700232AF4A0832604A198
:1019D000032744A193870600B3E7E700638A070A59
:1019E000EF20910D93063000179609001306461854
:1019F000930550061795090013050545EF20517B07
:101A000097F70B009387075683A7070063880702A1
:101A100097D70B0083A787CB83A7070083A7C700AF
:101A2000938607001306E00193051000179509003F
:101A300013054519EFE0C6076F00C00297D70B00EA
:101A400083A7C7C883A7070083A7C700938607009B
:101A5000130610019305100017950900130585184A
:101A6000EFE0060597D70B0083A747C683A70700BB
:101A700083A7C700832684E6032644A5979509001B
:101A80009385851713850700EFC01629EF20910471
:101A9000930720FE6F70C0678327C4A51387C70212
:101AA000832704A58326070023A0D70083264700A9
:101AB00023A2D7000327870023A4E7008327C4A419
:101AC000638807008327C4A4032784E623A0E700D4
:101AD000930700006F70C0638327C4A503A607089F
:101AE00083A6470893070600B3E7D7006398070269
:101AF00097D70B0083A787BD83A7070083A7C700DD
:101B0000930680061796090013068612979509001A
:101B10009385C51313850700EFC016209307800037
:101B2000232AF4E8832704A5638C0710032744A520
:101B3000832744E9637AF70E97F70B0093870743EF
:101B400003A7070083A74700B7160000B376D700A6
:101B50002324D4A093F707002326F4A0832684A08F
:101B60000327C4A093870600B3E7E700638A070A48
:101B7000EF2081749306300017960900130646FF84
:101B800093058006179509001305052CEF20516277
:101B900097F70B009387073D83A707006388070229
:101BA00097D70B0083A787B283A7070083A7C70037
:101BB000938607001306E0019305100017950900AE
:101BC00013054500EFD0D66E6F00C00297D70B000B
:101BD00083A7C7AF83A7070083A7C7009386070023
:101BE000130610019305100017950900130585FFD2
:101BF000EFD0166C97D70B0083A747AD83A70700DC
